:100000000C948C0F0C94BD0F0C94BD0F0C94BD0F71
:100010000C94BD0F0C94BD0F0C94BD0F0C94BD0F30
:100020000C94BD0F0C94BD0F0C94BD0F0C94BD0F20
:100030000C94BD0F0C94BD0F0C94BD0F0C94BD0F10
:100040000C94BD0F0C94BD0F0C94BD0F0C94BD0F00
:100050000C94BD0F0C94BD0F0C94BD0F0C94429CDE
:100060000C94BD0F0C9469770C943F770C94BD0FE2
:100070000C94BD0F0C94BD0F0C94BD0F0C94BD0FD0
:100080000C94BD0F0C94BD0F0C94BD0F0C94BD0FC0
:100090000C94BD0F0C94BD0F0C94BD0F0C949622C4
:1000A0000C94BD0F0C94BD0F0C94BD0F0C94BD0FA0
:1000B0000C94BD0F0C94BD0F0C94BD0F0C94BD0F90
:1000C0000C94BD0F0C94BD0F0C94BD0F0C94BD0F80
:1000D0000C94BD0F0C94BD0F0C94BD0F0C94BD0F70
:1000E0000C94BD0F07634236B79BD8A71A396856E0
:1000F00018AEBAAB558C1D3CB7CC5763BD6DEDFD4A
:10010000753EF6177231BF000000803F0800000006
:10011000BE922449123EABAAAA2ABECDCCCC4C3EFC
:1001200000000080BEABAAAAAA3E00000000BF00EB
:100130000000803F0000000000084178D3BB4387E7
:10014000D1133D190E3CC3BD4282AD2B3E68EC82FB
:1001500076BED98FE1A93E4C80EFFFBE01C4FF7F80
:100160003F00000000000C9487550C9483110C9400
:10017000AA420C94F40F0C94F51C0C949E2C0C9435
:100180002A9A0C9402430C94696C0C94BF540C94FE
:10019000F1610C94CB7A0C941FB10C94566C0C94B6
:1001A00036140C94CC110C9441880C949AB40C9491
:1001B00050980C942E1D0C94664A0C94CB420C94CF
:1001C000FF6C0C94F7920C94AD310C94C6330C94E4
:1001D000DA150C942F550C94434A0C94D8470C9480
:1001E000F7700C94BE6E0C9459330C944F790C94A8
:1001F00090AC0C944A120C94E9920C94756F0C9488
:10020000D4920C94D5700C94615C0C947E880C9400
:10021000C2300C94A33D0C94DE0F0C9445640C94F6
:1002200094120C94AC140C94744A0C94D3780C94DF
:10023000E3920C94A26E0C94C4110C943D120C9495
:10024000BB180C94B5300C94CB300C945BB20C946E
:1002500009930C9430320C948D6F0C94E1B20C9491
:1002600084110C94E1540C9405930C94FA540C945E
:10027000CB1E0C94DC920C94774A0C9408100C94CE
:10028000C30F0C94966C0C9488790C9490100C9479
:1002900096140C9498120C9437330C945B880C943D
:1002A000DF190C94923D0C9448330C94B3130C94C6
:1002B0009A1D0C941E100C94D8920C9459760C94A0
:1002C000D96F0C941B330C94556F0C94BC300C9468
:1002D0007E360C9403540C94DC780C942F710C949F
:1002E000359A0C94EA530C94622C0C943C3D0C947B
:1002F000A1630C9401930C94C16D0C94B0310C94D7
:10030000101C0C94FB920C9464540C94822D0C944D
:10031000304A0C94A8180C94FEA70C947D100C94F1
:1003200021610C94C76D0C94096F0C9487110C9487
:10033000D70F0C94052D0C9497100C94106F0C94FF
:1003400013930C943B320C94D3110C94427C0C9478
:1003500037540C94DC150C9478310C9439430C947C
:1003600028100C94D8320C94CD6E0C9405420C9449
:10037000F3780C948D550C94C76C0C94082E0C9447
:10038000571E0C940E930C94B02C0C94834A0C942E
:100390004F420C948F330C94694A0C94CF990C946F
:1003A00077980C94AC320C9480980C9454140C9460
:1003B00043330C9401330C947E530C947A320C9496
:1003C000A6830C94F76E0C946E100C942D3D0C9437
:1003D0003D790C949D120C94C2490C94483F0C94A6
:1003E000E0920C949B190C9485490C94686C0C94C5
:1003F0001C4A0C948F640C94F8320C947C160C9468
:10040000C8990C94376E0C94153F0C949C320C9444
:10041000CE920C9416300C94B1630C94EB7C0C943B
:100420006D100C943F6F0C94B5110C94E64F0C9426
:1004300005190C94BE6D0C944C6D0C945A4A0C9496
:10044000DA300C9403700C94C70F0C94279A0C9418
:100450007C120C94046E0C945B2E0C94AC5B0C948C
:1004600048880C9407100C94EC2D0C94862C0C945A
:10047000FF0F0C9458330C94B4530C9483420C9497
:10048000ED920C943A140C944E3D0C94D2AA0C9418
:100490006C100C94D3B20C945C120C942CB20C948F
:1004A000CE180C94CD120C94C2780C9440130C947A
:1004B000722D0C94DE1B0C94C4100C94FD1B0C9438
:1004C000E54E0C947A980C94309A0C94BF0F0C94CF
:1004D0003AB20C948F350C94703E0C94B8B20C94D4
:1004E00098880C94C2320C9429330C947D540C944B
:1004F0009A120C94C6310C940EA40C94F3920C94A2
:1005000051320C945F880C94423E0C948C110C94E4
:1005100072180C94E7420C940F930C942D9A0C943F
:10052000506E0C949D6D0C94AC110C9486120C942E
:100530000A7D0C94ED240C94E6330C9426B20C94B2
:10054000876B0C94A56C0C94B76D0C942A100C94CA
:100550008D330C94C8130C94DF3E0C9465710C948D
:1005600093310C9413140C94D12D0C94F8A70C9483
:1005700012A60C94347D0C94AE550C946D320C94F0
:10058000B96C0C949CAD0C9475110C947C320C9449
:100590008A556364696E6F70737578585B004E415D
:1005A0004E494E495459494E46CDCCCC3D0AD723ED
:1005B0003C17B7D13877CC2B329595E6241FB14F35
:1005C0000A000020410000C84200401C4620BCBE7A
:1005D0004CCA1B0E5AAEC59D742F00496E3A2000BE
:1005E0003D00494E3A003D004C45474143592049A2
:1005F0004E3A00000020002300260029002C002F86
:10060000003200000100000301060109012D3E0037
:10061000200023002D3E00200050656E6465643A82
:100620002023007261770076616C0074656D700044
:10063000736174006875650066616E005247420020
:10064000485356006D6F646500536574436D643A9A
:100650000053746F726564204558543A0073756690
:10066000666978436F64653A00584F4E0048414CC4
:1006700054002074696D653A004374726C205265B1
:10068000733A002054533A0020543A003D00506918
:100690006E3A004F4E3A416C726561647920416355
:1006A000746976650A0048414C543A416C72656140
:1006B000647920496E6163746976650A00584F4E0B
:1006C0003A416C7265616479204163746976650AA8
:1006D00000584F464620736B69707065642E205039
:1006E00072657620636D643A005475726E6564209D
:1006F0006F66662066726F6D3A00526573746F7232
:1007000065642066726F6D3A0049676E6F7265644A
:100710002C206368616E6E656C20636D643D002003
:10072000457865633A004163746976653A004841EB
:100730004C543A416C726561647920496E6163740E
:100740006976650A00584F4E3A416C72656164796A
:10075000204163746976650A00584F464620736BE2
:1007600069707065642E205072657620636D643AFE
:10077000005475726E6564206F66662066726F6DD8
:100780003A00526573746F7265642066726F6D3AD9
:10079000004E6F7420656E6F756768206D656D6FB4
:1007A000727920666F722067726F7570206F706546
:1007B000726174696F6E00206D73203A0041726D32
:1007C000656420666F7220002044697361726D65F4
:1007D0006400536B697070656420686F6D69652093
:1007E0007374756666004F75744F664D656D6F72F4
:1007F00079210A002000205375623D00204974656C
:100800006D3D0052414D3D00282D292000282B2907
:1008100020002076616C7565206973200020756E5C
:100820006B6E6F776E0A005D3D005B0020696E762F
:10083000616C6964002000206F6B003A00206661E3
:10084000696C6564003A005265747279696E67205C
:100850006D6F6462757320434D440A0020736563B5
:100860002072656D61696E696E670053746174759D
:10087000732064656666657265640A0020002D3E1B
:1008800000436F6E76657274696E6720002D3E00BE
:1008900057726F6E672041737369676E6D656E7412
:1008A0002000524742783A2000485356206469732A
:1008B00061626C65640020764C6576656C3A002058
:1008C000436F6E76563A0020436F6E76533A00209F
:1008D000486F743A00436F6C643A0020436F6E7641
:1008E000657274656420563A00436F6E7665727463
:1008F000656420533A002D3E0057726F6E672041A9
:10090000737369676E6D656E7420002D3E005772BB
:100910006F6E672041737369676E6D656E7420003A
:1009200053617665643A0020537566663A0020414B
:10093000543A00436F6E666967206368616E67654D
:1009400064206C6F63616C6C792C20706F727461C1
:100950006C2064697361626C6564002F636F6E66FE
:1009600069672E6A736F6E007265626F6F74200024
:10097000436D643A20002F636F6D6D616E642F00CC
:100980002F72616D2F002F6974656D2F002F6974B0
:10099000656D2F004C6F636174696F6E3A206874E7
:1009A00074703A2F2F6C617A79686F6D652E72754D
:1009B0002F707761003F6D61633D002669703D00D7
:1009C00026706F72743D00266E616D653D002F00CC
:1009D0002000436F6D706C6574652E2052656D6FDD
:1009E000766520746F706963200024636F6D6D619C
:1009F0006E6400536B697070696E672E2E00436CD5
:100A000065616E55702072657461696E65642074ED
:100A10006F7069632000220022004F75744F664D8D
:100A2000656D6F727921005D20003A5B000A005D00
:100A300000456D7074793A205B000A003A004D4120
:100A4000433A00554450205379736C6F6720696EA8
:100A5000697469616C697A65642E0A005379736CF4
:100A60006F6720706172616D733A003E003C005404
:100A70003A0043757272656E74204C414E20636F6C
:100A80006E6669672869702C646E732C67772C73A7
:100A900075626E6574293A000A557365207468653D
:100AA000736520636F6D6D616E64733A20276865AE
:100AB0006C7027202D207468697320746578740A1F
:100AC000276D61632064653A61643A62653A6566E0
:100AD0003A66653A3030272073657420616E642071
:100AE00073746F7265204D41432D61646472657348
:100AF0007320696E20454550524F4D0A276970207A
:100B00005B69705B2C646E735B2C67775B2C737511
:100B1000626E65745D5D5D5D27202D2073657420B8
:100B20007374617469632049500A2773617665277D
:100B3000202D20736176652063757272656E742056
:100B4000636F6E66696720696E204E5652414D3B59
:100B5000204F4E7C4F4646202D20656E61626C65AD
:100B60002F64697361626C65206175746F7361765F
:100B7000650A2767657427205B636F6E6669672067
:100B8000616464725D27202D2067657420636F6E39
:100B90006669672066726F6D207072652D636F6E77
:100BA000666967757265642055524C20616E6420D9
:100BB00073746F726520616464722C204F4E7C4F99
:100BC0004646202D20656E61626C652F64697361F5
:100BD000626C6520646F776E6C6F6164206F6E204D
:100BE000737461727475700A276C6F616427202DAD
:100BF000206C6F616420636F6E6669672066726F38
:100C00006D204E5652414D0A2770776427202D20C3
:100C1000646566696E6520616E642073746F7265C9
:100C2000204D5154542070617373776F72640A279A
:100C30006F746170776427202D20646566696E6526
:100C400020616E642073746F726520485454502084
:100C50004150492070617373776F72640A276C6F1B
:100C600067205B73657269616C5F6C6F676C65763A
:100C7000656C5D205B7564705F6C6F676C65766535
:100C80006C5D27202D20646566696E65206C6F673A
:100C9000206C6576656C2028302E2E37290A276B4C
:100CA000696C6C27202D20746573742077617463E0
:100CB00068646F670A27636C65617227202D206363
:100CC0006C65617220454550524F4D0A277265622E
:100CD0006F6F7427202D207265626F6F7420636FB1
:100CE0006E74726F6C6C657200536F6674207265FF
:100CF000626F6F74696E672E2E2E0052414D3D005B
:100D00000A5379736C6F6720000A312D7769726519
:100D100020000A6D71747420000A696E7075747316
:100D200020000A6974656D7320000A436F6E66695E
:100D300067757265643A0020416464723A006465C4
:100D400076230009445332343832206572726F7250
:100D50000009526573657420646F6E65000943680D
:100D600065636B696E6720666F7220312D576972FB
:100D70006520646576696365732E2E2E00445332B8
:100D80003438322D3130302070726573656E7400E6
:100D90004572726F7220312D7720696E697420233D
:100DA0003220467265653A0077737461742E20466E
:100DB0007265653A005465726D2E20467265653A1B
:100DC000004572726F7220312D7720696E69742030
:100DD000233100467265653A004453323438325F3D
:100DE0003130305F4932435F544F5F31575F425279
:100DF0004944474520696E6974003B003D005069D5
:100E00006E3A003B003D4C4F5700546865726D6F61
:100E10003A004F6E6520776972652052656164798A
:100E20000A004170706C79696E6720636F6E666945
:100E300067004C6F6164656420455441473A004E39
:100E40006F2073746F72656420636F6E66696700EC
:100E50004C6F616465642066726F6D204545505229
:100E60004F4D006C6F6164206661696C6564004C75
:100E70006F6164696E6720436F6E66696720667292
:100E80006F6D20454550524F4D00436F6E66696748
:100E9000206175746F736176653A000A5379736CDB
:100EA0006F67206465627567206C6576656C3A00D3
:100EB00053657269616C206465627567206C657644
:100EC000656C3A0053617665640A0053657420646A
:100ED000796E616D69632049500A00454550524F53
:100EE0004D20636C65617265640A004D5154542055
:100EF00050617373776F7264207570646174656498
:100F00000A004F54412050617373776F72642075EB
:100F10007064617465640A00636F756C64206E6F41
:100F2000742070617273653A200055706461746555
:100F3000640A004E6F20495020616472657373002B
:100F400052656C656173696E6720736F636B65745E
:100F500020616E6420726574727900205361766539
:100F600064004C6F6164696E67204854545020637C
:100F70006F6E666967206F6E20737461727475702E
:100F80003A004F4646004F4E002B002D004554615D
:100F9000673A200047657420455441473A2000488D
:100FA0005454502F312E312025690025733A2025C5
:100FB000730D0A0020485454502F312E310D0A4829
:100FC0006F73743A2025730D0A4163636570743A38
:100FD000202A2F2A0D0A436F6E6E656374696F6E47
:100FE0003A20636C6F73650D0A0025730020000DB5
:100FF0000A00474554006661696C656420746F207F
:10100000636F6E6E6563740A004552524F523A2008
:101010005365727665722072657475726E656420B0
:1010200000436F6E666967206E6F74206368616E3F
:101030006765640A00446F6E652E0A00436F6E6632
:1010400069672070617273696E67206661696C659B
:10105000640A00676F7420436F6E6669670A0066F2
:101060007265652000436F6E666967205552493A84
:1010700020687474703A2F2F002044656661756C87
:101080007420636F6E66696720736572766572207F
:10109000757365643A20006C617A79686F6D652EAE
:1010A0007275000A282D294D554C544956454E5409
:1010B000000A282B2950574D5F52454C4159000AD0
:1010C000282D294D444E53000A282D2955415254AC
:1010D000425249444745000A282B295359534C4F43
:1010E00047000A282D29504944000A282D294D433C
:1010F000503233303137000A282D294152544E45A1
:1011000054000A282B294F5441000A282D295350F6
:1011100049204C4544000A282D294D4F544F522058
:10112000435452000A282D29414320484149455241
:10113000000A282D294343533831312026204844C2
:101140004331303830000A282B295245535441523C
:10115000545F4C414E5F4F4E5F4D5154545F45526A
:10116000524F5253000A282D2948415244524553A8
:1011700045542C207573696E6720736F6674000A7E
:10118000282D29434F554E544552000A282D2944F5
:101190004854000A282B294453323438322D313038
:1011A00030000A282B294F57495245000A282D297B
:1011B0004D4F44425553000A282D29444D58000AEA
:1011C000282B2957697A6E657435313030000A282A
:1011D0002B294672656552616D207072696E746963
:1011E0006E67000A282B295741544348444F470053
:1011F0000A4669726D77617265204D4143204164F2
:1012000064726573732064653A61643A62653A6535
:10121000663A66653A6566006C617A79686F6D65F5
:101220002E7275000A436F6E666967207365727669
:1012300065723A003230313130334C0020432B2B71
:101240002076657273696F6E3A00613935366236A1
:10125000665F323032322D31312D3139000A4C6126
:101260007A79686F6D652E7275204C69676874486D
:10127000756220636F6E74726F6C6C6572200020F3
:101280004F464600204F4E002042595041535300D4
:10129000757074696D65006672656568656170007A
:1012A0002054696D65723A00204C6F636B733A008D
:1012B0002000204C6F636B733A000A52414D3D0091
:1012C00020457870697265640A00202D7461726728
:1012D0006574207A6F6E652D0020416C61726D20FF
:1012E000457870697265640A0020636D643A002075
:1012F0004375723A00205365743A00536176656411
:1013000020746F20454550524F4D00536176696EF1
:101310006720636F6E66696720746F204545505281
:101320004F4D2E2E00206973200044656C65746952
:101330006E6720636F6E662E2052414D2077617379
:101340003A0053746F707065640053746F70706905
:101350006E67206368616E6E656C73202E2E2E00A2
:101360004E6F7420756E6C6F636B656420696E20C0
:10137000313073202D20636F6E74696E7565202E79
:101380002E2E00556E6C6F636B696E6720636F6EF7
:10139000666967202E2E2E0020696E6974005265E2
:1013A0006C61792D4F75742023002073746F700069
:1013B00052656C61792D4F75742023003D3E003AD3
:1013C0000070756220616374696F6E200069646CDF
:1013D00065006F66660068656174696E67006661C6
:1013E0006E00647279696E6700636F6F6C696E6717
:1013F0000020697320004F75742000556E6B6E6F6E
:10140000776E207375666669782000556E6B6E6F17
:10141000776E20636D642000616374696F6E007283
:10142000656C61794374723A200020416464723AB9
:1014300000646576230020616C69766500204E6F3C
:1014400064653A00312D7769726520636F756E743B
:101450003A2000312D776972652073686F72746568
:1014600064005B305D3A2000202D202D202D20EFE0
:10147000BBBF003E003E31202D200020002E006921
:101480006E00735F6F7574006D79686F6D65002015
:101490002D3E2000456D69743A2000202D3E20002D
:1014A0004974656D436D643A2000202D3E2000494B
:1014B00074656D3A2000005EBCE2613FDD83C29C32
:1014C0007E20A3FD1F419DC3217FFCA2401E5F0122
:1014D000E3BD3E6082DC237D9FC1421CFEA0E1BFD4
:1014E0005D0380DE3C62BEE0025CDF81633D7C2206
:1014F000C09E1D43A1FF4618FAA427799BC584DA34
:101500003866E5BB5907DB856739BAE406581947E1
:10151000A5FB7826C49A653BD987045AB8E6A7F993
:101520001B45C6987A24F8A6441A99C7257B3A64C5
:1015300086D85B05E7B98CD2306EEDB3510F4E10F3
:10154000F2AC2F7193CD114FADF3702ECC92D38DA1
:101550006F31B2EC0E50AFF1134DCE90722C6D3353
:10156000D18F0C52B0EE326C8ED0530DEFB1F0AE85
:101570004C1291CF2D73CA947628ABF517490856B3
:10158000B4EA6937D58B5709EBB536688AD495CB61
:101590002977F4AA4816E9B7550B88D6346A2B7513
:1015A00097C94A14F6A8742AC896154BA9F7B6E845
:1015B0000A54D7896B35436F6E6E65637465642E0C
:1015C00000436F6E6E2E2061626F72746564003E20
:1015D0003E2000496E76616C696420636F6D6D61B9
:1015E0006E64003E3E3E004E6F204D414320636FCF
:1015F0006E666967757265643A2073657420666902
:10160000726D776172652773204D41430A004E6FFA
:101610002076616C696420454550524F4D206461CD
:1016200074612E20496E697469616C697A696E67AC
:101630002E00476F74204950206164647265737393
:101640003A00276970205B69705B2C646E735B2CB9
:1016500067775B2C7375626E65745D5D5D5D2720D9
:101660002D20736574207374617469632049500A76
:10167000004661696C656420746F20636F6E6669F3
:10168000677572652045746865726E657420757340
:10169000696E6720444843502E20596F752063615E
:1016A0006E20736574206970206D616E75616C6C5D
:1016B0007921000A7573657320444843500A00205D
:1016C0004D41534B3A002047573A0020444E533A7D
:1016D000004C6F616465642066726F6D20666C619A
:1016E00073682049503A005374617274696E6720C0
:1016F0006C616E004142434445464748494A4B4C61
:101700004D4E4F505152535455565758595A616285
:10171000636465666768696A6B6C6D6E6F70717221
:10172000737475767778797A303132333435363769
:1017300038392B2F3D004261736963200061726468
:1017400075696E6F3A004F544120696E6974696122
:101750006C697A65640A0044454641554C542070D2
:10176000617373776F726420666F72204F544120EB
:101770004150492E20557365206F74617077642045
:10178000636F6D6D616E6420746F2073657400709B
:10179000617373776F726400546F6F206D616E793F
:1017A000204D51545420636F6E6E656374696F6E83
:1017B000206572726F72732E205265737461727439
:1017C000204C414E002074727920616761696E205F
:1017D000696E2035207365636F6E6473006661699E
:1017E0006C65642C2072633D004177616974696E99
:1017F0006720666F722072657461696E656420741B
:101800006F7069637300636F6E6E656374656420E7
:1018100061732000202E2E2E0020757365723A0011
:101820003A000A417474656D7074696E67204D5199
:10183000545420636F6E6E656374696F6E20746FAD
:101840002000646973636F6E6E6563746564005530
:1018500073696E67204D5154542070617373776FB4
:1018600072642066726F6D20636F6E6669670044F4
:101870006576696365204E616D653A004174206C40
:101880006561737420646576696365206E616D655A
:1018900020616E642062726F6B6572204950206D0A
:1018A00075737420626520636F6E66696775726513
:1018B0006400757074696D652C6672656568656134
:1018C0007000247374617473006139353662366652
:1018D0005F323032322D31312D3139004C69676839
:1018E000744875622000246E616D650072656164E4
:1018F000790024737461746500526562696E6420B6
:10190000737563636573732E20495020616464723C
:101910006573733A004572726F723A20726562693C
:101920006E64206661696C0052656E65776564203F
:10193000737563636573732E20495020616464720C
:101940006573733A004572726F723A2072656E6504
:10195000776564206661696C000A4E6F206C696E61
:101960006B00526573746F72696E6720636F6E6689
:1019700069672066726F6D20454550524F4D00419A
:101980006363657074696E6720636F6D6D616E640B
:10199000732E2E2E0A004E6F204D51545420636F2B
:1019A0006E66696775726564004C6F6164696E6725
:1019B00020636F6E6669672066726F6D20706F724C
:1019C00074616C2064697361626C65642E20757348
:1019D0006520676574204F4E20746F20656E6162CC
:1019E0006C6500436F6E6669672069732076616C71
:1019F000696400436F6E74696E75652077697468F9
:101A00002070726576696F75736C79206C6F616494
:101A1000656420636F6E6669670000002200250020
:101A200028002B002E0031003400020100000501C7
:101A300008010B0100000A0B02090C0D0E08070338
:101A40000401000000000000000000000000000091
:101A50000000000000000000000000000000000086
:101A60001211100000000000000000000000000043
:101A70000000000000000000000000002100240021
:101A800027002A002D00300033000101000004016E
:101A900007010A0101021020200808102040102030
:101AA0004080020102010804020101020408102022
:101AB0004080804020100804020180040201804020
:101AC0002010080402010804020101020408102089
:101AD0004080010204081020408005050505070527
:101AE00008080808020202020A0A0808040404049A
:101AF00001010101010101010303030303030303C6
:101B0000040707070C0C0C0C0C0C0C0C0202020254
:101B100006060606060606060B0B0B0B0B0B0B0B3D
:101B20002F64617461002F736B6574636800416397
:101B3000636573732D436F6E74726F6C2D52657194
:101B4000756573742D507269766174652D4E657478
:101B5000776F726B3A2074727565004163636573C9
:101B6000732D436F6E74726F6C2D416C6C6F772D9B
:101B7000486561646572733A202A00416363657346
:101B8000732D436F6E74726F6C2D416C6C6F772D7B
:101B90004D6574686F64733A20504F53542C474519
:101BA000542C4F5054494F4E530041636365737337
:101BB0002D436F6E74726F6C2D416C6C6F772D437B
:101BC000726564656E7469616C733A2074727565D0
:101BD000004F5054494F4E530044454C4554450026
:101BE0005055540047455400504F5354006175748C
:101BF000686F72697A6174696F6E3A20004175741A
:101C0000686F72697A6174696F6E3A2000436F6E13
:101C100074656E742D4C656E6774683A20006F634E
:101C20007465742F73747265616D00696D616765A9
:101C30002F6A70656700696D6167652F6769660067
:101C4000746578742F68746D6C006170706C696372
:101C50006174696F6E2F6A736F6E00746578742F8C
:101C6000706C61696E00436F6E74656E742D54798B
:101C700070653A2000436F6E6E656374696F6E3AEB
:101C800020636C6F7365004163636573732D436FED
:101C90006E74726F6C2D416C6C6F772D4F7269672B
:101CA000696E3A20687474703A2F2F6C617A796883
:101CB0006F6D652E727500556E6B6E6F776E004E90
:101CC0006F74204D6F646966696564004F4B004D09
:101CD0006F766564207065726D616E656E746C7987
:101CE00000496E7465726E616C2053657276657220
:101CF000204572726F72005061796C6F616420547C
:101D00006F6F204C61726765004E6F7420666F754F
:101D10006E64005757572D41757468656E7469631A
:101D20006174653A204261736963207265616C6D0C
:101D30003D224163636573732072657374726963D6
:101D40007465642200556E617574686F72697A6596
:101D500064005061796C6F61642073697A652077E3
:101D6000726F6E670042616420726571756573748D
:101D700000485454502F312E312000200000000024
:101D80000000000000004F4E000000000000004F67
:101D90004646000000000000524553540000000079
:101DA00000544F47474C4500000048414C54000048
:101DB000000000584F4E000000000000584F4646FB
:101DC0000000000000494E43524541534500444540
:101DD000435245415345004845415400000000002E
:101DE000434F4F4C00000000004155544F0000008D
:101DF000000046414E5F4F4E4C590044525900007E
:101E00000000000053544F500000000000484947B4
:101E10004800000000004D454449554D0000004C6D
:101E20004F57000000000000454E41424C45000065
:101E30000044495341424C4500005452554500006E
:101E400000000046414C534500000000524742004C
:101E500000000000004853560000000000005772C8
:101E60006F6E67207061796C616400202D3E2041A7
:101E7000543A004368616E20747970653A004E6F81
:101E80002073746F7265642076616C756573202DA4
:101E90002064656661756C743A20002D3E005075B3
:101EA000623A2000636D640046414E5F4F4E4C59CC
:101EB0000044525900434F4F4C00484541540041A3
:101EC00055544F002D3E005075623A2000736574E2
:101ED0000064656C002D3E005075623A20002D3E76
:101EE000005075623A2000556E6B6E6F776E2063FE
:101EF0006D64200A004F4646004F4E0053617665E0
:101F00006420455441473A00536574204554414785
:101F10003A2000009AB40EA411241FBECFEFD1E2E4
:101F2000DEBFCDBF00E00CBF15E0A0E0B2E0EAE10B
:101F3000F5E901E00BBF02C007900D92AA39B10785
:101F4000D9F72AE0AAE9B5E001C01D92A837B20787
:101F5000E1F71FE0CBE8DFE000E006C021970109D0
:101F6000802FFE010E9443C5CA38D10780E00807D0
:101F7000A9F70E9420A40C947BCA0C940000FC01D9
:101F8000818D928D0895FC0184899589089525EAB3
:101F900033E0FC0131832083FB0140895189628950
:101FA0007389FC0142835383648375830895DC0144
:101FB000ED91FC91048CF58DE02D1994CF93DF9376
:101FC0001F92CDB7DEB76983DC01ED91FC910280F1
:101FD000F381E02D41E050E0BE016F5F7F4F199526
:101FE0000F90DF91CF910895FC019485FB018485CA
:101FF000981303C081E0943009F480E0089521E053
:10200000FC018485843009F420E0822F089508952E
:10201000CF93DF931F92CDB7DEB76983DC01ED91DB
:10202000FC910280F381E02D41E050E0BE016F5F42
:102030007F4F19950F90DF91CF910895DC01ED91BD
:10204000FC91068CF78DE02D199591E08927089574
:10205000862F089581E086270895DC0180E0615095
:1020600038F0ED91E827F0E0EA54FB4E8491F7CF89
:102070000895FC01818191E09093DE078093000830
:102080001092DF0710920108089520914306260F51
:102090003327331F21323105ECF42091D807FC019E
:1020A00090E080E0243069F082E00895A09143063A
:1020B0002191AC014F5D594FA40FB52FB11D2C9349
:1020C0000196861798F380914306680F6093430644
:1020D00080E0089581E0089508950895E0916906EB
:1020E00080916806E81730F4F0E0E659F94F8081F6
:1020F00090E008958FEF9FEF089590916906809189
:1021000068062FEF3FEF981748F4E92FF0E0E65903
:10211000F94F208130E09F5F90936906C9010895CF
:102120008091680690916906891B990B0895CF925A
:10213000DF92EF92FF920F931F93CF93DF937C0177
:10214000CB018A012091DE07222389F0EB016B018C
:10215000C40ED51ECC15DD0569F06991D701ED914E
:10216000FC910190F081E02DC7011995F3CF642F08
:102170000E944510C801DF91CF911F910F91FF90F0
:10218000EF90DF90CF900895CF93DF931F92CDB75C
:10219000DEB769832091DE072223F9F02091010840
:1021A000203258F021E030E0FC013383228390E0BC
:1021B00080E00F90DF91CF9108958091DF07E82FA5
:1021C000F0E0E052F84F998190838F5F8093DF07B2
:1021D0008093010881E090E0ECCF61E0CE010196B0
:1021E0000E944510F7CF90E0FC01E652F54EE491D5
:1021F000F0E0EE0FFF1FE65EF54EA591B4912C9135
:102200008C56954EFC018491822391E009F490E074
:10221000892F0895FC01DC018D918111FDCF30E003
:1022200020E050E040E08AE09191992301F14430B0
:1022300051055CF59E3271F42F3F310509F02CF504
:10224000DB01A40FB51F12962C934F5F5F4F30E058
:1022500020E0EACF829FD001839FB00D1124292F67
:10226000990F330B205331092A0F3B1FDDCF2F3F2E
:10227000310509F054F4443051053CF4640F751FE6
:10228000FB01228381E090E0089590E080E00895D2
:10229000CF93DF931F921F92CDB7DEB780916C0A68
:1022A00090916D0A009711F488E79AE0BE016F5F84
:1022B0007F4F681B790B072E000C880B990B0F9032
:1022C0000F90DF91CF9108959FE9980F963010F409
:1022D000875508959FEB980F963010F48753089513
:1022E00080538A3008F080E00895DC0115968D91C6
:1022F0009C91009739F0DC01ED91FC910680F7810B
:10230000E02D19940895089583E090E00895809158
:10231000B9059091BA050895FC01848195810895CD
:10232000DC011196EC911197E295EF70E150EB30E2
:1023300008F039C0F0E08827EF55FE4E8F4F0C941F
:1023400043C5C411C411D311AC11AC11B511CC11DA
:10235000CC11CC11AC11AC1114966D917D918D9175
:102360009C9117970E9475C3089514966D917D9165
:102370008D919C91179724E630E040E050E00E9458
:10238000DAC4CA01B901EECF14966C9170E090E006
:1023900080E00E9473C3089514966D917D918D9194
:1023A0009C911797089560E070E0CB010895FC01BF
:1023B000A7812A2F2E7FD1F0818182958F70815045
:1023C0008330A0F4A695A150BB0B2BE531E00E9411
:1023D0005AC524E630E040E050E00E94DAC4DA0159
:1023E000C90187569F4FAF4FBF4F08958FEF9FEFA3
:1023F0000895DC01ED91FC91309729F090859F7054
:1024000081E0953009F080E00895FC01A481B58158
:10241000109721F118969C9118979F708EEF890F55
:10242000823010F091111AC019964D935D936D93FF
:102430007C931C97A481B58118969C911897907FE6
:10244000926018969C930480F581E02D8085982FEA
:10245000907F903619F48F70806A80870895DC0130
:1024600019968D919C91009739F0DC01ED91FC91CA
:102470000280F381E02D19940895DC0155962C918A
:102480005597273731F4ED91FC91008CF18DE02DBB
:1024900019940895CF93DF93EC01E881F9810484C6
:1024A000F585E02D199529893A892F5F3F4F3A8BA1
:1024B000298BDF91CF910895CF93DF93EC018E8527
:1024C00081110DC081E090E049895A892C853D85B4
:1024D0004217530708F080E0DF91CF910895E8811B
:1024E000F9810484F585E02DCE0119958F3F910582
:1024F00049F780E090E0F0CFFC018485958568176E
:10250000790708F4CB01928B818B0895DC011E962C
:102510002C911E97222339F0ED91FC910190F081CE
:10252000E02D6FEF19940895FC0187859089089537
:1025300081E0089590E080E00895CF93DF93CDB7D8
:10254000DEB760970FB6F894DEBF0FBECDBF19821D
:102550001A821B821C821D821E821F8218868A811B
:102560008F7080618A836FEF3E819F81888529818A
:102570007A815B814C814C873E87888B372F452F32
:102580005C857E85892F988960960FB6F894DEBFAA
:102590000FBECDBFDF91CF910895CF92DF92EF9222
:1025A000FF920F931F93CF93DF93CDB7DEB7AF9713
:1025B0000FB6F894DEBF0FBECDBF7C016A0105EAFD
:1025C00013E01A8309831C861B8688EE93E0A0E043
:1025D000B0E08D879E87AF87B88B8DE793E09A87B1
:1025E0008987188F0F8B198E1A8E1B8E1C8E84E094
:1025F00089A31BA70AA71CA61DA61EA61FA680911D
:10260000310890913208A0913308B09134088EA31C
:102610009FA3A8A7B9A78B839C83AD83BE8318868D
:102620001F82AE01465D5F4FCE0101960E948E7DF6
:1026300081309105B1F4D701ED91FC910488F589C1
:10264000E02D1DA30CA38CA59DA5AEA5BFA58EA3B3
:102650009FA3A8A7B9A7A601BE016C5D7F4FC701C4
:102660001995AF960FB6F894DEBF0FBECDBFDF91C0
:10267000CF911F910F91FF90EF90DF90CF90089531
:10268000CF92DF92EF92FF920F931F93CF93DF933E
:10269000CDB7DEB7AF970FB6F894DEBF0FBECDBF94
:1026A0007C016A0105EA13E01A8309831C861B86F4
:1026B00088EE93E0A0E0B0E08D879E87AF87B88B6F
:1026C0008DE793E09A878987188F0F8B198E1A8E62
:1026D0001B8E1C8E84E089A31BA70AA71CA61DA61F
:1026E0001EA61FA68091310890913208A091330850
:1026F000B09134088EA39FA3A8A7B9A78B839C830E
:10270000AD83BE8318861F82AE01465D5F4FCE014A
:1027100001960E948E7D81309105B1F4D701ED9133
:10272000FC910684F785E02D1DA30CA38CA59DA527
:10273000AEA5BFA58EA39FA3A8A7B9A7A601BE015A
:102740006C5D7F4FC7011995AF960FB6F894DEBF49
:102750000FBECDBFDF91CF911F910F91FF90EF90F2
:10276000DF90CF900895CF93DF93EC01888D843074
:1027700061F00E945483E88DF0E0EE0FFF1FED56EC
:10278000F94F1182108284E0888FDF91CF910895F4
:10279000EF92FF921F93CF93DF93FC01208D2430A3
:1027A00039F080E0DF91CF911F91FF90EF90089575
:1027B0007B01EC0110E0812F0E94178481110FC072
:1027C000188F888D843069F3FD86EC861A8E198EF9
:1027D00020E0A70162E00E94688381E0E3CF8831B6
:1027E00079F31F5F143039F7ECCF0F931F93182F35
:1027F0000E94FB9604C096958795779567951A95E4
:10280000D2F78B019C0101501109210931090E3FBA
:102810001F4F2F4F3F4F20F061E070E080E090E0CD
:102820001F910F9108950F931F93CF93DF931F92E2
:10283000CDB7DEB78C01DC01ED91FC910084F18510
:10284000E02D1995892B79F0BE016F5F7F4FF8015C
:1028500084850E94197C898190E00F90DF91CF914F
:102860001F910F9108958FEF9FEFF7CFFC018485A3
:102870000C947C7CCF93DF931F92CDB7DEB741E001
:1028800050E0BE016F5F7F4FFC0184850E947C7C1D
:102890001816190634F4898190E00F90DF91CF91DA
:1028A00008958FEF9FEFF9CFFC018485843011F0FC
:1028B0000C945A7C90E080E00895CF93C62F0E943C
:1028C000391061EE87E398E00E94C4106C2F87E313
:1028D00098E00E94C410CF910C94B3941092D80742
:1028E00081E08093D7071092B20761E084E10E94F3
:1028F000179361E085E10E941793E9EBF0E0808196
:102900008E7F808380818D7F808388E48093B80070
:1029100085E48093BC00089569E87FE0811102C0DE
:102920006BE87FE084EC98E00C94FD7669EE7CE047
:1029300084EC98E00E94FD76F0E0E0E0199584EFE9
:1029400091E008956DE078E0811102C068E078E0E0
:1029500085E799E00C94FD764F925F926F927F929B
:10296000AF92BF92DF92EF92FF920F931F93CF939C
:10297000DF9300D000D0CDB7DEB77C01D62E80919A
:102980001D06882309F4BEC0D70114969C9180913E
:102990000402891708F4B6C080911B0690911C06AA
:1029A000BAE06B13F0C085539A4FFC011082D70137
:1029B00018960D911C910115110509F49FC0F8019D
:1029C000618572856115710591F445805680678037
:1029D00070848091250890912608A0912708B091D5
:1029E0002808481659066A067B0609F487C0D801EC
:1029F0001B964D915C911C974115510509F47EC0C1
:102A0000F701248153968C91539790E0322F3770C1
:102A100002C0959587953A95E2F780FF6FC0A22E88
:102A2000B12CC501887F9370892B39F451968D9113
:102A30009C91887F9370A82AB92AD8018D919C9186
:102A4000DC01ED91FC916115710509F486C00688E1
:102A5000F789E02D1995019709F050C06CE3F80152
:102A6000808191810E940A76A50170E060E02AE0F1
:102A7000D8018D919C910E94BA75F80122818081C4
:102A8000918165E774E1222311F063E774E10E940C
:102A9000FD76D8011D966D917C911E978D919C912C
:102AA0000E94977660E2F801808191810E940A7607
:102AB000D8011F966D917C9150978D919C910E94A9
:102AC0009776F80122818081918168E674E1222362
:102AD00011F062E674E10E94FD766BEC75E0D801BE
:102AE0008D919C910E949776F80180819181DC0103
:102AF000ED91FC91008CF18DE02D199510921C0642
:102B000010921B06D70115968D919C9116970097F0
:102B100009F44DC014963C9120910502231708F446
:102B200046C0DC01ED91FC910190F081E02D6D2D0E
:102B3000199526960FB6F894DEBF0FBECDBFDF9174
:102B4000CF911F910F91FF90EF90DF90BF90AF90CA
:102B50007F906F905F904F9008950488F589E02DE5
:102B600025EA33E03A832983D80115964D905D908C
:102B70006D907C9018974B825C826D827E82BE0144
:102B80006F5F7F4F67CF8F3491050CF0BBCFBDE0F7
:102B90006B1709F4B7CF9C012F5F3F4F30931C0692
:102BA00020931B0685539A4FFC016083ABCF81E0D5
:102BB00090E0BFCF0C94D6B7CF93C1E068EE73E03E
:102BC00080E090E00E94B6946C2F84EC98E00E9424
:102BD000308CCF5FC43191F784EF91E0CF910895AD
:102BE000CF93DF93009709F484C0FC012081222356
:102BF00009F47FC0EC016DEC7EE10E9476BA892B6E
:102C000009F456C064EA7EE1CE010E9476BA892BAF
:102C100009F451C064E476E0CE010E9476BA892BB3
:102C200009F44CC060E476E0CE010E9476BA892BAC
:102C300009F447C06CE376E0CE010E9476BA892B96
:102C400009F442C068E376E0CE010E9476BA892B8F
:102C5000F1F164E376E0CE010E9476BA892BD1F1DE
:102C600060E376E0CE010E9476BA892BB1F16BE287
:102C700076E0CE010E9476BA892B91F167E276E088
:102C8000CE010E9476BA892B71F161ED7EE1CE0111
:102C90000E9476BA892B51F163E276E0CE010E9460
:102CA00076BA892B31F58CE090E0DF91CF910895D1
:102CB00082E090E0FACF81E090E0F7CF88E090E00A
:102CC000F4CF85E090E0F1CF86E090E0EECF87E0B2
:102CD00090E0EBCF89E090E0E8CF8AE090E0E5CFAC
:102CE0008BE090E0E2CF83E090E0DFCF84E090E003
:102CF000DCCF90E080E0D9CFCF93DF93EC0160EBA5
:102D000073E185E799E00E94FD766C817D8185E71E
:102D100099E00E94378C6AEA73E185E799E00E94A6
:102D2000FD7685E799E00E94067660E08C810E943E
:102D300045931092BA051092B90581E090E0DF91B9
:102D4000CF910895EF92FF921F93CF93DF93192FA6
:102D50007B01C82FD92FD7FF03C0D195C195D109C9
:102D600061E08C2F0E94459382E0E816F10499F40B
:102D700060E08C2F0E94179368E872E185E799E084
:102D80000E94FD7685E799E0DF91CF911F91FF903A
:102D9000EF900C940676612FEF2851F46095661F32
:102DA0006627661F8C2F0E94179364E872E1E6CFB6
:102DB000661F6627661F8C2F0E9417936FE772E1CC
:102DC000DDCFCF93DF9300D000D01F921F92CDB7FD
:102DD000DEB7EEEAF8E0128A118A80E090E195878A
:102DE000848784E890E0948B838B81E0868780E001
:102DF00090E2908B878787E7858B1C821B828DE70B
:102E000092E09A838983FE83ED838FEF9FEF98870B
:102E10008F836BE073E184EC98E00E94FD76609113
:102E2000B4057091B505CE0101960E9494788EEAA2
:102E300098E00E943D126BEF72E184EC98E00E94F2
:102E4000FD7684EC98E00E9406760E948C9C289681
:102E50000FB6F894DEBF0FBECDBFDF91CF910895BE
:102E6000FC0186819781009799F0FC0120852F70E5
:102E7000223029F4618572858385948508952530F3
:102E800039F460E00E941588009711F0FC01F2CF40
:102E900060E070E0CB010895CF93DF93EB0163E036
:102EA000FC01808191810E941588009761F0FC01EE
:102EB00020852F70223039F4818592858C239D23C3
:102EC000DF91CF91089590E080E0FACFCF93C62FA5
:102ED00063E0FC01808191810E941588FC01892BAF
:102EE00019F19085892F8D70F9F4907F9260908709
:102EF00081859285A385B4858827AA27BB278C2B3B
:102F000081879287A387B48769E476E085E799E0B3
:102F10000E94FD766C2F85E799E00E94308C85E752
:102F200099E0CF910C940676CF91089563E0FC016F
:102F3000808191810E941588009719F0FC0181859C
:102F400008958FEF0895FF920F931F93CF93DF9310
:102F5000CDB7DEB764970FB6F894DEBF0FBECDBF16
:102F60008C01F62E8FE290E09A838983FE013396DE
:102F700088E0DF011D928A95E9F7F8016681FF205C
:102F800011F081E06827D80114968C910E94179364
:102F9000F80187819085A185B285883E9340A1057F
:102FA000B10508F48BC066EF73E185E799E00E94F4
:102FB000FD76D80114966D917C9185E799E00E9489
:102FC000378C61EF73E185E799E00E94FD766F2D04
:102FD00070E085E799E00E94378C85E799E00E94D0
:102FE000067668E174E1CE0101960E946BBAF801A1
:102FF000828193810E949617FF2009F46BC06EEDC9
:1030000073E18D3051F062EE73E18E3031F069EE94
:1030100073E18B3011F066ED73E1CE010B960E94E7
:103020007FBA61EC73E185E799E00E94FD76D801F3
:103030001296ED91FC9113970190F081E02D608143
:103040007181ED91FC910288F389E02D9E012F5F43
:103050003F4FAE01455F5F4FC8011995BC0185E741
:1030600099E00E94378C6FEB73E185E799E00E944D
:10307000FD76D8011296ED91FC910190F081E02D42
:103080006081718185E799E00E949776BE016F5F4C
:103090007F4F85E799E00E9497766CEB73E185E7B7
:1030A00099E00E94FD76BE01655F7F4F85E799E05C
:1030B0000E94977685E799E00E94067664960FB69F
:1030C000F894DEBF0FBECDBFDF91CF911F910F915E
:1030D000FF90089562ED73E1823009F49ECF6DECAC
:1030E00073E19BCFCF92DF92EF92FF920F931F93EA
:1030F000CF93DF93CDB7DEB760970FB6F894DEBFFE
:103100000FBECDBF7C016B01CA01B9012AE0AE013F
:103110004F5F5F4F0E941ABBD701ED91FC9102886F
:10312000F389E02D9801AE014F5F5F4FB601C701F3
:10313000199560960FB6F894DEBF0FBECDBFDF9134
:10314000CF911F910F91FF90EF90DF90CF90089556
:10315000892B71F0FB01828193810E94BA8962E020
:103160007FE084EC98E00E94FD7688EC90E0089582
:1031700090E080E0F2CF892B71F0FB018281938196
:103180000E946C896BEE7EE084EC98E00E94FD76F4
:1031900088EC90E0089590E080E0F2CF8091A00864
:1031A0009091A108892B51F00E94A19D882331F0B4
:1031B0006BED7EE084EC98E00E94FD761092C008F2
:1031C0001092BF0880E090E19093BB088093BA080A
:1031D00084E890E09093C2088093C10881E08093D6
:1031E000BC0880E090E29093BE088093BD0882E71F
:1031F0008093C3088EEA98E00E9486128EEA98E0D7
:103200000E943D1288EC90E00895EF92FF920F9398
:103210001F93CF93DF93CDB7DEB72C970FB6F894FB
:10322000DEBF0FBECDBF8C017B0185EA93E09A83A0
:1032300089831B821C821D821E8298878F83198638
:103240001A861B861C8605301105ECF0BE01695FED
:103250007F4FF701808591850E940A11892B99F093
:10326000CE0107960E945D8ABE01695F7F4FF7011C
:10327000868197810E940A11892B61F0CE01079601
:103280000E94078B0EC0CE0101960E945D8A043019
:10329000110554F7CE0101960E94078B03301105EA
:1032A0008CF1BE01695F7F4FF701848195810E9497
:1032B0000A11892B39F1CE0107960E94B28ABE010C
:1032C000695F7F4FF701828193810E940A11892BE8
:1032D00001F1CE0107960E94088A64EC7EE084EC3E
:1032E00098E00E94FD7688EC90E02C960FB6F8945A
:1032F000DEBF0FBECDBFDF91CF911F910F91FF9029
:10330000EF900895CE0101960E94B28A0230110515
:10331000B4F6CE0101960E94088A01301105E9F643
:10332000CE0101960E94088A6BEC7EE084EC98E066
:103330000E94FD76D2CF0F931F93CF93DF938C0122
:10334000EB010297C4F08A819B810E940ABA8093A4
:10335000050299270E94FB8B0230110549F08C81F0
:103360009D810E940ABA8093040299270E94058CCD
:10337000C8ECD0E002C0C0E9D1E060EB7EE084ECB4
:1033800098E00E94FD766091050284EC98E00E942E
:10339000308C6BE97EE084EC98E00E94FD766091D1
:1033A000040284EC98E00E94308C84EC98E00E9447
:1033B0000676CE01DF91CF911F910F910895CF93A3
:1033C000DF93EB010297A4F166E87FE08A819B819D
:1033D0000E9458BA892B29F40E945C8B6F770E9457
:1033E000A18B62E87FE08A819B810E9458BA892B79
:1033F00029F40E945C8B60680E94A18B6AE87EE0E1
:1034000084EC98E00E94FD760E945C8B6095661FBC
:103410006627661F70E084EC98E00E94378C84EC8D
:1034200098E00E94067688EC90E0DF91CF910895B5
:103430000E94E116F8CFDF92EF92FF920F931F9355
:10344000CF93DF938C01FC01808191810E943F8C9E
:10345000C82FD0E0C430D10584F40E94987A009738
:1034600021F0FC012085207F2087BC01F8018081AC
:1034700091810E94118C2196EDCFF801C081D181FC
:1034800060E0CE010E941588FC01D184F801D0864D
:1034900061E0CE010E9415887C01F801938382834C
:1034A00062E0CE010E941588F8019583848364E070
:1034B000CE010E941588F80197838683F0E1DF1220
:1034C00052C08BE090E00E943AB7EC011B830A8364
:1034D00084E392E0998388831E82C8010E944C8C09
:1034E00097FD49C09D838C838C819D81009719F045
:1034F0008634910524F080E290E09D838C83E11472
:10350000F10409F447C0F70180858F70853009F018
:1035100041C0C7010E943F8C8230E0F161E0C701E9
:103520000E941588FC01892BA9F180858F7082305B
:1035300051F561857285838594850E9475C320E06D
:1035400030E04AE754E40E94D4C30E9447C66115A4
:1035500071058105910511F16F83788789879A87B5
:10356000F801D287C187DF91CF911F910F91FF9012
:10357000EF90DF9008959195819591099D838C83BB
:1035800081E08E83B1CF833029F461857285838594
:103590009485D5CF60E070E0CB01D1CF88E893E18E
:1035A000A0E0B0E08F839887A987BA87D9CFCF935F
:1035B000DF93EC01798368831A8619861B861C8E3B
:1035C0001B8E0E94F911882329F0CE01DF91CF9143
:1035D0000C941B1ADF91CF910895CF92DF92EF9256
:1035E000FF920F931F93CF93DF93EC016A017B014E
:1035F0008E819F81892BD9F4888199810E943F8C8B
:10360000082F10E00530110594F40E94987A009775
:1036100021F0FC012085207F20879F838E83BC01C1
:10362000888199810E94118C0F5F1F4FEBCFEE8133
:10363000FF81309749F18085982F9F7019F5807F21
:1036400082608087EE81FF81C186D286E386F48620
:1036500061E576E085E799E00E94FD762AE030E0BA
:10366000B701A60185E799E00E94117685E799E008
:10367000DF91CF911F910F91FF90EF90DF90CF904E
:103680000C9406769230F1F2DF91CF911F910F9159
:10369000FF90EF90DF90CF900895EF92FF920F93FD
:1036A0001F93CF93DF93EC018B011D821C821A8242
:1036B0001B82E880F980E114F10409F472C0809162
:1036C000B4059091B505892B09F46BC0672B09F4FB
:1036D0008701F80180858F708630A9F467EA73E06E
:1036E000C8010E94A087009719F0FC0181858A8398
:1036F0006BE875E0C8010E94A087009709F458C0E4
:10370000FC0181858B8369EA73E0C7010E94A08771
:10371000009709F043C06BED75E085E799E00E94E2
:10372000FD766B8185E799E00E94308C69ED75E04C
:1037300085E799E00E94FD766A8185E799E00E941D
:10374000308C85E799E00E940676E880F9800E9437
:10375000987A8C010097D1F0FC018085807F82608F
:103760008087118612861386148680819181009746
:1037700011F00E94D6B789EA93E00E9439C9F80196
:1037800091838083B801C7010E94118C69EA73E0BC
:10379000888199810E94A087009719F009969D83DE
:1037A0008C83DF91CF911F910F91FF90EF9008953F
:1037B000F801808191810E940ABAA4CF1F93CF9310
:1037C000DF93FC01162FC389D489818992899C01DA
:1037D0002F5F3F4F328B218BC80FD91FCE010E9424
:1037E00092C4181721F0612FCE010E949AC481E083
:1037F00090E0DF91CF911F910895FC01818992891A
:10380000248535858217930740F423893489820FF4
:10381000931F0E9492C490E008958FEF9FEF089548
:103820002F923F924F925F926F927F928F929F92D0
:10383000AF92BF92CF92DF92EF92FF920F931F93BE
:10384000CF93DF93CDB7DEB762970FB6F894DEBFA4
:103850000FBECDBF5C014B0129013A01CA01B9017C
:103860000E9440C61B013F926F9387EE93E09F93A7
:103870008F93CE0101967C019F938F930E9429CA5A
:103880000F900F900F900F900F900F9020E030E06E
:10389000A901C301B2010E9476C6181624F077FA76
:1038A000709477F87094F70101900020E9F7319750
:1038B0006F01CE18DF088EE28083A2E0B0E0AC0F8B
:1038C000BD1FAC0DBD1DBA8BA98BB10137FE03C066
:1038D000719561957109072E000C880B990B0E9458
:1038E00075C39B01AC01C301B2010E9461C520E018
:1038F00030E040E251E40E94D4C30E9440C6605DC3
:10390000E989FA896083FE01EC0DFD1D1382D50162
:10391000ED91FC910288F389E02D9801A701B40193
:10392000C501199562960FB6F894DEBF0FBECDBFE4
:10393000DF91CF911F910F91FF90EF90DF90CF908B
:10394000BF90AF909F908F907F906F905F904F90BF
:103950003F902F9008959B0190E00496982F882720
:10396000642F820F931F0C94FE7BCF93DF93C82F9D
:10397000D0E02496DC2FCC27C60FD71F0E94837B74
:103980008FE00E94987B8D2F0E94987B8C2F0E9445
:10399000987B80E00E94987BC82F0E94817B8C2FAF
:1039A000DF91CF910895CF93DF93C82FD62F472F64
:1039B00060E170E00E94AB1C4D2F61E170E08C2F44
:1039C000DF91CF910C94AB1C90E0982F882744E0B6
:1039D00050E0845F9B4F0C94CF7BFC018485843046
:1039E00011F00C94178480E00895CF93DF93FC01CD
:1039F00024852430D9F0EC010E94ED1C843189F03B
:103A0000882379F0883169F021E08C3159F4E8811C
:103A1000F9810084F185E02DCE01199521E0892BF3
:103A200009F420E0822FDF91CF91089580E0FBCF51
:103A300044E050E0BC018FE090E00C94CF7B44E088
:103A400050E0BC0185E090E00C94CF7B44E050E076
:103A5000BC0181E090E00C94CF7B08958F929F92FF
:103A6000AF92BF92CF92DF92EF92FF920F931F938C
:103A7000CF93DF93CDB7DEB72D970FB6F894DEBFA7
:103A80000FBECDBF7C0110E000E038EE832E33E0A6
:103A9000932EA12CB12C4DE2C42E43E0D42E1C82D7
:103AA0001B828D829E82AF82B886DA82C9820D87A0
:103AB000CE0101960E94ED1C811135C0F7014481B1
:103AC000558120E061E0802F0E94688380E590E0CE
:103AD0000E94229163E070E0802F0E94B51C833128
:103AE00029F462E070E0802F0E948191F7018481C7
:103AF0009581000F111FF801ED56F94F91838083D6
:103B00002D960FB6F894DEBF0FBECDBFDF91CF91DB
:103B10001F910F91FF90EF90DF90CF90BF90AF90EB
:103B20009F908F9008950F5F1F4F0430110509F08B
:103B3000B6CFE6CFCF92DF92EF92FF921F93CF9353
:103B4000DF93FC011485143089F1EC0180E590E0ED
:103B50000E94229168E070E0812F0E9481910E9472
:103B6000FB966B017C01CE010E94ED1C8823A1F025
:103B700062E370E080E090E00E94B6940E94FB96C1
:103B80006C197D098E099F09683E73408105910576
:103B900050F38C850E945483EC85F0E0EE0FFF1FFC
:103BA000ED56F94F1182108284E08C87DF91CF911E
:103BB0001F91FF90EF90DF90CF9008954F925F920A
:103BC0006F927F928F929F92AF92BF92CF92DF922D
:103BD000EF92FF921F93CF93DF93CDB7DEB72D9770
:103BE0000FB6F894DEBF0FBECDBF7C0193E9A92EBE
:103BF00096E0B92E10E0D12CC12C28EE422E23E005
:103C0000522E612C712C3DE2832E33E0932E1C82C8
:103C10001B824D825E826F8278869A8289821D879E
:103C2000D5012D913D915D01F70184819581281782
:103C30003907B1F4CE0101960E94ED1C843199F14F
:103C4000CE0101960E94ED1C8C3151F4CE010196FB
:103C50000E945414892B21F4CE0101960E949A1DD2
:103C60001F5F1430A1F6CD2841F4D701ED91FC91EE
:103C70000084F185E02DC70119952D960FB6F894B3
:103C8000DEBF0FBECDBFDF91CF911F91FF90EF90B0
:103C9000DF90CF90BF90AF909F908F907F906F906C
:103CA0005F904F900895CC24C394D12CD9CF8F929C
:103CB0009F92AF92BF92CF92DF92EF92FF920F93BB
:103CC0001F93CF936C015B017A01FC01C485C43062
:103CD000A1F481E090E0F60193838283F12CE12C42
:103CE000C701CF911F910F91FF90EF90DF90CF9080
:103CF000BF90AF909F908F9008958A0141305840B7
:103D000010F000E018E080E590E00E9422918C2FF6
:103D10000E9439924C0163E070E08C2F0E94B51C28
:103D2000873111F08C3129F58016910660F380E51A
:103D300090E00E9422919801A50170E060E08C2F34
:103D40000E94D99160E270E08C2F0E94819162E024
:103D500070E08C2F0E94B51C84FD13C063E070E0FE
:103D60008C2F0E94B51C811107C08C2F0E94548398
:103D7000B0CF10E000E0DBCF80E590E00E94229120
:103D8000E6CF40E162E070E08C2F0E94AB1C012B7B
:103D900009F0A6CF9ECF3F924F925F926F927F9293
:103DA0008F929F92AF92BF92CF92DF92EF92FF924B
:103DB0000F931F93CF93DF93CDB7DEB72D970FB639
:103DC000F894DEBF0FBECDBF6C015B014A010E94BB
:103DD000DE1D83E9E82E86E0F82E312C10E000E0AD
:103DE00098EE492E93E0592E612C712C1C821B8277
:103DF0004D825E826F8278868DE293E09A8389831A
:103E00003D86F701219131917F01F60184819581F1
:103E10002817390771F4CE0101960E94ED1C8731F5
:103E200041F4A401B501CE0101960E94571E080F6E
:103E3000191F3394F4E03F12D9CFC8012D960FB665
:103E4000F894DEBF0FBECDBFDF91CF911F910F91D0
:103E5000FF90EF90DF90CF90BF90AF909F908F90AA
:103E60007F906F905F904F903F900895CF93DF9336
:103E700091E0909320068823B9F0C091B800D091CA
:103E8000BA008091BC008A7B8093BC0060E084E132
:103E90000E94179360E085E10E9417930E946E14C0
:103EA000D093BA00C093B800DF91CF910895CF921C
:103EB000DF92EF92FF920F931F93CF93FC01C1818A
:103EC0000E949E936B017C018091D807811164C090
:103ED00081E08093D8078093D7079FEF9093D60710
:103EE0001092D5071092D4078093B3078091B3073F
:103EF000CC0FC82BC093B3078091B207813009F073
:103F000081C01092B2070E949E936B017C01809148
:103F1000B3078093BB008091DA079091DB07A091F3
:103F2000DC07B091DD07892B8A2B8B2BA1F00E9437
:103F30009E930091DA071091DB072091DC07309106
:103F4000DD076C197D098E099F09061717072807D9
:103F5000390708F442C08091BC0083FDD8CF85ECBE
:103F60008093BC000E949E936B017C018091D807D6
:103F7000813009F449C08091D507811167C08091D3
:103F8000D507E4EBF7E0AAE6B6E090E0981751F128
:103F900021912D939F5FFACF8091DA079091DB07F3
:103FA000A091DC07B091DD07892B8A2B8B2B09F4BC
:103FB0008BCF0E949E930091DA071091DB0720912E
:103FC000DC073091DD076C197D098E099F09061702
:103FD00017072807390708F077CF8091D9070E9483
:103FE000361F80E0109269068093680687E398E0A8
:103FF0000E947D10CF911F910F91FF90EF90DF9065
:10400000CF90089585EEACCF8091DA079091DB07D1
:10401000A091DC07B091DD07892B8A2B8B2B09F44B
:10402000A5CF0E949E930091DA071091DB072091A3
:10403000DC073091DD076C197D098E099F09061791
:1040400017072807390708F091CFC7CF81E099CF2C
:10405000AF92BF92CF92DF92EF92FF921F93CF93D6
:10406000DF93EC010E94FB966B017C0128EEC20EEF
:1040700023E0D21EE11CF11C10E08BE4A82EB12C31
:104080000E94FB966C157D058E059F0598F460EFE8
:10409000CE010E945D14CE010E94571F182F80FF91
:1040A0000BC0ED85FE85309709F01995C501019784
:1040B000F1F7E6CF81E08A83812FDF91CF911F91C5
:1040C000FF90EF90DF90CF90BF90AF9008951F9337
:1040D000CF93DF93EC01162F0E942820CE010E947F
:1040E000391062ED87E398E00E94C410612F70E000
:1040F0006095709584E0660F771F8A95E1F7612BD4
:1041000087E398E00E94C4100E94B394CE010E94FD
:10411000571F811711F084E08A83DF91CF911F919F
:104120000895CF93DF93EC0163EC0E945D14CE0100
:10413000DF91CF910C94571F0F931F93CF93DF9371
:10414000EC010E94282080FD36C0CE010E94912003
:1041500060E0CE010E946720CE010E942820CE019F
:104160000E94391064EB87E398E00E94C4100E941B
:10417000B394CE010E942820082F10E082FF16C0C1
:1041800082E08A838881882341F0CE010E949120B9
:10419000682F6160CE010E94672015950795802FDA
:1041A0008170DF91CF911F910F9108958A818230A4
:1041B00049F71A82E7CF80E0F4CFCF93DF93EC0189
:1041C0000E949120682F6460CE01DF91CF910C9402
:1041D00067200F931F93CF93DF93EC01162F042FCB
:1041E0000E942820002319F0CE010E94DD20CE017C
:1041F0000E94391065EA87E398E00E94C410612F9D
:1042000087E398E00E94C410DF91CF911F910F9136
:104210000C94B3946F927F928F929F92AF92BF92C1
:10422000CF92DF92EF92FF920F931F93CF93DF9382
:10423000FC01248521118CC0872E762EEC010E9472
:104240009C20882309F486C0CE010E94282040E0EB
:1042500060EFCE010E94E92010E000E066246A943D
:10426000AA24A394B12CE02EE694E694E694F12CD3
:10427000802F8770650101C0CC0C8A95EAF78B8589
:10428000082E000C990B0817190734F5FE01EE0DE6
:10429000FF1D93809C20CE010E942820CE010E9409
:1042A000391068E787E398E00E94C410992011F064
:1042B00080E8982E692D87E398E00E94C4100E9440
:1042C000B394CE010E942820982F907485FF0BC0D4
:1042D000992369F08EEF2AC099249394081719073F
:1042E000D1F2912CD8CF911102C087FF602EFE0130
:1042F000EE0DFF1D938187FF28C0C92AC3820F5F7F
:104300001F4F0034110509F0AECF6B86FFEF6F121F
:1043100002C081E08C872396E72DF82DCF01089607
:1043200029912193E817F907D9F781E0DF91CF911F
:104330001F910F91FF90EF90DF90CF90BF90AF90C3
:104340009F908F907F906F900895C094C922D6CF90
:1043500080E0ECCF8FEFEACFEF92FF920F931F93A5
:10436000CF93DF938C017B0140E065E50E94E9205B
:10437000E70188E0E80EF11C699140E0C8010E9465
:10438000E920CE15DF05C1F7DF91CF911F910F9185
:10439000FF90EF900895CF92DF92EF92FF920F93EC
:1043A0001F93CF93DF938C01EB017A01FC01858190
:1043B00096810E949C208823C1F1BE01F80185816D
:1043C00096810E94AC2140E06EEBF80185819681D8
:1043D0000E94E920E7016701F9E0CF0ED11CF80146
:1043E000E580F680C7010E942820C7010E9439108D
:1043F00066E987E398E00E94C4100E94B394C70165
:104400000E94282061EEC7010E945D14C7010E942E
:10441000571F8993CC16DD0611F7F8018581968127
:104420000E949C2091E0813009F090E0892FDF917B
:10443000CF911F910F91FF90EF90DF90CF90089553
:10444000CF93DF93EA010E94CB21982F882341F07C
:1044500068E0CE010E942D1091E02885281390E09D
:10446000892FDF91CF910895CF93DF9300D000D0B3
:1044700000D0CDB7DEB7AE014F5F5F4F0E94202264
:10448000882331F08D818F33A9F020F48F31A1F092
:1044900080E007C08F3521F08F37D1F78CE001C065
:1044A0008BE029960FB6F894DEBF0FBECDBFDF912B
:1044B000CF9108958AE0F5CF89E0F3CF85ED809321
:1044C000BC008091DA079091DB07A091DC07B091E6
:1044D000DD070796A11DB11D23E0B695A795979519
:1044E00087952A95D1F72091BC0024FD03C0109236
:1044F000D80708954091DA075091DB076091DC07F7
:104500007091DD07452B462B472B69F30097A105DA
:10451000B10541F025E32A95F1F700000197A109C3
:10452000B109E1CF8091D9070C94361F1F920F92E9
:104530000FB60F9211240BB60F922F933F934F9308
:104540005F936F937F938F939F93AF93BF93EF93FB
:10455000FF938091B900887F803609F44DC008F040
:1045600040C0883209F4A9C028F5803109F49DC003
:10457000C8F4882309F4FBC0883009F496C0FF9181
:10458000EF91BF91AF919F918F917F916F915F91CB
:104590004F913F912F910F900BBE0F900FBE0F9038
:1045A0001F901895883109F488C0803241F78093B4
:1045B000D60714C0803409F49DC040F48033B9F3A9
:1045C0008833E9F68093D60785ECB0C0803509F4CE
:1045D00085C0883509F496C0883489F60E945E2229
:1045E000CECF883909F48CC038F5883729F050F4DB
:1045F000883611F0803719F683E08093D80710923F
:10460000670657C0883809F47BC0803919F08038B4
:1046100009F0B5CF80916706803208F071C0E09153
:10462000670681E08E0F809367068091BB00F0E003
:10463000E95BF94F80833DC0803B39F0E0F4803A7C
:1046400009F479C0883A09F09ACF84E08093D807BA
:104650001092440610924306E0914106F091420602
:1046600019958091430681110FC081E08093430624
:104670001092210609C0803C09F4A6CF883C09F4B9
:10468000A3CF883B09F07BCFE091440681E08E0FF9
:1046900080934406F0E0EF5DF94F80818093BB008A
:1046A000909144068091430629C08091B30780937E
:1046B000BB0085EC8093BC0062CF9091D5078091C0
:1046C000D407981758F5E091D50781E08E0F8093B5
:1046D000D507F0E0EC54F84F8081E9CFE091D507A1
:1046E00081E08E0F8093D5078091BB00F0E0EC5401
:1046F000F84F80839091D5078091D4079817C8F21E
:1047000085E8D8CFE091D50781E08E0F8093D5075B
:104710008091BB00F0E0EC54F84F80838091D70784
:1047200081115CCF81E08093B20784EA8093BC0062
:104730001092D80724CF85EC8093BC001092D80744
:1047400080916706803230F4E0916706F0E0E95B23
:10475000F94F10826091670670E0E0914506F09194
:10476000460687E496E019951092670608CF1092E6
:10477000D60734CF4F925F926F927F92AF92BF92E3
:10478000CF92DF92EF92FF920F931F93CF93DF931D
:1047900000D01F92CDB7DEB72B013C0129833A83AD
:1047A0004B835C83A6019501C801B701640D751D9B
:1047B000861D971D211531054105510511F00E94F7
:1047C000B8C429813A814B815C81621773078407E1
:1047D0009507D0F4241535054605570530F521E039
:1047E000822F0F900F900F900F90DF91CF911F911C
:1047F0000F91FF90EF90DF90CF90BF90AF907F90A0
:104800006F905F904F900895461657066806790698
:1048100050F421E089819A81AB81BC818415950592
:10482000A605B705E8F220E0DBCF21E046165706E3
:1048300068067906A8F2F7CF8F929F92AF92BF9247
:10484000CF92DF92EF92FF920F931F93CF93DF935C
:104850007C014A015901C0911E06D0911F06062F06
:10486000660F110B209709F45CC088858F70863025
:1048700009F055C06CEA73E0CE010E94A0876C017C
:1048800082E08816910449F061EB73E0E3E08E1654
:10489000910429F0D0E0C0E006C065EB73E0CE01E2
:1048A0000E94A087EC01C114D104D9F1F6018085E2
:1048B0008F708430B1F561857285A801C7010E94AF
:1048C000D2C9A8016AEB73E0C7010E94B4C920975E
:1048D00079F188858F70843059F569857A85A801CA
:1048E000C7010E94B4C9A8016AEB73E0C7010E9426
:1048F000B4C9A114B10429F0A801B501C7010E94EF
:10490000B4C9C701DF91CF911F910F91FF90EF9034
:10491000DF90CF90BF90AF909F908F900895D0E0A0
:10492000C0E0A80168E874E1C7010E94ADBAC9CF30
:10493000F2E08F16910481F083E08816910429F04B
:1049400060918C0670918D06CACFA80162E874E16F
:10495000C7010E948FBAC7CFA8016FE774E1F8CFF3
:10496000CF92DF92EF92FF920F931F93CF93DF933B
:10497000CDB7DEB7C154D1090FB6F894DEBF0FBE74
:10498000CDBF6C01AB0130E020E060E4CE010196C8
:104990007C010E941C24F70101900020E9F7319767
:1049A0008F010E191F09A801B701C6010E94C4C9D1
:1049B000892B11F010E000E0C801CF5BDF4F0FB68C
:1049C000F894DEBF0FBECDBFDF91CF911F910F9145
:1049D000FF90EF90DF90CF900895CF92DF92EF920B
:1049E000FF920F931F93CF93DF93CDB7DEB7C054E1
:1049F000D1090FB6F894DEBF0FBECDBF80919B06E4
:104A000090919C06059709F449C06115710509F458
:104A100045C069017A018B0140E450E0CE01019666
:104A20000E94D2C96FE270E0CE0101960E9499C93E
:104A3000892B41F4980143E050E060E4CE010196F7
:104A40000E941C244FE350E0B601CE0101960E9463
:104A5000B4C90E94BB87882309F180919B0690917D
:104A60009C060697D9F480910208811117C0B701FE
:104A7000CE0101960E94C99781E090E0C05CDF4FB3
:104A80000FB6F894DEBF0FBECDBFDF91CF911F915F
:104A90000F91FF90EF90DF90CF90089590E080E02D
:104AA000EDCF4F925F926F927F928F929F92AF92D3
:104AB000BF92DF92EF92FF920F931F93CF93DF93FA
:104AC000CDB7DEB760970FB6F894DEBF0FBECDBF8F
:104AD000FC0119861A861B861C869A859F70906633
:104AE0009A87A081B181109709F4F7C08C9188232F
:104AF00009F4F3C000811181D8019C91992309F434
:104B000043C09D3209F4EDC090539A3028F00F5FF6
:104B10001F4F11830083EECFC801D12CDC017D0132
:104B2000E81AF90A2D91022E000C330B205331099B
:104B30002A303105A0F35F016EE270E0C8010E94E7
:104B400099C9FC01009709F448C0DC014D018E1A97
:104B50009F0A11968C911197082E000C990BC09703
:104B600011960A9798F38181282F082E000C330B99
:104B7000205331092A30310518F480330CF06EC00F
:104B800020E030E0A90108C0D12CF12CE12CD3CFDA
:104B900029E030E040E050E0AAE0B0E00E94F9C433
:104BA0002B013C012281822F022E000C990BC09711
:104BB0008A30910570F420330CF458C02A330CF07D
:104BC00059C0092E000CAA0BBB0B480E591E6A1EB9
:104BD0007B1E8114910409F052C0C8010E9428BABA
:104BE0002A852F70206A2A872B013C016CE270E035
:104BF000D5018D919C910E9499C9009709F068C0D8
:104C0000F501118210824D865E866F86788A88E073
:104C1000FE013996DE01119601900D928A95E1F719
:104C200029813A814B815C816D817E818F8198855C
:104C300060960FB6F894DEBF0FBECDBFDF91CF9167
:104C40001F910F91FF90EF90DF90BF90AF909F90DA
:104C50008F907F906F905F904F9008958A330CF003
:104C600097CF032E000C440B550B96CF80E090E0BD
:104C7000DC01ABCF89E090E0A0E0B0E0A6CFC801B6
:104C8000B3E08B169104DCF4E8E0EE16F104BCF41A
:104C90000E9428BA9B01AC01A4E6B0E00E94F9C4CE
:104CA000DD2041F07094609450944094411C511C5C
:104CB000611C711C460E571E681E791E97CF0E94FC
:104CC00006BA2B013C018A858F7080678A878ECF58
:104CD0000196D5018D939C9396CF412C512C320196
:104CE00092CFC8010196DD24D39418CFEF92FF92A2
:104CF0000F931F93CF93DF93EC01A881B981109795
:104D000061F18C91882349F108811981F801808132
:104D1000882351F08D3241F080538A3028F00F5FA4
:104D20001F4F19830883F0CFC8010E940ABA7C0183
:104D30006CE270E0C8010E9499C9009751F4198291
:104D40001882C701DF91CF911F910F91FF90EF90D3
:104D50000895019699838883F4CFF12CE12CF1CF4B
:104D60004F925F926F927F928F929F92AF92BF927B
:104D7000CF92DF92EF92FF920F931F93CF93DF9327
:104D8000CDB7DEB761970FB6F894DEBF0FBECDBFCB
:104D90000E94FB969B01AC016091C7057091C8050C
:104DA0008091C9059091CA05A12CB12C650118E824
:104DB000E12E13E1F12E00E010E00E94BA238823D7
:104DC00019F1E0908A06F0908B06D70112968C912B
:104DD000823089F563E574E185E799E00E94FD760C
:104DE00085E799E00E94067680918A0690918B066D
:104DF0000E949C200E94FB966093C7057093C80593
:104E00008093C9059093CA0561960FB6F894DEBFEA
:104E10000FBECDBFDF91CF911F910F91FF90EF900B
:104E2000DF90CF90BF90AF909F908F907F906F90CA
:104E30005F904F9008958091C5059091C605892B8C
:104E400009F0DDC083E190E00E943AB78C0186E56D
:104E50009CE6F801928B818BF682E58214821082A7
:104E600089E0818381E0828383831093C605009368
:104E7000C5050E94FB966B017C01F0E1CF0EF7E2C5
:104E8000DF1EE11CF11CD8011596ED91FC911697DF
:104E90008FEF8387148613821482158216821782FD
:104EA00010861186128614961C9299249394BE0142
:104EB000665F7F4FF801858196810E940A2118164E
:104EC0000CF071C00E94FB966C157D058E059F0548
:104ED00008F069C067E0CE010A960E942D109989FA
:104EE0008913E5CFD8018C91811138C015968D9129
:104EF0009C910E949C20BE01665F7F4FF8018581D6
:104F000096810E94AC2140E064EBD80115968D910A
:104F10009C910E94E920F801A580B680C5010E94FD
:104F20002820C5010E94391067E887E398E00E94B5
:104F3000C41060E887E398E00E94C4100E94B39414
:104F4000C5010E942820B82ED80115968D919C91FC
:104F50000E949C20B5FC02C0F8019082AE014F5F18
:104F60005F4FBE01665F7F4FC8010E94CB21D80111
:104F70001196BC908A85803109F48CC2BE01665FAF
:104F80007F4FC8010E9434228B1558F5F8018181AA
:104F9000D80111968C93119714968C9114978F5F6A
:104FA00014968C9384CF10E000E08091C505909119
:104FB000C6052091C3053091C40502171307ECF410
:104FC0009801B3E0220F331FBA95E1F76091C10554
:104FD0007091C205620F731F0E94E9940F5F1F4F0B
:104FE000E4CF8A85803111F48CE0D2CFBE01665FB8
:104FF0007F4FC8010E943422CBCFFC0112828091E6
:10500000BF059091C0052091C3053091C40582175A
:1050100093070CF4D5C00E94FB962B013C01E09154
:105020008A06F0918B06309759F08FEF83871486AC
:1050300013821482158216821782108611861286B8
:105040004091C3055091C405E091BB05F091BC05AA
:1050500090E080E0841795070CF48EC08824839438
:10506000912C80918A0690918B06009709F48DC04F
:105070002091C3053091C405F3E0220F331FFA9548
:10508000E1F76091C1057091C205620F731F0E9424
:105090000A2118160CF079C08091C3059091C405BF
:1050A00041970CF072C00E94FB969B01AC01A12CB1
:1050B000B12C650118E8E12E13E1F12E00E010E0BB
:1050C000C301B2010E94BA2381115FC0C090C10523
:1050D000D090C205A090C305B090C405850173E0CF
:1050E000000F111F7A95E1F70C0D1D1D67E0C80137
:1050F0000E942D10D80117969C91F12CE12C891358
:10510000B0CFEA14FB040CF057C148E050E0B801FE
:10511000C6010E9453C9B8E0CB0ED11C892B09F0FF
:105120004BC0EE0CFF1CE091BB05F091BC05EE0DF1
:10513000FF1D808191818160918380836DE374E1A3
:1051400085E799E00E94FD768091C3059091C405A2
:1051500063E0880F991F6A95E1F72091C1053091AE
:10516000C205820F931F0E949C8F66E374E185E75E
:1051700099E00E94217775CF21913191DF0112973B
:105180002E7F2D933C93019665CF64E474E185E70F
:1051900099E00E94FD766091C3057091C40585E792
:1051A00099E00E94378C85E799E00E94067610927C
:1051B000C0051092BF051ECEEFEFEE1AFE0AA1CF7A
:1051C0000091C1051091C2059C0143E0220F331FDD
:1051D0004A95E1F7020F131FD8012C91283209F0EC
:1051E000DBC0AE014F5F5F4FB8018091C505909164
:1051F000C6050E942022811105C020E030E04EEF5C
:1052000052EC3EC06A8170E0762F6627770F770FE9
:10521000770F2981B8E02B9F90011124262B372B83
:10522000F80180818031D1F4688570E08F81AB0115
:10523000481B5109CA019695982F882797958795FD
:105240000E942FC5CB014097B90113E0660F771F6D
:105250001A95E1F760789C01260F371F213854EE2C
:1052600035075CF2B901330F880B990B0E9475C3A7
:1052700020E030E040E05CE30E94D4C39B01AC013D
:10528000E091BD05F091BE058091BF059091C005EC
:10529000BC01A3E0660F771FAA95E1F7A091C105B5
:1052A000B091C2056A0F7B1F309709F019950091E4
:1052B000C5051091C605E090BF05F090C00573E0EC
:1052C000EE0CFF1C7A95E1F78091C1059091C20523
:1052D000E80EF91ED7018C91803109F463C0B70143
:1052E000C8010E943422D82E882309F451C0F80145
:1052F000858196810E949C20882309F449C0B701CA
:10530000D80115968D919C910E94AC21F8014081A5
:1053100064E4858196810E94E920D80112968C91DF
:105320008823B1F1E7EFED0D4EEE842E42E0942E8E
:10533000E33038F4F0E0EE0FFF1FE157FD4F8080BF
:105340009180E114F10489F1F8018381882369F1E6
:10535000808181112AC00E94FB962B013C01092CFF
:10536000000CAA08BB08AE014F5F5F4FB701C80130
:105370000E94CB21898181110BC00E94FB96681984
:1053800079098A099B09641575058605970558F3FF
:105390008091BF059091C00501969093C0058093C0
:1053A000BF0528CD6CE0D62EA2CFB401990C880B96
:1053B000990B0E94B694ECCF8091C5059091C605DB
:1053C000892B09F44ECE88E0815008F44ACEF801CA
:1053D000E80FF11D90819923B9F3AA0CBB1C8091B1
:1053E000BB059091BC05A80EB91ED5018D929C926B
:1053F00061E374E185E799E00E94FD766091C30561
:105400007091C40585E799E00E94378C6AE274E1E7
:1054100085E799E00E94FD768091C3059091C405CF
:1054200023E0880F991F2A95E1F72091C10530915B
:10543000C205820F931F0E949C8F85E799E00E940E
:1054400006768091C3059091C40533E0880F991FBB
:105450003A95E1F76091C1057091C205680F791F17
:10546000FB018081883261F48091C5059091C60569
:105470000E94E99480918A0690918B060E94DD201B
:105480008091C3059091C40501969093C4058093C3
:10549000C305E7CDFCE0FB1508F478CDA5CD6DE59F
:1054A00072E184EC98E00E94FD766AE472E184EC9B
:1054B00098E00E94FD766CE372E184EC98E00E9433
:1054C000FD7664E372E184EC98E00E94FD7684EC62
:1054D00098E00E94067664E272E184EC98E00E9413
:1054E000FD7668E172E184EC98E00E94FD7660EF61
:1054F00071E184EC98E00E94FD7663EE71E184EC4A
:1055000098E00E94FD766EEC71E184EC98E00E94D8
:10551000FD766FEB71E184EC98E00E94FD7667EB1D
:1055200071E184EC98E00E94FD766CEA71E184EC14
:1055300098E00E94FD7662EA71E184EC98E00E94B6
:10554000FD7663E971E184EC98E00E94FD766BE8FA
:1055500071E184EC98E00E94FD766FE771E184ECE4
:1055600098E00E94FD7665E671E184EC98E00E9487
:10557000FD7666E471E184EC98E00E94FD7661E3DB
:1055800071E184EC98E00E94FD7664E271E184ECC4
:1055900098E00E94FD7666E171E184EC98E00E945B
:1055A000FD766AE071E184EC98E00E94FD7662E0AD
:1055B00071E184EC98E00E94FD7667EF70E184EC85
:1055C00098E00E94FD766AEE70E184EC98E00E941B
:1055D000FD7662EE70E184EC98E00E94FD7667ED66
:1055E00070E184EC98E00E94FD7668EC70E184EC58
:1055F00098E00E94FD766FEB70E184EC98E00E94E9
:10560000FD7661EB70E184EC98E00E94FD7663EA40
:1056100070E184EC98E00E94FD7684EC98E00C94B4
:105620000676009789F0FC0120852F70253061F403
:105630000E941588009741F0FC0120852F702430CE
:1056400019F481859285089590E080E00895CF92C5
:10565000DF92EF92FF920F931F93CF93DF9300D0CF
:1056600000D0CDB7DEB780911D0681119AC0809120
:105670009B0690919C0602970CF493C08091B40510
:105680009091B505009709F48CC06EEB73E00E9411
:10569000A0878C01009709F484C00E943F8CE82EFB
:1056A000F12CE114F10409F47CC070E060E0C80161
:1056B0000E94112B6C01EA94EF2809F481C061E08B
:1056C000C8010E941588FC0101851285CE01019652
:1056D0000E942591CE0101960E9443916CE57AE0EB
:1056E00084EC98E00E94FD76B60184EC98E00E947C
:1056F000977665EC73E084EC98E00E949776B801A9
:1057000084EC98E00E94378C65EC73E084EC98E0C0
:105710000E94977661EA77E084EC98E00E949776A1
:1057200084EC98E00E94067662E072E083E999E0FA
:105730000E94C813D0928909C092880910938B09DE
:1057400000938A0981EA97E0892BE9F58CEB93E0D5
:1057500090938D0980938C0980918E0690918F068D
:10576000009741F070E060E00E94112B90938D064D
:1057700080938C0680918C0690918D06009731F174
:1057800090938F0980938E0910929109109290093D
:1057900081E080931D0663E47AE084EC98E00E9447
:1057A000FD7626960FB6F894DEBF0FBECDBFDF9113
:1057B000CF911F910F91FF90EF90DF90CF900895C0
:1057C00002E012E083CF81EA97E0C2CF82EA92E062
:1057D000892B19F48CEB93E0D3CF82EA92E0D0CFFF
:1057E0002F923F924F925F926F927F928F929F92F1
:1057F000AF92BF92CF92DF92EF92FF920F93CF932F
:10580000DF9300D01F92CDB7DEB77C017A83698326
:105810005C834B83DB011C92FC016081662309F4ED
:105820004EC030FF4CC0F9E06F9FB00111246358A7
:10583000724ECD010E94ADBAD70111968C91807F36
:1058400041F04B815C8167EC73E089819A810E9411
:10585000B4C9E981FA8101900020E9F731972981E3
:105860003A81E21BF30B19012E0E3F1E4B815C8126
:105870004E1B5F0B415051095C834B83D70111963E
:10588000EC9111978E2F807F09F4F7C0E295EF70AD
:10589000E150EC3008F0F1C0F0E08827ED5AF34D0C
:1058A0008F4F0C9443C5622C052D722DD12DEC2DFC
:1058B000B02C822D822D822D9E2C862C082E2980A4
:1058C0003A80DCCFF7018481282F30E050E040E0BF
:1058D000002359F030E0A4E6B0E00E940CC52FEFA1
:1058E00030E040E050E00E94DAC45F934F933F9372
:1058F0002F9389EC93E09F938F93FC81FF932B81EF
:105900002F933F922F920E94ECC9B2C017968C91B0
:1059100017978F9316968C9116978F9315968C9157
:1059200015978F9314968C918F938CEC93E09F93A3
:105930008F93BC81BF93EB81EF93E3CF17968C914C
:1059400017978F9316968C9116978F9315968C9127
:1059500015978F9314968C918F9380ED93E0E7CFFA
:105960001496CD90DD90ED90FC901797F7FE34C023
:1059700084E6882E912CA12CB12CC701B601A5017B
:1059800094010E94DAC49B01AC0188279927DC01AD
:10599000821B930BA40BB50BBF93AF939F938F9375
:1059A00066277727CB016C197D098E099F09A50110
:1059B00094010E94DAC45F934F933F932F9384ED39
:1059C00093E09F938F933C813F934B814F933F9202
:1059D0002F920E94ECC94CC0C701B60124E630E00A
:1059E00040E050E00E94DAC49F938F937F936F93BF
:1059F0005F934F933F932F9385ED93E09F938F9306
:105A00009C819F93AB81AF93E2CFC7010E94D711D6
:105A1000BC01D7011696CC9016971796DC90179775
:105A2000D0FADD24D0F814969C9114971596FC902A
:105A3000EB80BC80292F30E050E040E077FD35C09E
:105A4000011135C07F936F931F921F921F929F93F6
:105A50001F92FF92DF92CF928EED93E09F938F93F0
:105A6000FC81FF932B812F933F922F920E94ECC9D0
:105A70000FB6F894DEBF0FBECDBF89819A810F901B
:105A80000F900F900F90DF91CF910F91FF90EF90BB
:105A9000DF90CF90BF90AF909F908F907F906F904E
:105AA0005F904F903F902F900895002361F0292F31
:105AB00030E0A4E6B0E00E940CC52FEF30E040E0FB
:105AC00050E00E94DAC45F934F933F932F931F924D
:105AD000FF92DF92CF9281EE93E09F938F93BF92DC
:105AE000EF9275CF15968C9115971F928F931696FE
:105AF0009C91169717968C9181708F939F9384EE4B
:105B000093E015CF14968D909D90AD90BC90179713
:105B100020E030E0A901C501B4010E946EC3240158
:105B2000350187FF04C077FA709477F87094C30149
:105B3000B2010E9440C66B01072E000C880B990B26
:105B40000E9475C39B01AC01C301B2010E9461C5F3
:105B500020E030E04AE754E40E94D4C30E94CBC660
:105B60000E9440C6062F772E20E030E0A901C50133
:105B7000B4010E946EC387FF07C07F920F93DF922C
:105B8000CF928AEE93E0D3CE7F920F93DF92CF92A3
:105B90008BEE93E09F938F933C813F934B814F9388
:105BA000B0CE14968C9114971F928F9315968C916A
:105BB00015971F928F9316968C911F928F9381EE5B
:105BC00093E09F938F93BC81BF93EB81EF933F92C0
:105BD0002F920E94ECC94CCF17968C9117971F9269
:105BE0008F9314968C9114971F928F9315968C9186
:105BF00015971F928F9316968C911F928F938EED0F
:105C000093E09F938F93BC81BF93EB81EF93DFCEA3
:105C100014966D917C914B815C81C1010E94D2C927
:105C20002CCFEF92FF920F93CF93DF93CDB7DEB7D8
:105C3000A0970FB6F894DEBF0FBECDBF7C0100E089
:105C400020E033E040E250E0BE016F5F7F4F0E94F2
:105C5000F02BBE016F5F7F4F85E799E00E9497763A
:105C60006EE279E085E799E00E94FD76F7016181B7
:105C700062956F7085E799E00E94308C67E279E069
:105C800085E799E00E94FD76F70161816F7085E7F5
:105C900099E00E94308C85E799E00E940676A096F4
:105CA0000FB6F894DEBF0FBECDBFDF91CF910F913D
:105CB000FF90EF900895AF92BF92CF92EF92FF9234
:105CC0000F931F93CF93DF9300D000D01F921F92AA
:105CD000CDB7DEB75C0109831A832B833C834D83E8
:105CE0005E836F8378876FE174E185E799E00E94B6
:105CF000FD76CE0101960E94112EE114F10439F0D7
:105D000068E174E1C7010E9476BA009721F1F501BC
:105D10000281138101151105E1F08981811159C0BA
:105D20008A818F70813009F459C038F1823019F1BD
:105D3000082F10E06BEF73E185E799E00E94FD7694
:105D4000B80185E799E00E94378C85E799E00E94C9
:105D5000067690E080E028960FB6F894DEBF0FBE7E
:105D6000CDBFDF91CF911F910F91FF90EF90CF901A
:105D7000BF90AF900895CC20B9F0CE0101960E945B
:105D80002288892B09F440C0C8010E943017672B74
:105D9000682B692BD9F480E00E94F513AB01BC019C
:105DA000C8010E94ED1A12C0C8010E9496178D30DA
:105DB00058F48A3010F4813049F4CE0101960E94E3
:105DC0002288892B19F0E0CF8E30B9F381E090E082
:105DD000C2CF8230C9F0A0F48130B1F26BE074E13F
:105DE00085E799E00E94FD76698185E799E00E9448
:105DF000308C85E799E00E94067601E010E09ACFAA
:105E00008A50853008F2EACF40E050E0BA01C8017C
:105E10000E94ED1A60E0C5010E94A317D7CFCF9270
:105E2000DF92FF920F931F93CF93DF938C01EB01CF
:105E30006A01CB010E94F911F82E882309F459C098
:105E4000D0FE05C0D8016C91CE010E946617D1FE2C
:105E500047C0F801448155816681778181818295AF
:105E60008F70873030F08930E0F08A50823008F44B
:105E700049C0CE010E940512EC81FD81309781F16D
:105E800080858F709EEF980F923010F0811128C09E
:105E9000D80111969C91907F80858F70892B808787
:105EA0001FC0EC81FD813097D9F080858F709EEF07
:105EB000980F923010F0811113C041875287638789
:105EC0007487EC81FD818085807F83608087EC8191
:105ED000FD818085982F907F8F7080679036F9F2D2
:105EE00060E279E085E799E00E94FD76C8010E94B2
:105EF000112E8F2DDF91CF911F910F91FF90DF9089
:105F0000CF900895CE010E940512EACFCF92DF9282
:105F1000EF92FF920F931F93CF93DF93611571055B
:105F200009F460C06A017B018C01CB010E94F91168
:105F3000D82F882389F1D70114968D919C910097D1
:105F400009F43FC0FC01C0852C2F2F703EEF320FAB
:105F5000323010F021112AC0C595C595C595C5955B
:105F6000D0FE5EC0C7010E949617F8018083CC2343
:105F700051F1C295C07F81818F70C82BC183D70139
:105F80001496ED91FC9181859285A385B485F801E5
:105F900084839583A683B7838D2FDF91CF911F9143
:105FA0000F91FF90EF90DF90CF900895253049F446
:105FB00060E00E941588009721F0DC011896CC91D2
:105FC000CBCFC0E0CDCFD7011496ED91FC91808569
:105FD0008295807F8595859585958595823021F080
:105FE000833081F0D0E0D8CF4185528563857485B8
:105FF000F80181818F70806A818344835583668331
:106000007783CACF4185528563857485F801818184
:106010008F70806781834483558366837783BCCF89
:10602000CC2389F2C295C07FF801A5CF0F931F93AF
:10603000CF93DF9300D000D01F921F92CDB7DEB771
:1060400019821A821B821C821D821E821F82188660
:106050002A812F702A83FC0102811381C8010E94CA
:1060600096178230D1F08530C1F08823B1F040E03E
:1060700052E0B801CE0101960E94862FCE01019612
:106080000E94228828960FB6F894DEBF0FBECDBFBF
:10609000DF91CF911F910F91089590E080E0F2CFB2
:1060A000CF93DF9300D000D01F921F92CDB7DEB701
:1060B000FC01862F8F706181607F682B618388E08F
:1060C000DE01119601900D928A95E1F729813A81BE
:1060D0004B815C816D817E818F81988528960FB67A
:1060E000F894DEBF0FBECDBFDF91CF910895CF935F
:1060F000DF9300D000D01F921F92CDB7DEB7FC0116
:10610000608398E0DE01119601900D929A95E1F777
:1061100029813A814B815C816D817E818F81988557
:1061200028960FB6F894DEBF0FBECDBFDF91CF919A
:106130000895DC011196EC911197E295EF70E15012
:10614000EB3008F037C0F0E08827E655FF4C8F4F62
:106150000C9443C5BC30BC30DA30B530B530CB30F0
:10616000C230C230C230B530B53014966D917D91D9
:106170008D919C911797089514966C9170E090E022
:1061800080E0089514966D917D918D919C91179763
:106190000E9440C6089514966D917D918D919C91B9
:1061A000179724E630E040E050E00E94DAC4CA01CC
:1061B000B901089560E070E0CB010895CF93DF93BB
:1061C000EC016115710539F48F8181708F8381E055
:1061D000DF91CF9108958981982F92959F7029F131
:1061E00080E09430A8F79B01770F440B550B295999
:1061F000310941095109A4E6B0E00E94F9C42BE538
:1062000031E040E050E00E94DAC437FF02C030E0E5
:1062100020E02536310514F024E630E02F5F220F10
:106220008F818170282B2F83D2CF8F7080628983DA
:10623000DACF2F923F924F925F926F927F928F921E
:106240009F92AF92BF92CF92DF92EF92FF920F9305
:106250001F93CF93DF93CDB7DEB76A970FB6F8944D
:10626000DEBF0FBECDBF1C0109871A872B873C8775
:106270004D875E876F87788B22E1E216F10408F084
:1062800035C0F701E455FD4F30813D8BCE010996B5
:106290000E94D71197FD04C0BC01C1010E94DE30ED
:1062A0009A85892F8F70D1011196EC911197E07F1B
:1062B000E82B1196EC93119789858C93E295EF70FA
:1062C000EC3008F063C0F0E08827E659FE4C8F4FB1
:1062D0000C9443C5593393319331F83278318D336F
:1062E000C232013301330133C232C2321D8ACECFF2
:1062F00010E092959F709D3008F011C4E92FF0E0F6
:106300008827EA57FE4C8F4F0C9443C5C631C633DD
:10631000E633C6338F338F33C633C6338F358F356D
:10632000C633C6339C3292959F709D3008F014C1DD
:10633000E92FF0E08827E056FE4C8F4F0C9443C5C0
:10634000C6317A326D323032B031AD3151327C32B9
:10635000AC32AC323B323B329C328889F1018783CC
:106360008F85D10116968C9316978E8515968C93F2
:1063700015978D8514968C9314979295907F11960E
:106380008C9111978F70982B11969C93FD89FF2308
:1063900009F463C0D10111968C9182958F702F2FD3
:1063A00030E08217130609F458C061E878E085E709
:1063B00099E00E94FD76F101618162956F7085E739
:1063C00099E00E94308C6EE778E085E799E00E94C2
:1063D000FD766D8985E799E00E94308C6CE778E066
:1063E00085E799E00E94FD76D1010C9119821A820D
:1063F0001B821C821D821E821F8218868D898295B7
:10640000807F9A819F70892B8A830983EE24EA9486
:10641000FE2C11961C91119712962C91129713969F
:106420003C91139714964C91149715965C9115977F
:1064300016966C91169717967C91CE0101960E9444
:106440001931F1012083318342835383648375833F
:1064500086839783C1010E94112E88E0F1016FC1EC
:106460008F859889F1018683878190FB80F98783E6
:106470008E8585838BCF8D859E85AF85B889B7FD49
:106480000EC08F3F9105A105B10529F024F08FEFD3
:1064900090E0A0E0B0E0D10114968C9377CF80E03B
:1064A000FACF6D857E858F85988920E06D39BFEFA5
:1064B0007B078B079B076CF02FEF6115E4E67E07E7
:1064C0008105910534F424E630E040E050E00E947C
:1064D000DAC4D10114962C9359CF8F859889F10194
:1064E0008683878190FB80F987838E8585838D8560
:1064F00084834CCF8D85CFCFCD84DE84EF84F88824
:1065000020E030E0A901C701B6010E946EC360E03F
:1065100087FD0FC020E030E04FE753E4C701B6012C
:106520000E9476C66FEF181624F0C701B6010E94CC
:1065300047C6F10164832ACFD10111968C9111973E
:106540008F70806C11968C9311978D859E85159612
:106550009C938E9314971ACF6EE079E085E799E0CB
:106560000E94FD766A8562956F7085E799E00E94CA
:10657000308C6BE079E085E799E00E94FD76F101CF
:106580006181C0C092959F70933091F09C30A1F2D0
:106590004D855E856F857889F101448355836683D7
:1065A00077839295907F81818F70982B9183EECE27
:1065B000C1010E942288D10114968C9314978F8573
:1065C000988916968C93169717968C91179790FB2F
:1065D00080F917968C9317978E8515968C9315973F
:1065E00011968C9111978F70806211968C93CECEFC
:1065F000CE0109960E942288D10114968C9314979B
:10660000EFCF92959F709D3008F066C0E92FF0E0C3
:106610008827E25FFC4C8F4F0C9443C5C631293369
:106620005833D832583358331B3348334833483300
:10663000373343339C328D859E85AF85B889F10110
:1066400084839583A683B78381818F7080668183DD
:106650009DCE6D8570E090E080E00E9473C3D10113
:1066600014966D937D938D939C9317978FCE6D8524
:106670007E858F8598890E9475C3F1016483758337
:106680008683978383CE6D857E858F859889E5CFB8
:106690009295907FF10181818F70982B91838D85E8
:1066A0009E85AF85B88984839583A683B7836ECE94
:1066B0009295907FD10111968C9111978F70982BA4
:1066C00011969C938D859E85AF85B889F101848351
:1066D0009583A683B7835ACE69EF78E085E799E082
:1066E0000E94FD766A8562956F7085E799E00E9449
:1066F000308C66EF78E085E799E00E94FD76D10165
:1067000011966C9162956F7085E799E00E94308CCC
:1067100085E799E00E94067639CE11E0EACD4D85F5
:106720005E856F857889F10144835583668377831D
:106730009295907F81818F70982B918388E0DE0104
:10674000119601900D928A95E1F729813A814B814A
:106750005C816D817E818F8198856A960FB6F894F1
:10676000DEBF0FBECDBFDF91CF911F910F91FF9084
:10677000EF90DF90CF90BF90AF909F908F907F90E1
:106780006F905F904F903F902F900895963009F44E
:10679000C1C048F46D85913071F06FEF70E09330B7
:1067A00051F060E008C0973009F4C0C09A506D8580
:1067B0007E859230B0F784E68F8788898E7F888BBC
:1067C0001E868A858F7080628A876D872E8530E06D
:1067D000AFEFB0E00E940CC5C12CD12C7601CA9459
:1067E0006115F4E67F078105910544F424E630E065
:1067F00040E050E00E94DAC469017A01112309F4F3
:1068000075C0DA8AC98A2D852E8B022F10E08889FF
:106810008695A82FA150BB0BB88FAF8B119609F0AE
:10682000A4C09601203831050CF087C08FE790E0B6
:106830008C199D09809FD001819FB00D909FB00D54
:1068400011242FEF30E00E945AC521E83EE740E0D6
:1068500050E00E94DAC4D10117962C93ABE9B0E066
:10686000A70196010E94F9C43FE7432E512C612CE9
:10687000712CA30192010E94DAC42C593F4F4F4F53
:106880005F4F5901AEEFB1E0A70196010E94F9C434
:10689000A30192010E94DAC4D8010E94F9C42FEF2B
:1068A00030E040E050E00E94DAC489012F3F31051A
:1068B00019F014F00FEF10E069EE78E085E799E049
:1068C0000E94FD76B50185E799E00E94378C6BED5B
:1068D00078E085E799E00E94FD76B80185E799E0C8
:1068E0000E94378C85E799E00E94067669EA78E095
:1068F00085E799E00E94FD7685E799E00E9406769B
:1069000062EA78E085E799E00E94FD76C1010E9485
:10691000112E3CCD6D857E858F85988924E630E0EB
:1069200040E050E00E94DAC4B90145CF6D857E8514
:106930008F8598890E9440C63ECFA7012058310913
:1069400041095109ABE9B0E00E94F9C42FE730E0FA
:1069500040E050E00E94DAC42C593F4F4F4F5F4F48
:106960005901D10117961C92A7CF2F89388DAAEB18
:10697000BFEF0E9452C524E6822E912CA12CB12C8F
:10698000A50194010E94DAC429013A01B4E64B0E34
:10699000511C611C711C26E430E0AF89B88D0E9447
:1069A0005AC5A50194010E94DAC449015A01EEE1D9
:1069B0008E0E911CA11CB11C29893A892038310501
:1069C0000CF094C08FE790E0821B930B809FD00166
:1069D000819FB00D909FB00D1124A50194010E94DC
:1069E00004C59B01AC01AFEFB0E00E94F9C424E6FE
:1069F0003AE640E050E00E94DAC4D10117962C93A9
:106A0000A7019601240D351D461D571DAEEFB1E0BF
:106A10000E94F9C423EE30E040E050E00E94DAC466
:106A2000298B3A8B4B8B5C8BE989FA89FA8FE98F3A
:106A3000AFEFB0E0A70196010E94F9C42FE730E064
:106A400040E050E00E94DAC47901FE89AF2FB0E047
:106A500029893A894B895C890E94F9C42FEF30E07B
:106A600040E050E00E94DAC489012F3F310519F05F
:106A700014F00FEF10E065ED78E085E799E00E94F3
:106A8000FD762AE030E0B301A20185E799E00E949B
:106A900011766FEC78E085E799E00E94FD762AE0B8
:106AA00030E0B501A40185E799E00E94117667EC1A
:106AB00078E085E799E00E94FD76B70185E799E0E7
:106AC0000E94378C6FEB78E085E799E00E94FD76B5
:106AD000B80185E799E00E94378C66EB78E085E79E
:106AE00099E00E94FD76698D7A8DF8CEA701960116
:106AF0002058310941095109ABE9B0E00E94F9C4BD
:106B00002FE730E040E050E00E94DAC42C593F4FBC
:106B10004F4F5F4F7901D10117961C92ACCF60E9BE
:106B200078E085E799E00E94FD766A8562956F704E
:106B300085E799E00E94308C6DE878E01CCDFC017F
:106B40009181892F82958F7021F0823029F080E029
:106B500008959F70906291839B0177FF02C030E09F
:106B600020E02E3681E0380714F02DE631E0268350
:106B7000878130FB80F9878381E008950F931F930D
:106B8000CF93DF938C01FC01C081D1816FE270E073
:106B9000CE010E94E1C90097D9F0FC011192CF010A
:106BA0000E94F015EC016DE576E085E799E00E9422
:106BB000FD76BE0185E799E00E94378C85E799E074
:106BC0000E940676CE01DF91CF911F910F9108951B
:106BD000CE010E94F015EC01892BA1F3F80111827E
:106BE0001082F0CF8F929F92AF92BF92CF92DF929E
:106BF000EF92FF920F931F93CF93DF93CDB7DEB742
:106C000067970FB6F894DEBF0FBECDBF8C017B0136
:106C10004C018BE0880E911C9F8A8E8AF8011286A7
:106C200011861386148E138E672B09F463C0A0900F
:106C30009D06B0909E06A114B10409F45BC06FE2FA
:106C400070E0C7010E9499C96C01892B09F44AC000
:106C5000F701DE01119690E080E0BD012191222331
:106C600041F02F3231F08431910519F02D930196C6
:106C7000F5CF860F971FFC011082C5010E94A087E7
:106C8000F80191838083B6016F5F7F4F4FE050E042
:106C9000C4010E94D2C9CE0146960E94BE35F801B9
:106CA000948F838F8E899F89892B09F41386C8015D
:106CB0000E94F911882319F0C8010E941B1A6796D7
:106CC0000FB6F894DEBF0FBECDBFDF91CF911F91FD
:106CD0000F91FF90EF90DF90CF90BF90AF909F907B
:106CE0008F900895B701C5010E94A087F801918394
:106CF0008083DDCFF80111821082D9CF8F929F92CD
:106D0000AF92BF92CF92DF92EF92FF920F931F93B9
:106D1000CF93DF93CDB7DEB7CD55D1090FB6F89439
:106D2000DEBF0FBECDBF8C016B016115710519F07F
:106D300041155105D1F46AE37AE085E799E00E94B4
:106D4000FD7661E37AE085E799E00E94FD76B8017F
:106D500085E799E00E9497766FE27AE085E799E00F
:106D60000E94FD7685E799E030C0460F571FDA0193
:106D70001C920E9448114B016DE27AE085E799E090
:106D80000E94FD76B40185E799E00E94378C6AE2A3
:106D90007AE085E799E00E94FD76B80185E799E001
:106DA0000E94977667E27AE085E799E00E94FD7697
:106DB000BAE38B16B1E09B06F4F46AE17AE08EEC5C
:106DC00098E00E94FD768EEC98E00E940676C35A09
:106DD000DF4F0FB6F894DEBF0FBECDBFDF91CF916E
:106DE0001F910F91FF90EF90DF90CF90BF90AF90E9
:106DF0009F908F90089568E17AE085E799E00E947E
:106E0000FD76B60185E799E00E94977666E17AE023
:106E100085E799E00E94FD7685E799E00E94067675
:106E20001A821982FE0133968EE3DF011D928A9544
:106E3000E9F780919B0690919C060597D9F563E050
:106E400070E0C8010E94B0247C01892B09F045C084
:106E5000E0914908F0914A08808180FFB8CF62E054
:106E600070E0C8010E94B024892BD9F064E270E080
:106E7000C8010E94E1C9892B09F0A9CF6EEF79E022
:106E800085E799E00E94FD76B80185E799E00E94C8
:106E9000977685E799E00E940676C8010E9467927E
:106EA00096CF61E070E0C8010E94B024892B09F4FC
:106EB0008ECFDCCF61E070E0C8010E94B0247C017D
:106EC000892B21F562E070E0C8010E94B0247C01AA
:106ED00063EF79E0892B09F441CFE00EF11E6AEEF1
:106EE00079E0C7010E9476BA892BC1F4F6010190BE
:106EF0000020E9F73197EC19FD09329778F0C801C5
:106F00000E946792C6010E94CD7761CF4FE350E0A7
:106F1000B801CE0101960E94D2C9DFCF64E270E0D1
:106F2000C8010E94E1C9892B09F051CFB701CE01F8
:106F30008F5B9F4F0E94F235CE018F5B9F4F0E9467
:106F4000F911882339F1B601CE018F5B9F4F0E9462
:106F5000018D18161906F4F489818823D9F08091DF
:106F60009B0690919C060597A9F062ED79E085E774
:106F700099E00E94FD76BE016F5F7F4F85E799E043
:106F80000E94977685E799E00E940676CE010196E9
:106F90000E946792CE018F5B9F4F0E942F1217CFE6
:106FA000CF93DF93EB0163E0FC01808191810E942C
:106FB0001588FC01892BA9F080858D7091F4C0950E
:106FC000D095CF6FAE0170E060E081859285A3859A
:106FD000B4858C239523A623B72381879287A38723
:106FE000B487DF91CF910895CF93DF93EB0163E0F6
:106FF000FC01808191810E941588FC01892BB9F0E8
:107000009085892F8D7099F4907F92609087CC271E
:10701000CE01B0E0A0E04185528563857485842B64
:10702000952BA62BB72B81879287A387B487DF91F7
:10703000CF910895CF92DF92EF92FF920F931F931B
:10704000CF93DF9300D000D01F921F92CDB7DEB751
:107050006C017B0160FF03C0E894E0F8F3F8F3FCF7
:107060000DC00E944811663971058105910530F007
:1070700080919B0690919C060597E9F4B7016627DD
:107080007370C6010E94F4376BE678E085E799E0FB
:107090000E94FD768FEF9FEF28960FB6F894DEBF23
:1070A0000FBECDBFDF91CF911F910F91FF90EF9059
:1070B000DF90CF90089519821A821B821C821D8254
:1070C0001E821F8218868A818F708A8340E053E077
:1070D000B601CE0101960E94862F60E073E0C601E2
:1070E0000E944C17E82AF92A09811A812B813C81D8
:1070F0004D815E816F817885C6010E94E497CCCF77
:107100002F923F924F925F926F927F928F929F92B7
:10711000AF92BF92CF92DF92EF92FF920F931F93A5
:10712000CF93DF93CDB7DEB7C15CD1090FB6F8942A
:10713000DEBF0FBECDBF4C01C755DF4F0883C95A14
:10714000D040C655DF4F1883CA5AD040C555DF4FCF
:107150002883CB5AD040C455DF4F3883CC5AD04017
:10716000C355DF4F4883CD5AD040C255DF4F5883B7
:10717000CE5AD040C155DF4F6883CF5AD040C0555A
:10718000DF4F7883C05BD040CF54DF4FF982E88275
:10719000C15BD040CF53DF4FC882C15CD0400E945A
:1071A000FB96C354DF4F688379838A839B83CD5BCF
:1071B000D040C655DF4F8881CA5AD0408F70282EE4
:1071C000312CC0909B06D0909C06C554DF4FD982CD
:1071D000C882CB5BD040CF54DF4FE881F981C15BDF
:1071E000D040309721F0808181110C94E044D4018B
:1071F0001B968C91882341F0C4010B96CF54DF4F2E
:1072000099838883C15BD0402114310411F00C9420
:107210002945CF54DF4FE881F981C15BD0403097D9
:1072200011F00C94E444F401238C348C21143104C7
:1072300011F40C942945C655DF4F8881CA5AD040B5
:107240008F7011F00C942945622DCE0187559F4F08
:107250000E945030C756DF4F2883C959D040C656C8
:10726000DF4F3883CA59D040C556DF4F4883CB59CA
:10727000D040C456DF4F5883CC59D040C356DF4F5F
:107280006883CD59D040C256DF4F7883CE59D04065
:10729000C156DF4F8883CF59D040C056DF4F988307
:1072A000C05AD0400C942945D4018D919C910097EF
:1072B00009F403C2B4E02B16310409F0A8C00E94FF
:1072C0003F8C082F10E0063011058CF40E94987A4C
:1072D000009721F0FC012085207F2087BC01D4018C
:1072E0008D919C910E94118C0F5F1F4FECCF65E038
:1072F000F401808191810E9415888C01892BE9F429
:1073000010E000E0C801CF53DF4F0FB6F894DEBFA6
:107310000FBECDBFDF91CF911F910F91FF90EF90E6
:10732000DF90CF90BF90AF909F908F907F906F90A5
:107330005F904F903F902F900895C755DF4F888101
:10734000C95AD0408031E0F6CE0187559F4F0E9448
:10735000993016161706180619062CF4D801189637
:107360008C918D7089F0F80180858F70808768EC32
:1073700077E085E799E00E94FD7685E799E00E9435
:10738000067601E010E0BECF0E94FB966B017C0107
:10739000CE0187559F4F0E949930C60ED71EE81E1A
:1073A000F91ED8011996CD92DD92ED92FC921C97B0
:1073B000C755DF4F8881C95AD0408295807F82604F
:1073C00018968C936DEB77E085E799E00E94FD7647
:1073D000CE0187559F4F0E949930AB01BC012AE036
:1073E00030E085E799E00E94117667EB77E085E76A
:1073F00099E00E94FD76F801418552856385748588
:107400002AE030E085E799E00E941176B6CFC755B3
:10741000DF4F1881C95AD040143009F4C3C228F490
:10742000112391F1B12CA12C76C288EF810F82300B
:10743000C8F788E0FE01E755FF4FDE011196019085
:107440000D928A95E1F7C655DF4FE881CA5AD040C0
:107450008E2F807F09F422C3E295EF70E150EB306C
:1074600008F01CC3F0E08827E75CF54C8F4F0C94C4
:1074700043C53C3D3C3D4E3D2D3D2D3DA33D923D04
:10748000923D923D2D3D2D3D19821A821B821C8218
:107490001D821E821F8218868A818F708A83C6553C
:1074A000DF4F8881CA5AD040807F09F4BBCFF9E012
:1074B0002F16310409F431C20CF002C12114310439
:1074C00009F422C182E02816310409F0ABCFB12CB7
:1074D000A12CCD54DF4F1882C35BD040DD24DA9459
:1074E000B401CE0101960E946E8C8A81982F9295EC
:1074F0009F70945F9F70923060F4C655DF4F988103
:10750000CA5AD04092959F70923019F48F70806261
:107510008A83D40118969C91973071F4C655DF4F39
:107520008881CA5AD040807E803211F0803421F4A4
:107530008A818F7080628A83F401A185B285892F48
:1075400090E0109741F0ED91FC911197028CF38D32
:10755000E02DCD0119957C01C755DF4F0881C95A2F
:10756000D040C655DF4F1881CA5AD040C555DF4FAD
:107570002881CB5AD040C455DF4F3881CC5AD040F7
:10758000C355DF4F4881CD5AD040C255DF4F588197
:10759000CE5AD040C155DF4F6881CF5AD040C05538
:1075A000DF4F7881C05BD040CE0101960E94193137
:1075B000CF57DF4F2883C158D040CE57DF4F388395
:1075C000C258D040CD57DF4F4883C358D040CC5726
:1075D000DF4F5883C458D040CB57DF4F6883C5581E
:1075E000D040CA57DF4F7883C658D040C957DF4FC5
:1075F0008883C758D040C857DF4F9883C858D040B9
:10760000CE0101960E94112ECD54DF4FC880C35B7E
:10761000D040CC2051F1C655DF4F8881CA5AD040A6
:1076200082958F709FE0980F9F70923020F08A5F54
:107630008F708230D0F48A8182958F708150823031
:10764000A0F42D8130E0AFEFB0E00E940CC56115D1
:1076500024E67207810591050CF007C124E630E0AD
:1076600040E050E00E94DAC42D8388E0FE013196AC
:10767000DE01A755BF4F01900D928A95E1F78AE090
:10768000B82AC12CD40118968C911897873009F02C
:1076900090C5C954DF4FE881F981C75BD040EE3512
:1076A000F1400CF06AC461E977E08EEC98E00E944A
:1076B000FD768EEC98E00E9406760FEF1FEF22CE4B
:1076C0009AE02916310409F4D2C0ABE02A1631043D
:1076D00009F0A8CEB401CE0101960E946E8CCE01B5
:1076E00087559F4F0E94D711BC01CE0101960E9481
:1076F000DE3088E0FE013196DE01A755BF4F0190D4
:107700000D928A95E1F704C1C4010E94F44D8C01E9
:1077100061E070E01816190614F070E060E085E78B
:1077200099E00E94378C67EC73E085E799E00E944E
:107730009776CE0187559F4F0E949930AB01BC01CF
:107740002AE030E085E799E00E94117685E799E02C
:107750000E940676CE0187559F4F1016110614F031
:107760000C94CE440E949930672B682B692B09F04A
:1077700073C062E0CE0187559F4F0E947730CF568D
:10778000DF4F2883C159D040CE56DF4F3883C259CE
:10779000D040CD56DF4F4883C359D040CC56DF4F41
:1077A0005883C459D040CB56DF4F6883C559D04069
:1077B000CA56DF4F7883C659D040C956DF4F8883F9
:1077C000C759D040C856DF4F9883C859D040AA2423
:1077D000A394BA2CB1E0CD54DF4FB883C35BD04043
:1077E000DD24D3947DCE61E0CE0187559F4F0E946A
:1077F0007730C757DF4F2883C958D040C657DF4F6F
:107800003883CA58D040C557DF4F4883CB58D04043
:10781000C457DF4F5883CC58D040C357DF4F6883DD
:10782000CD58D040C257DF4F7883CE58D040C15793
:10783000DF4F8883CF58D040C057DF4F9883C0595F
:10784000D040AA24A394BA2CE1E0CD54DF4FE883C2
:10785000C35BD040D12C44CEB12CA12CF1E0CD544F
:10786000DF4FF883C35BD040BBCF2FEFFDCEB40119
:10787000CE0101960E946E8CC255DF4F8881CE5A90
:10788000D0409A8192959F7061F0923071F0B12C46
:10789000A12CCC24C394CD54DF4F1882C35BD040BD
:1078A0001CC29A819F7090629A8390E08536910500
:1078B00014F084E690E08E8388E0FE013196DE01CC
:1078C000A755BF4F01900D928A95E1F762E0CE0176
:1078D00087559F4F0E945030EA962FAFEA97EB965C
:1078E0003FAFEB97EC964FAFEC97ED965FAFED9710
:1078F000EE966FAFEE97EF967FAFEF97C158DF4FE1
:107900008883CF57D040C058DF4F9883C058D040AD
:10791000A12CBAE0BB2EC12CBECFB401CE01019682
:107920000E946E8CC155DF4F6881CF5AD040C05540
:10793000DF4F7881C05BD0407170CE0101960E940C
:107940009F35CD54DF4F8883C35BD040882309F433
:10795000A9C288E0FE013196DE01A755BF4F019014
:107960000D928A95E1F762E0CE0187559F4F0E9404
:107970005030E2962FAFE297E3963FAFE397E4965D
:107980004FAFE497E5965FAFE597E6966FAFE69762
:10799000E7967FAFE797E8968FAFE897E9969FAFB6
:1079A000E997B6CFC4010E94F44D181619065CF58C
:1079B00062E0CE0187559F4F0E947730AA962FAF85
:1079C000AA97AB963FAFAB97AC964FAFAC97AD963F
:1079D0005FAFAD97AE966FAFAE97AF967FAFAF97F5
:1079E000E0968FAFE097E1969FAFE197AA24A3942A
:1079F000BA2CC12C91E0CD54DF4F9883C35BD040AB
:107A0000DD24D3943FCE61E0CE0187559F4F0E9485
:107A10007730A2962FAFA297A3963FAFA397A496D5
:107A20004FAFA497A5965FAFA597A6966FAFA69701
:107A3000A7967FAFA797A8968FAFA897A9969FAF55
:107A4000A997AA24A394BA2CC12CA1E0CD54DF4F4E
:107A5000A883C35BD040D12C15CEC355DF4F2881FE
:107A600039814A815B81CD5AD040A4E6B0E00E94C2
:107A7000F9C42B013C010DC0C355DF4F4880CD5ADE
:107A8000D040B4E64B9E20011124052C000C660862
:107A90007708411451046104710429F4E5E04E2E85
:107AA000512C612C712C193041F4709460945094D5
:107AB0004094411C511C611C711CB401CE018755BE
:107AC0009F4F0E946E8C60E0CE0187559F4F0E94B1
:107AD00077306A962FAF6A976B963FAF6B976C962D
:107AE0004FAF6C976D965FAF6D976E966FAF6E9759
:107AF0006F967FAF6F97A0968FAFA097A1969FAF1D
:107B0000A197E2E02E16310409F477C02CF5211478
:107B1000310409F087CC91E0CD54DF4F9883C35BEB
:107B2000D04070C020E030E048EC52E4C355DF4F55
:107B3000688179818A819B81CD5AD0400E94D4C3CB
:107B40000E9440C696CFC355DF4F488059806A8057
:107B50007B80CD5AD0409DCF29E02216310409F414
:107B6000A6C18AE02816310409F05CCCC655DF4F67
:107B70008881CA5AD04082958F70823009F0F2C154
:107B8000C301B20124E630E040E050E00E94DAC4D4
:107B9000C255DF4F8881CE5AD04090E0280F391F60
:107BA00037FF02C030E020E02536310514F024E62E
:107BB00030E0C255DF4F2883CE5AD04062E0CE017C
:107BC00087559F4F0E9450302A962FAF2A972B96A9
:107BD0003FAF2B972C964FAF2C972D965FAF2D97DD
:107BE0002E966FAF2E972F967FAF2F9760968FAF01
:107BF000609761969FAF61978BCECD54DF4F18820F
:107C0000C35BD040D40119968D919C911A9700972F
:107C100089F518968C9190E060E5A62EB12CC12CC8
:107C2000D12C8530910549F0A12CB12C65014497E8
:107C300021F0A12CB12C6501AA94C655DF4FE88133
:107C4000CA5AD040E295EF70E150EB3008F020C105
:107C5000F0E08827E15DF14C8F4F0C9443C5423E24
:107C6000423E483F483F483F153FDF3EDF3EDF3E54
:107C7000703E703EDC01ED91FC91028CF38DE02DA5
:107C80001995CACFC355DF4F1881CD5AD040C301D3
:107C9000B20124E630E040E050E00E94DAC4DA01AC
:107CA000C901810F911DA11DB11DB7FF03C080E067
:107CB00090E0DC018F3F9105A105B10529F024F08A
:107CC0008FEF90E0A0E0B0E0C355DF4F8883CD5A3E
:107CD000D040A12C5AE0B52EC12CDD24DA94D2CCB0
:107CE000C355DF4FE880F9800A811B81CD5AD0400F
:107CF000B4E64B16510461047104DCF5A4E6B0E06F
:107D0000A80197010E94F9C4460E571E681E791EED
:107D1000A114B104C104D104B9F0A60195010E94D7
:107D2000F9C4362F272FB301A20177FF03C040E02B
:107D300050E0BA01432E522E3C014415550566050C
:107D4000770514F42A013B01C355DF4F488259825D
:107D50006A827B82CD5AD040C655DF4F8881CA5A8D
:107D6000D0408F708066C655DF4F8883CA5AD04096
:107D7000B0CFC301B20124E630E040E050E00E9401
:107D8000DAC4E20EF31E041F151FA114B104C104CE
:107D9000D10461F017FF03C0E12CF12C8701AE1470
:107DA000BF04C006D10614F486017501C355DF4F28
:107DB000E882F9820A831B83CD5AD0408ACFC3550B
:107DC000DF4F688179818A819B81CD5AD0400E94A2
:107DD00040C67B018C01C301B20124E630E040E0E3
:107DE00050E00E94DAC4CA01B9016E0D7F1D801FE8
:107DF000911FA114B104C104D10461F097FF03C025
:107E000060E070E0CB01A616B706C806D90614F4E8
:107E1000C601B5010E9475C3C355DF4F68837983DE
:107E20008A839B83CD5AD04054CFC355DF4F88817E
:107E30009981AA81BB81CD5AD040480E591E6A1E35
:107E40007B1EA114B104C104D104C9F0A4E6B0E0C2
:107E5000A60195010E94F9C4362F272FB301A20174
:107E600077FF03C040E050E0BA01432E522E3C01A0
:107E7000441555056605770514F42A013B01C355E1
:107E8000DF4F488259826A827B82CD5AD04021CF0F
:107E900088E0FE013196DE01A755BF4F01900D929B
:107EA0008A95E1F7B12CA12CCC24C39416CFC655EA
:107EB000DF4F8881CA5AD04082958F70823009F096
:107EC00051C0C301B20124E630E040E050E00E941E
:107ED000DAC4C155DF4F8881CF5AD040C055DF4F3B
:107EE0006881C05BD040962F9170280F391F2E36C5
:107EF000E1E03E072CF437FF05C02DE631E002C07B
:107F000030E020E0C155DF4F2883CF5AD040C05524
:107F1000DF4F8881C05BD04030FB80F9C055DF4F18
:107F20008883C05BD04062E0CE0187559F4F0E949E
:107F3000503062962FAF629763963FAF6397649617
:107F40004FAF649765965FAF659766966FAF66971C
:107F500067967FAF679768968FAF689769969FAF70
:107F60006997D6CC88E0FE013196DE01A755BF4F58
:107F700001900D928A95E1F78ACCCF53DF4FD880DC
:107F8000C15CD040DD20D9F01296ED91FC91908536
:107F90009F709530A1F4C554DF4F88819981CB5BE8
:107FA000D040059761F0CF54DF4F48815981C15BC4
:107FB000D040BE0167557F4FCF010E94344DC75559
:107FC000DF4F8881C95AD040853009F4CAC020F4F7
:107FD000833079F1C5016CC0863009F47CC08730EC
:107FE000C9F7C4010E949617182F863009F062C0A5
:107FF00061E777E085E799E00E94FD7666E070E052
:1080000085E799E00E94378C85E799E00E94067623
:1080100062E0CE0187559F4F0E94773029AF3AAF7B
:108020004BAF5CAF6DAF7EAF8FAF21969FAF219707
:108030003CC0C4010E949617853019F003E010E09F
:1080400061C962E877E085E799E00E94FD7665E026
:1080500070E085E799E00E94378C85E799E00E94FF
:108060000676B401CE0187559F4F0E946E8C61E069
:10807000CE0187559F4F0E94773022962FAF2297CF
:1080800023963FAF239724964FAF249725965FAF53
:10809000259726966FAF269727967FAF2797289626
:1080A0008FAF289729969FAF2997C501816091606E
:1080B000D12C30C069E577E085E799E00E94FD7634
:1080C000612F70E085E799E00E94378C85E799E0A1
:1080D0000E940676B3CFC4010E94F44D181619060B
:1080E000CCF1B401CE0187559F4F0E946E8C61E0A8
:1080F000CE0187559F4F0E94773029AB3AAB4BABEF
:108100005CAB6DAB7EAB8FAB98AFC501816091600E
:1081100046E0D42E5C016894A0F8C655DF4F288154
:10812000CA5AD040322F3F70323058F4C755DF4F13
:108130003881C95AD040332321F05C016894A0F8FB
:10814000B0F8207F59F16894B1F801E010E0C11057
:10815000E4C497C265E477E085E799E00E94FD7684
:108160006DCFC4010E94F44D18161906A4F462E004
:10817000CE0187559F4F0E94773029A73AA74BA77A
:108180005CA76DA77EA78FA798ABC50181609160A2
:1081900035E0D32EBFCF6EE277E0DECF40E052E095
:1081A000B401CE0187559F4F0E94862F8111CBCFFE
:1081B000CCCF9FEFD912BBC0C4010E94F44DDD2487
:1081C000D394181619060CF4B5C0D12C66E277E0EA
:1081D00085E799E00E94FD76ED2C0D2C000CFF0840
:1081E000C954DF4FF982E882C75BD040B70185E709
:1081F00099E00E94378C6FE177E085E799E00E9473
:10820000FD76CD54DF4FF880C35BD0406F2D70E01A
:1082100085E799E00E94378C85E799E00E94067611
:10822000CF54DF4FE880F980C15BD040E114F10406
:1082300009F48DC069EF7EE1C7010E9476BA01E0C2
:1082400010E0892B09F44BC065EF7EE1C7010E9465
:1082500076BA02E010E0892B09F441C06DE676E0C1
:10826000C7010E9476BA05E010E0892BC1F169E6EA
:1082700076E0C7010E9476BA06E010E0892B79F11A
:108280006AEB7EE1C7010E9476BA0AE010E0892B12
:1082900031F165EB7EE1C7010E9476BA0BE010E098
:1082A000892BE9F06FEB7EE1C7010E9476BA0CE002
:1082B00010E0892BA1F068EA7EE1C7010E9476BA3E
:1082C0000DE010E0892B59F061EB7EE1C7010E94BF
:1082D00076BA10E000E0892B11F40EE010E0C40142
:1082E0000E949617682E712C6114710431F4C954E0
:1082F000DF4F68807980C75BD0400115110509F414
:1083000045C060167106E9F069E077E085E799E01D
:108310000E94FD76B30185E799E00E94378C85E7DE
:1083200099E00E9406760DEF1FEF0C948239DD2054
:1083300009F44CCFA1E0CD54DF4FA883C35BD040FC
:1083400045CFCF54DF4F19821882C15BD040C7554B
:10835000DF4F9881C95AD0409F3008F076C1E92F8D
:10836000F0E08827E954FE4B8F4F0C9443C5394306
:10837000E742CB4205423943AA4283424F42394346
:10838000394302430243024302430243D401199694
:108390008D919C91009711F40C948039DC01ED9142
:1083A000FC910488F589E02DCD54DF4FC880C35B74
:1083B000D040C755DF4F0881C95AD040C655DF4F5E
:1083C0001881CA5AD040C555DF4F2881CB5AD040BA
:1083D000C455DF4F3881CC5AD040C355DF4F488158
:1083E000CD5AD040C255DF4F5881CE5AD040C155EA
:1083F000DF4F6881CF5AD040C055DF4F7881C05BD6
:10840000D04019958C010C948239C4010E949617B2
:10841000853009F013CE6AEF76E085E799E00E9497
:10842000FD7665E070E085E799E00E94378C85E78E
:1084300099E00E940676B401CE0187559F4F0E94B5
:108440006E8CF40180858530D9F46CE0CE018755BF
:108450009F4F0E94773029A33AA34BA35CA36DA33F
:108460007EA38FA398A76894A0F8B0F8D12C0FEF43
:108470001FEFF1E0CD54DF4FF883C35BD04067CEF0
:1084800061E0CE0187559F4F0E947730298F3A8F48
:108490004B8F5C8F6D8F7E8F8F8F98A3E4CFC4013D
:1084A0000E949617182F863059F569EE76E085E719
:1084B00099E00E94FD7666E070E085E799E00E9411
:1084C000378C85E799E00E94067662E0CE018755F9
:1084D0009F4F0E947730298B3A8B4B8B5C8B6D8B37
:1084E0007E8B8F8B988F6894A0F8B0F8D12C0FEF0B
:1084F0001FEF21E0CD54DF4F2883C35BD04027CE50
:1085000061ED76E0D9CDD11022C0B401CE018755FE
:108510009F4F0E946E8C61E0CE0187559F4F0E9455
:10852000773029873A874B875C876D877E878F876F
:10853000988B6894A0F8B0F826E0D22E0FEF1FEFCA
:1085400081E0CD54DF4F8883C35BD04000CE6DEB1C
:1085500076E002CEDD20E1F062E0CE0187559F4F4C
:108560000E94773029833A834B835C836D837E83BB
:108570008F8398876894A0F8B0F895E0D92E0FEF14
:108580001FEF91E0CD54DF4F9883C35BD040DFCD28
:1085900066EA76E0E1CDC655DF4F8881CA5AD04001
:1085A0008F70823008F05FC0C4010E94961785303A
:1085B00009F444CD6894A0F8B0F8D12C0FEF1FEF68
:1085C000A1E0CD54DF4FA883C35BD040C0CDC655DA
:1085D000DF4F8881CA5AD0408F70823008F0E5C0E2
:1085E000DD2081F063E976E085E799E00E94FD7681
:1085F00061E0C4010E94661760E079E0C4010E9456
:108600001A381CCDC655DF4F8881CA5AD040282F52
:108610002F70223008F0D0C0992309F4D4C0807F95
:1086200031F4B401CE0187559F4F0E946E8C68943F
:10863000A0F8B3E0BB2AD12C0FEF1FEFE1E0CD543F
:10864000DF4FE883C35BD04082CDC655DF4F8881C2
:10865000CA5AD040807F19F46894B0F807CF23E05D
:10866000B22AD12C6BCF91E0CD54DF4F9883C35BFE
:10867000D040C11052C2D12C0FEF1FEFA114B10492
:1086800039F0A501B401CE0187559F4F0E940F2FED
:10869000D40119968D919C91009709F49BC0CF54F9
:1086A000DF4FE880F980C15BD040DC01ED91FC91A7
:1086B0000488F589E02DCD54DF4FC880C35BD040DE
:1086C000C755DF4F0881C95AD040C655DF4F1881C2
:1086D000CA5AD040C555DF4F2881CB5AD040C45527
:1086E000DF4F3881CC5AD040C355DF4F4881CD5A37
:1086F000D040C255DF4F5881CE5AD040C155DF4FD0
:108700006881CF5AD040C055DF4F7881C05BD040E0
:1087100019958C01F40181859285DC01ED91FC9124
:10872000028CF38DE02D1995059711F46894A0F84B
:10873000DD2021F06D2DC4010E946617C554DF4F66
:10874000E881F981CB5BD040359721F0B501C401B8
:108750000E941A3869E776E085E799E00E94FD7685
:10876000B80185E799E00E94378C62E776E085E7FB
:1087700099E00E94FD760E94FB96AB01BC01C354B8
:10878000DF4FC880D980EA80FB80CD5BD0404C1998
:108790005D096E097F0985E799E00E942D8C85E7C8
:1087A00099E00E9406760C948239A1E0CD54DF4F07
:1087B000A883C35BD0405DCFB1E0CD54DF4FB88319
:1087C000C35BD04056CFE1E0CD54DF4FE883C35BBD
:1087D000D0404FCFF4018085853009F462C08630E7
:1087E00009F0A6CFC4010E944C8C7C01009709F4CB
:1087F0009FCF712C612C97FF06C0F194E194F10892
:1088000066246394712CC70101978634910508F0A2
:108810008FCFC755DF4F0881C95AD04010E0CE2C0A
:1088200061E08E2D0E944593672859F101301105B2
:1088300021F061E00C30110509F460E0062F10E032
:108840008C2D0E9417936EE876E085E799E00E94F0
:10885000FD76B70185E799E00E94378C6CE876E0F9
:1088600085E799E00E94FD76B80185E799E00E94CE
:10887000378C85E799E00E9406766894A0F8B0F8F6
:1088800086C00130110551F091E080E00C301105F7
:1088900009F090E0092F182F602FD2CF01E010E0EF
:1088A000FBCFF2E02F16310409F474C023E0221646
:1088B000310429F02A94232809F03ACFDECFC401ED
:1088C0000E943017892B49F4D401ED91FC9160810D
:1088D000718183EF93E00E94389ACE0187559F4FB4
:1088E0000E94901120E030E048EC52E40E94D4C392
:1088F0000E9440C6C954DF4F688379838A839B8373
:10890000C75BD040C954DF4F48805980C75BD04017
:1089100088E00E94F513CD54DF4F688379838A8302
:108920009B83C35BD040CD54DF4F68807980C35BAD
:10893000D04068E876E085E799E00E94FD76C9546A
:10894000DF4F68817981C75BD04085E799E00E945D
:10895000378C63E876E085E799E00E94FD76CD5498
:10896000DF4F488159816A817B81C35BD040662794
:1089700077272AE085E799E00E94BA7585E799E0B4
:108980000E940676B301A201C4010E94ED1A01E023
:1089900010E0CECE6894A0F8B1F8F9CF0E949930DB
:1089A000672B682B692B11F00C94F33BB12CA12C95
:1089B00021E0CD54DF4F2883C35BD0400C942A3C88
:1089C0002114310409F045C08081882311F40C94EE
:1089D0001339CE018F549F4F0E94BE351C01C655DE
:1089E000DF4F8881CA5AD0408F7071F5622DCE0159
:1089F00087559F4F0E945030CF55DF4F2883C15A73
:108A0000D040CE55DF4F3883C25AD040CD55DF4FCE
:108A10004883C35AD040CC55DF4F5883C45AD04006
:108A2000CB55DF4F6883C55AD040CA55DF4F788396
:108A3000C65AD040C955DF4F8883C75AD040C85561
:108A4000DF4F9883C85AD0402114310411F40C949C
:108A500013390E9448116B01C954DF4F7983688331
:108A6000C75BD04063E078E085E799E00E94FD763F
:108A7000B60185E799E00E94378C6CEF77E085E7D7
:108A800099E00E94FD76D401ED91FC9160817181A5
:108A900085E799E00E94977666EF77E085E799E0B1
:108AA0000E94FD76CF54DF4F68817981C15BD04051
:108AB00085E799E00E94977664EF77E085E799E093
:108AC0000E94FD76C954DF4FE881F981C75BD04031
:108AD00066EE77E0E83CF10514F40C94553BCE01CA
:108AE00087559F4F0E94112ECF54DF4FE881F981A7
:108AF000C15BD040309711F40C945439808184329A
:108B000011F00C94543962ED77E085E799E00E940A
:108B1000FD7685E799E00E9406760CEF1FEF0C9436
:108B200082392F923F924F925F926F927F928F92F3
:108B30009F92AF92BF92CF92DF92EF92FF920F93EC
:108B40001F93CF93DF93CDB7DEB7C955D1090FB6C9
:108B5000F894DEBF0FBECDBF3C01562E6296EFAE3D
:108B600062976396FFAE639764960FAF64976596BE
:108B70001FAF659766962FAF669767963FAF67976B
:108B800068964FAF689769965FAF69976A96CFAE60
:108B90006A972D2C4A2C3B2C009709F45CC1FC01F0
:108BA00080858295807F859585958595859584308E
:108BB00009F43CC12CF4882309F441C180E02DC0A4
:108BC000853009F444C08630C9F762E074E0C3011F
:108BD0000E94A0874C01009709F46FC0B12CA12C12
:108BE000D12CC12C6296EFAC62976396FFAC639771
:108BF00064960FAD649765961FAD659766962FAD29
:108C0000669767963FAD679768964FAD6897699688
:108C10005FAD6997652D0E949145C75ADF4F0FB62A
:108C2000F894DEBF0FBECDBFDF91CF911F910F91A2
:108C3000FF90EF90DF90CF90BF90AF909F908F907C
:108C40007F906F905F904F903F902F90089580910C
:108C500091068F5F8093910686809780811491049E
:108C600031F1A42CB32C6A96CFAC6A97D22C6296C1
:108C7000EFAC62976396FFAC639764960FAD649711
:108C800065961FAD659766962FAD669767963FAD63
:108C9000679768964FAD689769965FAD6997652D40
:108CA000C4010E949145F40182809380D7CF8091C6
:108CB000910681508093910681CF66E074E0C301F4
:108CC0000E94A0877C016BE074E0C3010E94A08732
:108CD0006C01552039F0F1E05F1609F488C010E00E
:108CE00000E00CC060E174E0C3010E94A0874C0169
:108CF00065E174E0C3010E94A0878C018114910496
:108D000009F443010115110509F48301E114F1048B
:108D100021F46A96EFAC6A97F22CC114D10411F4D5
:108D2000C42CD32C8114910409F492C0F4018085E1
:108D30008F70843009F08CC08184928401151105F4
:108D400009F491C0F80180858F70843009F08BC0E0
:108D500001851285E114F10409F4C9C0811491045C
:108D600009F490C06FEA74E185E799E00E94FD760E
:108D7000F7016185728585E799E00E9497766AEA36
:108D800074E185E799E00E94FD76B40185E799E0FA
:108D90000E94977685E799E00E940676CE018F5A69
:108DA0009F4F0E94112EC114D10409F0F8C0F701A1
:108DB00080858F70843009F0F0C061857285CE01A6
:108DC00001960E94F235CE0101960E94F911882386
:108DD00049F08114910409F469C0B401CE010196EF
:108DE0000E94018DCE0101960E942F12D6C06AE129
:108DF00074E0C3010E94A0874C016FE174E0C301DD
:108E00000E94A0878C018114910409F0CDC060E11B
:108E100074E0C3010E94A0874C010115110509F4FB
:108E200067CF892B09F072CF430170CF10E000E0CB
:108E3000912C812CD12CC12CF12CE12C5FCF10E096
:108E400000E0912C812CD12CC12CF12CE12C5ECF97
:108E5000912C812C73CFCA2CDB2C6A96EFAC6A97CD
:108E6000F22C912C812C00E020E033E040E150E036
:108E7000BE016F5B7F4FCE018F5A9F4F0E94F02B38
:108E80008C0168CF60EA74E185E799E00E94FD7685
:108E9000F7016185728585E799E00E9497766BE915
:108EA00074E185E799E00E94FD7678CFCC24C394E5
:108EB000F12CE12C62960FAD629763961FAD63971C
:108EC00064962FAD649765963FAD659766964FADF6
:108ED000669767965FAD679768966FAD6897699676
:108EE0007FAD6997CE0101960E9480387BCFC11477
:108EF000D10409F452C00115110509F44EC0F60160
:108F000080858F70843009F044C064E974E185E79E
:108F100099E00E94FD76F6016185728585E799E00A
:108F20000E9497766FE874E185E799E00E94FD76EC
:108F3000B80185E799E00E94977685E799E00E945D
:108F40000676F6016185728540E450E0CE01019617
:108F50000E94D2C90E94BB878823D9F08091020861
:108F6000811117C06FE270E0CE0101960E9499C98D
:108F7000892B51F4F6012185328543E050E060E40D
:108F8000CE0101960E941C24B801CE0101960E94D8
:108F9000C997E114F10409F00ACF81E03ECE011532
:108FA000110509F0ACCF03CF892B09F0AFCEA0CECD
:108FB0008F929F92AF92BF92CF92DF92EF92FF92E9
:108FC0000F931F93CF93DF93CDB7DEB7E0970FB624
:108FD000F894DEBF0FBECDBF84E0E0E1F2E0DE0139
:108FE000119601900D928A95E1F7FE0135968CE17C
:108FF000DF011D928A95E9F7CE010196DB01685FDA
:109000007F4FFD900F2D10E0E4E015950795EA9550
:10901000E1F70E5A1D4FF8011081FC011083EF2D6E
:10902000EF70F0E0EE5AFD4F1081FC0111830296C3
:109030006A177B0731F7198A1A8A8091B4059091D3
:10904000B505892B09F46CC069017A0185E799E0BF
:109050000E9406766FE67AE085E799E00E94FD7649
:1090600042E0C701B6010E94F08F6DE67AE085E725
:1090700099E00E94FD76BE016F5F7F4F85E799E022
:109080000E9497766BE67AE085E799E00E94FD768C
:1090900085E799E00E940676BE016F5F7F4F809161
:1090A0009F069091A0060E94A0874C0120E030E02E
:1090B0004EEF52ECC701B6010E946EC3882381F1C6
:1090C00020E030E04AEA52E4C701B6010E946EC3D4
:1090D000882331F120E030E0A901C701B6010E94E8
:1090E0006EC38823E9F019A61AA61BA61CA68AA59A
:1090F0008F7080678AA7CDA6DEA6EFA6F8AA63E0E8
:10910000CE0189960E945030B12CA12CD12CC12CBB
:1091100079018A019B01AC016FEFC4010E94914566
:10912000E0960FB6F894DEBF0FBECDBFDF91CF91B2
:109130001F910F91FF90EF90DF90CF90BF90AF9075
:109140009F908F9008956F927F928F929F92AF928F
:10915000BF92CF92DF92EF92FF920F931F93CF9324
:10916000DF93CDB7DEB7A0970FB6F894DEBF0FBE82
:10917000CDBF8C01862E7A01DC018D919C911197D7
:10918000892B09F460C01496ED91FC91309709F495
:109190005AC080818071BFEF6B1357C0B1F481E07A
:1091A000A0960FB6F894DEBF0FBECDBFDF91CF9172
:1091B0001F910F91FF90EF90DF90CF90BF90AF90F5
:1091C0009F908F907F906F9008954330510539F3B1
:1091D000818082942FE0822269E176E085E799E040
:1091E0000E94FD76D80113966C9185E799E00E9464
:1091F000308C67E176E085E799E00E94FD76D80142
:109200001496ED91FC9161816F7085E799E00E9461
:10921000308C64E176E085E799E00E94FD76682D68
:1092200085E799E00E94308C85E799E00E940676F8
:10923000D8011496ED91FC9181818F70881207C03E
:1092400080818F7E808380E0ABCF8111FCCF198E2F
:109250001A8E1B8E1C8E1D8E1E8E1F8E18A28A8D3E
:109260008F708A8FD8011496ED91FC9181818F7057
:10927000881579F1B3E0EB16F10459F162E176E07B
:1092800085E799E00E94FD76F801638185E799E022
:109290000E94308C60E176E085E799E00E94FD76DF
:1092A000D8011496ED91FC9161816F7085E799E08A
:1092B0000E94308C6DE076E085E799E00E94FD76B3
:1092C000682D85E799E00E94308C85E799E00E943F
:1092D0000676F80120813181FCE0F81508F416C10A
:1092E000E82DF0E08827E858F64B8F4F0C9443C5E3
:1092F0008549C249434A5A4A664A434A1C4A434A34
:10930000694A744A304A774A834AD8011496CD9004
:10931000DC90F60181818F70853009F4F7C050F43C
:109320008230C1F062E374E0C9010E94A0873C0171
:10933000912C4BC08730D1F08A30A1F76BE274E0FA
:10934000C9010E94A0873C01D6019C9092FA992401
:1093500090F83BC065E274E0C9010E94A0873C011F
:10936000D6019C9090FA992490F82FC064E274E0A2
:10937000C9010E94A0873C01F601908091FA9924CE
:1093800090F823C067E374E0C9010E94A0873C0104
:10939000D8011496ED91FC91808180FB992490F87E
:1093A000982F9E7F80FF916090836114710469F40F
:1093B00061E0CE0149960E947730298B3A8B4B8B26
:1093C0005C8B6D8B7E8B8F8B988FF801A080B1802A
:1093D00066E074E0C5010E94A0876C016BE074E058
:1093E000C5010E94A0875C01892B81F4C114D104BE
:1093F00069F460E0CE0149960E94773029833A8370
:109400004B835C836D837E838F839887D80114960A
:10941000ED91FC916114710409F07CC0898D81117A
:1094200079C0B82DBF708B2E8181807F882A818280
:1094300080818F7E8083B3CE6CE374E0C9010E948B
:10944000A0873C01D8011496ED91FC91808181FBAD
:10945000992490F8982F9D7F81FF92609083B5CFDB
:1094600062E474E0C9010E94A0873C01D80114960F
:10947000ED91FC91808182FB992490F8982F9B7F3D
:1094800082FF9460EBCF62E374E0C9010E94A08781
:109490003C01892B09F04CCF62E0CE0149960E9435
:1094A000773029873A874B875C876D877E878F87E0
:1094B000988B3ECF68E474E0C9010E94A0873C010C
:1094C000D8011496ED91FC9190804CCF6DE474E03E
:1094D000F3CF63E574E0C9010E94A0873C01D80185
:1094E0001496ED91FC9149CF69E574E0F4CF60E604
:1094F00074E0C9010E94A0873C01D8011496ED9147
:10950000FC91908023CF66E674E0F3CF912C712C10
:10951000612C5BCF83E0E816F104B9F0982D9F70C1
:10952000892E8181807F882A818280818F7E8083BD
:10953000E98CFA8C0B8D1C8D2D8D3E8D4F8D58A195
:10954000692DC3010E9491452ACE81818F708815B3
:1095500009F425CE829490EF8922882A8182808125
:10956000806168CF2F923F924F925F926F927F926D
:109570008F929F92AF92BF92CF92DF92EF92FF9223
:109580000F931F93CF93DF93CDB7DEB7A5970FB699
:10959000F894DEBF0FBECDBF5C013B01D0909C05AF
:1095A000DD2009F4B8C0809191068F5F8093910609
:1095B000E0919D06F0919E06309709F4A4C0868044
:1095C000978040909D0650909E064114510409F4E6
:1095D00096C08114910409F492C0D40118968C911C
:1095E0008F70853091F7C4010E943F8C823068F300
:1095F000B401CE0101960E94D71ACE0101960E94B5
:10960000F911882309F45EC060E074E0CE01019690
:109610000E944C17892B09F455C01E8E1F8E18A26C
:1096200019A21AA21BA21CA21DA28F8D8F708F8F50
:1096300040E053E0BE016F5F7F4FCE014E960E9427
:10964000862F67E478E085E799E00E94FD7660E088
:1096500074E0CE0101960E94D0378A859B850097E1
:1096600089F1DC01ED91FC910488F589E02DCC2491
:10967000C394F12CE12C0E8D1F8D28A139A14AA194
:109680005BA16CA17DA119958F3F9807D9F0E98165
:10969000FA8160817181892BE9F485E799E00E9464
:1096A000977665E478E085E799E00E94FD766DE3C2
:1096B00078E085E799E00E94FD7685E799E00E94D1
:1096C0000676D12CF40182809380CE0101960E940F
:1096D0002F1277CF85E799E00E9497766BE378E0C9
:1096E00085E799E00E94FD7667E378E085E799E0F9
:1096F0000E94FD7685E799E00E940676E3CF85E734
:1097000099E00E940676809191068150809391069F
:10971000D11010929C0565E0D5018D919C910E941D
:1097200015884C01009709F483C0FC01D084D594BE
:10973000D594D594D59421843284438454840E9452
:10974000FB96DD2009F474C0261A370A480A590A24
:109750001E8E1F8E18A219A2DE8E1F8D1F70106A1A
:109760001F8F2AA23BA24CA25DA2F4E06F167104E7
:1097700039F5E12C90E1F92E0D2D28A139A14AA14E
:109780005BA16CA17DA1C5010E94E497C201B1015A
:1097900028EE33E040E050E00E94DAC4BA01A901AB
:1097A0002AE030E085E799E00E9411766CE578E0E8
:1097B00085E799E00E94FD7685E799E00E940676AC
:1097C00057FE36C022E022163104410420E852063A
:1097D0007CF1E12C80E1F82E0E8D1F8D28A139A19E
:1097E0004AA15BA16CA17DA1C5010E94E4971982E9
:1097F0001A821B821C821D821E821F8218861A8179
:109800001F701A83D982CC24C394F12CE12C0D2D26
:109810002B813C8140E05E816F817885C5010E948B
:109820008038D40118968C9118978F7018968C9365
:10983000B1E06B167104B9F460E073E0C5010E94F9
:109840004C17009781F020919B0630919C062630A2
:10985000310549F4BC01C5010E941A3860E073E08B
:10986000C5010E94D037F501818592850097D9F412
:1098700090E080E0A5960FB6F894DEBF0FBECDBF96
:10988000DF91CF911F910F91FF90EF90DF90CF90DC
:10989000BF90AF909F908F907F906F905F904F9010
:1098A0003F902F900895DC01ED91FC910484F585A3
:1098B000E02D1995892BE1F2F50181859285DC0176
:1098C000ED91FC910480F581E02DB3011995D2CF83
:1098D000AF92BF92CF92DF92EF92FF920F931F93BE
:1098E000CF93DF93CDB7DEB76D970FB6F894DEBF99
:1098F0000FBECDBF0E94FB969B01AC016091AE05EF
:109900007091AF058091B0059091B105A12CB12C5B
:10991000650118EEE12E13E0F12E00E010E00E9448
:10992000BA23F82E882351F00E94FB966093AE056F
:109930007093AF058093B0059093B1058091910627
:109940008F5F80939106E0919D06F0919E060681BF
:10995000178194E0C92ED12CF11003C082E0C82EEB
:10996000D12CA0909D06B0909E06A114B10429F1BF
:109970000115110511F1F80180858F708530A9F767
:10998000C8010E943F8C823080F3B801CE0101965D
:109990000E94D71ACE0101960E94F911882329F05E
:1099A000B601CE0101960E94B24AF80102811381EC
:1099B000CE0101960E942F12D4CF80919106815042
:1099C0008093910680919B0690919C060597D9F112
:1099D000FF20C9F110E06091B6057091B7056115DF
:1099E000710589F111112FC0FB0180858F708530C1
:1099F00091F4CE0101960E94D71A61E070E0CE0189
:109A000001960E94B24A11E0892B09F410E0CE01C0
:109A100001960E942F12E091B605F091B70530979C
:109A200091F0828193819093B7058093B605892B3D
:109A300091F6E0919D06F0919E0686819781909324
:109A4000B7058093B6056D960FB6F894DEBF0FBECE
:109A5000CDBFDF91CF911F910F91FF90EF90DF90DD
:109A6000CF90BF90AF9008954F925F926F927F9288
:109A70008F929F92AF92BF92CF92EF92FF920F93ED
:109A80001F93CF93DF93CDB7DEB76D970FB6F894E2
:109A9000DEBF0FBECDBF009709F4A4C0FC01208536
:109AA0002F70253009F09EC02A015B0186809780C7
:109AB000809191068F5F809391068114910409F43F
:109AC0008CC0F40180858F70843009F082C061857C
:109AD000728580919D0690919E060E94A0873C0110
:109AE000009709F476C0FC0180858F70853009F0FD
:109AF00070C0B301CE0101960E94D71AA114B1041F
:109B0000A9F0CE0101960E94F911882379F0C12CA9
:109B10007201F501008111812281338144815581D7
:109B200066817781CE0101960E94803860E0C30192
:109B30000E9415880097D1F1FC0120852F702230FA
:109B4000A9F581859285A385B4850797A105B105FF
:109B500069F561E0C3010E941588A201B5010E9468
:109B6000344DA114B10489F5882379F180919106CF
:109B7000815080939106CE0101960E942F1281E0C0
:109B80006D960FB6F894DEBF0FBECDBFDF91CF91BB
:109B90001F910F91FF90EF90CF90BF90AF909F904B
:109BA0008F907F906F905F904F900895A114B104B3
:109BB00061F4CE0101960E94F911882331F0CE01A3
:109BC00001960E94F44D892B89F6CE0101960E94E0
:109BD0002F12F4018280938070CF80919106815082
:109BE0008093910680E0CCCFDF92EF92FF920F93AB
:109BF0001F93CF93DF9300D000D01F921F92CDB759
:109C0000DEB77C0119821A821B821C821D821E8291
:109C10001F8218868A818F708A83D701ED91FC910B
:109C20006081718185E799E00E94977665E378E02D
:109C300085E799E00E94FD76C7010E94F911811124
:109C40001BC06CE278E085E799E00E94FD7685E72D
:109C500099E00E9406760FEF1FEFC80128960FB615
:109C6000F894DEBF0FBECDBFDF91CF911F910F9152
:109C7000FF90EF90DF900895C7010E949617D82EAD
:109C8000F70181859285009791F0DC01ED91FC91BF
:109C90000688F789E02D19958C0197FD08C081E0B1
:109CA0000115110509F480E00E94A214D6CFF70136
:109CB0008085873059F0F5E0DF1689F1FD15F8F061
:109CC00081E0D81619F1A2E0DA1649F140E052E03D
:109CD000B701CE0101960E94862FF701808587305B
:109CE00009F444C010F5833009F469C0843011F1DF
:109CF0006DE178E085E799E00E94FD7613C0B6E05B
:109D0000DB1621F086EF8D0D833000F76DE078E0F3
:109D100085E799E00E94FD7601E010E09ECF80E0AB
:109D20000E94A21410E000E098CF883009F447C0E8
:109D30008930F1F6CE0101960E9422888C0162E101
:109D400078E085E799E00E94FD76B80185E799E023
:109D50000E94378C85E799E00E94067691E080E0CA
:109D6000012B09F490E0092F182F77CF0280F3819F
:109D7000E02D80858F7010E000E0853001F76AE209
:109D800078E085E799E00E94FD7650E040E070E0E1
:109D900060E0F701828193810E94344DF82E082FF4
:109DA00010E067E278E085E799E00E94FD768F2D6C
:109DB0000E94A21485E799E00E9406764ECFCE015C
:109DC00001960E9499308B01BACF2F923F924F9209
:109DD0005F926F927F928F929F92AF92BF92CF923B
:109DE000DF92EF92FF920F931F93CF93DF93CDB744
:109DF000DEB760970FB6F894DEBF0FBECDBF6130FF
:109E0000710509F494C0DC0112966D917C91611585
:109E1000710509F48CC04C0119821A821B821C82C4
:109E20001D821E821F8218868A818F708A8340E07D
:109E300052E0CE0101960E94862FCE0101960E942B
:109E400022881C01F401828193810E9430172B012A
:109E50003C01D40117962D913D914D915C911A973B
:109E6000D1010E9404C52FEF30E040E050E00E9495
:109E7000B8C429873A874B875C870E94FB969B0171
:109E8000AC0189859A85AB85BC850097A105B10594
:109E900009F468C0A12CB12C65017C018D01C301BE
:109EA000B2010E94BA2389874114510461047104EC
:109EB000F1F1D40117968D919D910D90BC91A02D3B
:109EC0008D879E87AF87B88B0E94FB969B01AC0164
:109ED0008D859E85AF85B8890097A105B10561F094
:109EE000A12CB12C65017C018D01C301B2010E943E
:109EF000BA23882309F451C0D40112966D907C9046
:109F000080E00E94F513AB01BC01C3010E94ED1A71
:109F1000232869F0F40184810E94F310D40116967D
:109F20009C91891304C061E0C4010E94A31790E0D2
:109F300080E060960FB6F894DEBF0FBECDBFDF9114
:109F4000CF911F910F91FF90EF90DF90CF90BF9036
:109F5000AF909F908F907F906F905F904F903F90C9
:109F60002F90089591E099879FCFB985BB23F1F099
:109F700060E0C4010E94A317F401828193810E94D2
:109F8000F44D892BA1F640E050E0BA01D4011296BD
:109F90008D919C910E94ED1ACACFF40184810E9498
:109FA000F310D40116969C918913DFCF232809F46E
:109FB000BECFF40184810E94F310D40116969C91C7
:109FC0008913B5CFB985B111B2CFADCFCF93DF93A0
:109FD000EC016EE973E185E799E00E94FD766C8102
:109FE0007D8185E799E00E94378C68E973E185E718
:109FF00099E00E94FD7685E799E00E94067661E08F
:10A000008C810E9445936E818C810E9417938A8176
:10A010009B81009729F040E050E0BA010E94ED1AC0
:10A0200081E090E09093BA058093B9058A819B8185
:10A030000E94F44D181619065CF40A80DB81C02DCD
:10A0400080E00E94F513AB01BC01CE010E94ED1A25
:10A0500081E090E0DF91CF9108952F923F924F924F
:10A060005F926F927F928F929F92AF92BF92CF92A8
:10A07000DF92EF92FF920F931F93CF93DF93CDB7B1
:10A08000DEB7C955D1090FB6F894DEBF0FBECDBFFC
:10A090000E94FB969B01AC016091AA057091AB05F3
:10A0A0008091AC059091AD05A12CB12C650110E318
:10A0B000E12E15E7F12E00E010E00E94BA2388237C
:10A0C00009F401C2E0919D06F0919E06309709F4D3
:10A0D000FAC1809191068F5F809391062680378028
:10A0E00010E02114310409F434C1F10180858F702E
:10A0F0008530F9F460E0C1010E941588FC0181857A
:10A100009285A385B4850597A105B10591F4B101A8
:10A11000CE0101960E94D71ACE0101960E94F91134
:10A1200066968FAF6697811108C0CE0101960E9496
:10A130002F12F10122803380D4CF25961CAE1DAEA4
:10A140001EAE1FAE259729961CAE1DAE1EAE1FAECD
:10A15000299740E052E0BE016F5F7F4FCE018F5BD9
:10A160009F4F0E94862FCE0101960E9430176B01EF
:10A170007C0169966FAF69976A96DFAE6A97CE01E8
:10A1800001960E944C8C4C01CE018F5B9F4F0E9428
:10A19000901165966CAF7DAF8EAF9FAF6597CE0186
:10A1A00001960E949617182FB601DD0C880B990BAB
:10A1B0000E9475C320E030E048EC52E40E94CEC516
:10A1C0002B013C01CE0101960E94F44D68969FAF91
:10A1D0008EAF689765EF72E185E799E00E94FD76A2
:10A1E00042E065966CAD7DAD8EAD9FAD65970E94EA
:10A1F000F08F6FEE72E185E799E00E94FD7642E014
:10A20000C301B2010E94F08F69EE72E185E799E027
:10A210000E94FD76612F70E085E799E00E94378CFF
:10A22000E114F10409F48EC088E00E94F5139B014B
:10A23000AC0144275527B70190E080E0AA24AA94F6
:10A24000BA2CC12CD12C17E2E12E19E0F12E00E03E
:10A2500010E00E94BA23882371F1F10160817181BD
:10A260008EEC98E00E94977669ED72E18EEC98E0B2
:10A270000E94FD76F101608171818DE694E00E947B
:10A28000389A90E080E0BC0169964FAD69976A9674
:10A290005FAD6A97CE0101960E94ED1A62E070E010
:10A2A000C4010E94A216CE0101960E942F1266964A
:10A2B0001FAD66973ECF20E030E048E152E4C30195
:10A2C000B2010E9476C618163CF4F10160817181DA
:10A2D00089E794E00E94389A68968EAD9FAD6897A2
:10A2E000892B19F461E070E0DBCF20E030E040E83A
:10A2F0005FE365966CAD7DAD8EAD9FAD65970E94B9
:10A3000061C59B01AC01C301B2010E946EC370E044
:10A3100060E087FDC5CFA301920165966CAD7DAD70
:10A320008EAD9FAD65970E946EC31816DCF66AEC81
:10A3300072E185E799E00E94FD7685E799E00E9449
:10A340000676B1CF60EC72E185E799E00E94FD7678
:10A35000AACF809191068150809391060E94FB962E
:10A360006093AA057093AB058093AC059093AD05FF
:10A370000E9448112B013C010E94FB966B017C015D
:10A380000E94BB87882309F468C08091020881116C
:10A3900064C030E020E041E050E060E4CE0101968E
:10A3A0000E941C2440E450E062EC78E1CE0101966A
:10A3B0000E948FBA6AEB73E0CE0101960E948EC9AB
:10A3C00040E450E067E972E1CE0101960E948FBA45
:10A3D0002AE0AE014F5B5F4FC301B2010E941ABB7E
:10A3E000BE016F5B7F4FCE0101960E94C99730E09E
:10A3F00020E041E050E060E4CE0101960E941C2480
:10A4000040E450E062EC78E1CE0101960E948FBA00
:10A410006AEB73E0CE0101960E948EC940E450E0E1
:10A4200060E972E1CE0101960E948FBAC701B601C0
:10A4300028EE33E040E050E00E94B8C4CA01B90100
:10A440002AE0AE014F5B5F4F0E941ABBBE016F5BFB
:10A450007F4FCE0101960E94C997112309F44DC088
:10A460006AEB72E185E799E00E94FD760E9448114F
:10A47000AB01BC0185E799E00E942D8C62EB72E193
:10A4800085E799E00E94FD7660919106062E000C0A
:10A49000770B85E799E00E94378C60EA72E185E7E7
:10A4A00099E00E94FD764091A6055091A705609124
:10A4B000A8057091A90585E799E00E942D8C85E794
:10A4C00099E00E940676C75ADF4F0FB6F894DEBFB8
:10A4D0000FBECDBFDF91CF911F910F91FF90EF90F5
:10A4E000DF90CF90BF90AF909F908F907F906F90B4
:10A4F0005F904F903F902F90089560EB72E185E759
:10A5000099E00E94FD760E944811AB01BC0185E7ED
:10A5100099E00E942D8C68EA72E1B2CF3F924F928F
:10A520005F926F927F928F929F92AF92BF92CF92E3
:10A53000DF92EF92FF920F931F93CF93DF93CDB7EC
:10A54000DEB7CE56D1090FB6F894DEBF0FBECDBF31
:10A55000DC0114962D913C91232B09F41FC69B011D
:10A56000225031092230310508F091C23B014C01E3
:10A57000FC018281803409F4F7C208F04AC08430BB
:10A5800008F085C280919B058F5F80939B05A30196
:10A590006FEFC4010E94A348D40112960C91129748
:10A5A0000695017013961C9113978AEC810F8031E8
:10A5B00008F043C066E874E08D919C910E94A087EA
:10A5C0007C010097D1F1FC0180858F708530A9F561
:10A5D0008091B409181324C08091B509803401F525
:10A5E0008091B6099091B7095C01990FCC08DD08FC
:10A5F00060E0C7010E941588FC0181859285A385D2
:10A60000B485A816B906CA06DB060CF065C0512C45
:10A610003EC0823409F4A8C208F439C28058AFCFD2
:10A620001093B40980E48093B509812F0E9481932F
:10A630009093B7098093B609D7CF212F30E0F90165
:10A64000EC5CF54E8491F901EC56F54E1491F9014C
:10A65000E652F54EF490FF2009F43BC081110E94B0
:10A66000B092EF2DF0E0EE0FFF1FED50FA4FA591E5
:10A67000B491EC911E2331E020E009F430E0832F07
:10A68000922F552453940817190609F0C0CFF3E010
:10A690006F16710409F488C0D4011496ED91FC91F1
:10A6A000E181EF70E150EC3008F07EC0F0E08827E7
:10A6B000E35AFC4A8F4F0C9443C57E53FA54B4536B
:10A6C000EA53FA540354FA54375464547D54BF5433
:10A6D000E15490E080E0D5CF61E0C7010E94158889
:10A6E00055245394FC0181859285A385B4858A15F0
:10A6F0009B05AC05BD050CF0CACF89CF0E94FB9627
:10A700009B01AC0144275527D4011496ED91FC918F
:10A710006281738190E080E0AA24AA94BA2CC12CB3
:10A72000D12C18EEE12E13E0F12E00E010E00E9493
:10A73000BA238823C9F1F4010081118168E474E02F
:10A74000C8010E94A087892B41F46DE474E0C80120
:10A750000E94A087892B09F40EC142E050E063E01B
:10A76000C4010E94A34820C00E94FB969B01AC013B
:10A7700044275527D4011496ED91FC916281738191
:10A7800090E080E0AA24AA94BA2CC12CD12C1CE21F
:10A79000E12EFF24F39400E010E00E94BA2342E08F
:10A7A00050E064E0811184C0D4011496ED91FC91D5
:10A7B000808183FB992790F9951509F4D2C1982FD0
:10A7C000907E09F439C1982F907E90528F71892B19
:10A7D000808358C10E94FB969B01AC0144275527FA
:10A7E000D4011496ED91FC916281738190E080E038
:10A7F000AA24AA94BA2CC12CD12C16E9E12EF12C52
:10A8000000E010E0CACF0E94FB969B01AC014427F8
:10A810005527D4011496ED91FC916281738190E0EB
:10A8200080E0AA24AA94BA2CC12CD12C18EEE12ED7
:10A8300013E0F12E00E010E00E94BA23882309F40F
:10A84000B3CFF4010081118163E574E0C8010E9477
:10A85000A087892B41F469E574E0C8010E94A087B4
:10A86000892B09F488C042E050E068E079CF0E946B
:10A87000FB969B01AC0144275527D4011496ED911A
:10A88000FC916281738190E080E0AA24AA94BA2CA2
:10A89000C12CD12C1CE2E12EFF24F39400E010E047
:10A8A0000E94BA2342E050E069E0882309F47CCF9B
:10A8B000C4010E94A3480E94FB96D4011496ED9116
:10A8C000FC917383628370CF0E94FB969B01AC0165
:10A8D00044275527D4011496ED91FC916281738130
:10A8E00090E080E0AA24AA94BA2CC12CD12C16E9BD
:10A8F000E12EF12C00E010E0D3CF0E94FB969B01EB
:10A90000AC0144275527D4011496ED91FC91628146
:10A91000738190E080E0AA24AA94BA2CC12CD12C97
:10A9200018EEE12E13E0F12E00E010E00E94BA23B1
:10A93000882309F439CFF4010081118160E674E0C5
:10A94000C8010E94A087892B39F466E674E0C8012B
:10A950000E94A087892B21F042E050E06BE000CFFD
:10A9600062E474E0C8010E94A08742E050E066E023
:10A97000892B09F4F5CE42E050E06DE0F1CE0E9463
:10A98000FB969B01AC0144275527D4011496ED9109
:10A99000FC916281738190E080E0AA24AA94BA2C91
:10A9A000C12CD12C1CE2E12EFF24F39400E010E036
:10A9B0000E94BA23882309F4F7CE42E050E06CE00D
:10A9C00077CF0E94FB969B01AC0144275527D40109
:10A9D0001496ED91FC916281738190E080E0AA244D
:10A9E000AA94BA2CC12CD12C16E9E12EF12C00E04E
:10A9F00010E0DECF0E94FB969B01AC014427552757
:10AA0000D4011496ED91FC916281738190E080E015
:10AA1000AA24AA94BA2CC12CD12C18E5E12E12E05C
:10AA2000F12E00E010E00E94BA23882309F4BCCE86
:10AA300042E050E060E094CE0E94FB96D401149670
:10AA4000ED91FC91159773836283E181EF7055203E
:10AA500009F445C0E230F1F050F4EE23E9F1D401FD
:10AA60001496ED91FC91808150FA83F9B1CEE530D6
:10AA700089F0A3016AE0E73091F7C4010E94A3487E
:10AA80008111EDCF80919B05815080939B0590E0D3
:10AA900080E086C3F401008111816CE374E0C80199
:10AAA0000E94A087892BA9F463E574E0C8010E9485
:10AAB000A087892B71F469E574E0C8010E94A08722
:10AAC000892B39F464E274E0C8010E94A087892BC5
:10AAD00019F0A30166E0D1CFA30161E0CECFE15030
:10AAE000ED3008F0BCCFF0E08827E658FA4A8F4FE7
:10AAF0000C9443C587552F558A558A552F558D552A
:10AB00002F55AE55AE55AE55AE55AE558A55A3012F
:10AB100062E0B3CFA30165E0B0CF0D911C916CE36F
:10AB200074E0C8010E94A087892BA9F463E574E052
:10AB3000C8010E94A087892B71F469E574E0C801FF
:10AB40000E94A087892B39F464E274E0C8010E9456
:10AB5000A087892B19F0A30167E08FCFA30160E0E4
:10AB60008CCF8F71806434CEB3E06B16710409F41E
:10AB70008ECF66E874E0F401808191810E94A08705
:10AB80008C01D40113968C919091B4098913EBC078
:10AB90009091B509903409F0E6C08091B609909182
:10ABA000B7093C010115110509F40DC1F801208513
:10ABB0002F70253009F007C1C8010E943F8C382E44
:10ABC000F3E0F81708F0DBC063E0C8010E941588C5
:10ABD000DC0119968D919C913AE0E32EE89E60018C
:10ABE000E99ED00C1124A396DFAECEAEA39762E00F
:10ABF000C8010E941588DC0119968D919C91E89EF0
:10AC00002001E99E500C11246201052C000CEE0875
:10AC1000FF08AF96CCAEDDAEEEAEFFAEAF9761E013
:10AC2000C8010E9415885C0160E0C8010E94158877
:10AC3000DC011996CD90DD90ED90FC901C97A796C5
:10AC4000CCAEDDAEEEAEFFAEA7979301072C000CA5
:10AC5000440B550B2C193D094E095F09A396CEAC48
:10AC6000DFACA397B601DD0C880B990BAF96CCAC8B
:10AC7000DDACEEACFFACAF976C197D098E099F0976
:10AC80000E94A8C4D50119962D913D914D915C91DA
:10AC90001C97A796CCACDDACEEACFFACA7972C19FB
:10ACA0003D094E095F09A7962CAF3DAF4EAF5FAF90
:10ACB000A7970E94DAC4AF96ACACBDACCEACDFAC0B
:10ACC000AF97A20EB31EC41ED51E45E0E42E3E145F
:10ACD00009F468C081E090E0A396EEACFFACA397C6
:10ACE000A701FF0C660B770B4A155B056C057D050C
:10ACF0000CF461C0B601A5016201052C000CEE0840
:10AD0000FF084C155D056E057F050CF459C06A01FE
:10AD10007B0122E032126BC06301770CEE08FF0862
:10AD200060E0C8010E941588FC0181859285A38599
:10AD3000B485C816D906EA06FB060CF44AC261E0DF
:10AD4000C8010E941588FC0181859285A385B48580
:10AD50008C159D05AE05BF050CF099CE81E090E005
:10AD6000A0E0B0E039C28093B40990E49093B509B3
:10AD70000E9481939093B7098093B60912CF8AE01D
:10AD8000869D5001879DB00C11240B2C000CCC0823
:10AD9000DD08512C412C20E038E2A3963FAF2EAFC6
:10ADA000A39798CF64E0C8010E941588DC0119962A
:10ADB0008D919C9191CF66246A9423E0722E9CCF52
:10ADC000712C612CA6CF2AE0289F6001299FD00C0E
:10ADD00011240D2C000CEE08FF08512C412C20E012
:10ADE00038E2A3963FAF2EAFA39781E090E0D40165
:10ADF0001496ED91FC9162817381A301461B570B60
:10AE000057FF03C0519541955109841795070CF4DC
:10AE1000BFC08081982F929596959770963008F0D4
:10AE2000BAC09F5F9295990F907E8F71892BB2C0A7
:10AE3000F70161857285DB018C9181115AC2A114E1
:10AE4000B10409F472C0D50118968C9118978F70CF
:10AE5000843009F06AC019966D917C91CE010196FB
:10AE60000E94F235CE0101960E94F911882309F45F
:10AE700058C06114710409F45FC0E114F10431F0A9
:10AE8000F70180858F70843009F441C025961CAE8F
:10AE90001DAE1EAE1FAE259729961CAE1DAE1EAE72
:10AEA0001FAE299723961FAD23971F7023961FAFC0
:10AEB000239781E022968FAF2297CC24C394F12C64
:10AEC000E12C01E024962FAD249725963FAD2597E0
:10AED00040E027965FAD279728966FAD2897299673
:10AEE0007FAD2997CE0101960E9480381AC00115C6
:10AEF000110529F0F80180858F70843019F06DE814
:10AF000074E0F7C161857285FB01808196CF618510
:10AF10007285FB018081882321F0CE0101960E9479
:10AF2000018DCE0101960E942F12D4011496ED914D
:10AF3000FC9173826282ABCD0115110531F0D8010D
:10AF400018968C918F708430E9F025961CAE1DAE5A
:10AF50001EAE1FAE259729961CAE1DAE1EAE1FAEAF
:10AF6000299723961FAD23971F7023961FAF239712
:10AF700082E022968FAF2297CC24C394F12CE12C4F
:10AF800002E0A0CFF80161857285DB018C91C3CF0F
:10AF900080818F7180838081803AB8F0C201550C26
:10AFA000AA0BBB0BC816D906EA06FB0671F0A396DE
:10AFB000EEADFFADA397CF01FF0FAA0BBB0BC816D9
:10AFC000D906EA06FB0609F062CD6616770609F493
:10AFD0005ECD6D961CAE1DAE1EAE1FAE6D976B9610
:10AFE0008FAD6B978F7080666B968FAF6B976D96FA
:10AFF0008CAD9DADAEADBFAD6D9765968CAF9DAF81
:10B00000AEAFBFAF6597AAE0B0E0A70196010E947E
:10B01000F9C469966CAF7DAF8EAF9FAF699762EE52
:10B0200075E085E799E00E94FD76D40113966C9156
:10B0300085E799E00E94308C60EE75E085E799E045
:10B040000E94FD76CE018F5A9F4F0E94112E62E022
:10B0500074E0F401808191810E94A087B12CA12C21
:10B06000D12CC12C6296EFAC62976396FFAC6397CC
:10B0700064960FAD649765961FAD659766962FAD84
:10B08000669767963FAD679768964FAD68976996E4
:10B090005FAD69976FEF0E949145D4010D911C91AE
:10B0A00066E074E0C8010E94A0877C016BE074E058
:10B0B000C8010E94A0878C010097E1F1FC01808506
:10B0C0008F708430B9F56185728540E450E0CE011F
:10B0D00001960E94D2C96FE270E0CE0101960E94F3
:10B0E00099C9892B59F4D80119962D913C9143E0C7
:10B0F00050E060E4CE0101960E941C2400E020E0B4
:10B1000032E040E150E0BE016F5B7F4FCE018F5ACD
:10B110009F4F0E94F02B0E94BB87882359F080919B
:10B120000208811107C0BE016F5B7F4FCE010196FF
:10B130000E94C997E114F10409F4F7CEF701808564
:10B140008F70843009F0F1CE61857285CE01019651
:10B150000E94F235CE0101960E94F911882309F46C
:10B16000E0CECC24C394F12CE12C62960FAD629713
:10B1700063961FAD639764962FAD649765963FAD58
:10B18000659766964FAD669767965FAD67976896C9
:10B190006FAD689769967FAD6997A4CE8FEF9FEFEB
:10B1A000C259DF4F0FB6F894DEBF0FBECDBFDF919F
:10B1B000CF911F910F91FF90EF90DF90CF90BF90B4
:10B1C000AF909F908F907F906F905F904F903F9047
:10B1D000089580E090E0DC01F40124813581F901DB
:10B1E00042815381052E000C660B770B841795075F
:10B1F000A607B70709F44BCC3C01D4010D911C9173
:10B2000066E074E0C8010E94A0875C016BE074E016
:10B21000C8010E94A0876C01A114B10419F4892B04
:10B2200009F483CE67E374E0C8010E94A0877C0123
:10B2300062E374E0C8010E94A0878C0168EE75E0AB
:10B2400085E799E00E94FD76F401638185E799E046
:10B250000E94308C66EE75E085E799E00E94FD76ED
:10B26000B30185E799E00E94378C85E799E00E9459
:10B270000676C114D10409F4E2CDD60118968C915A
:10B2800018978F70843009F0DACD19966D917C9102
:10B2900040E450E0CE0101960E94D2C90E94BB87D3
:10B2A000882309F4CCCD809102088111C8CD6FE2CA
:10B2B00070E0CE0101960E9499C9892B51F4F601E4
:10B2C0002185328543E050E060E4CE0101960E9482
:10B2D0001C246114710409F40ACEE114F10439F05C
:10B2E000D70118968C918F70843009F4A1CD6AE84B
:10B2F00074E0CE0101960E94C997A1CD8F929F92D2
:10B30000AF92BF92CF92DF92EF92FF920F931F9373
:10B31000CF93DF9300D000D0CDB7DEB72091B20538
:10B320003091B305232B09F4C5C02091A505211147
:10B33000C1C04C018091A5058F5F8093A5058091C8
:10B3400091068F5F809391060E94FB969B01AC0152
:10B350006091A1057091A2058091A3059091A4052B
:10B36000A12CB12C65011BE0E12EF12C00E010E0D6
:10B370000E94BA23882309F452C0E091B205F091EB
:10B38000B3050681178101151105B9F1F801808512
:10B390008F70863071F562E074E0C8010E94A0876A
:10B3A0000097D1F0FC0120852F702530A9F4E680AC
:10B3B000F780E114F104E9F0FA82E982B801CE01E4
:10B3C00001960E944D1BB401CE0101960E948E523F
:10B3D000F701E280F380EDCF1A83098370E060E02B
:10B3E000CE0101960E944D1BB401CE0101960E9430
:10B3F0008E52F80102811381C6CFF3E08F169104BB
:10B4000051F00E94FB966093A1057093A205809372
:10B41000A3059093A4051092B4091092B50983E096
:10B4200088169104E9F10E94FB969B01AC016091A2
:10B430009D0570919E0580919F059091A005A12C7E
:10B44000B12C650118E8E12E13E1F12E00E010E0C7
:10B450000E94BA23882321F1E091B205F091B3054F
:10B46000068117810115110589F0F80180858F701B
:10B47000863041F41A83098370E060E0CE010196C2
:10B480000E944D1BF80102811381ECCF0E94FB96B4
:10B4900060939D0570939E0580939F059093A005F2
:10B4A000809191068150809391068091A5058150ED
:10B4B0008093A50526960FB6F894DEBF0FBECDBFCC
:10B4C000DF91CF911F910F91FF90EF90DF90CF9080
:10B4D000BF90AF909F908F9008954F925F926F9220
:10B4E0007F92AF92BF92CF92DF92EF92FF920F9333
:10B4F0001F93CF93DF93CDB7DEB76D970FB6F89458
:10B50000DEBF0FBECDBF63E873E185E799E00E941F
:10B51000FD7685E799E00E9406760E94FB962B0156
:10B520003C0180919106882371F10E94FB969B015A
:10B53000AC01A12CB12C650110E1E12E17E2F12E36
:10B5400000E010E0C301B2010E94BA2381111BC0C8
:10B550000E944E788091A10681116BC080919B065C
:10B5600090919C06059741F080919D0690919E06D2
:10B57000892B11F00E94684C0E942D5082E090E0CF
:10B580000E947E59CECF80919106FF24F3948823A8
:10B5900059F060E673E18EEC98E00E94FD768EEC47
:10B5A00098E00E940676F12C6AE473E185E799E061
:10B5B0000E94FD7685E799E00E9406768091B805A5
:10B5C0008F5F8093B805E0919D06F0919E063097BD
:10B5D000D1F10681178101151105A9F1D80118963D
:10B5E0008C918F708530B9F7C8010E943F8C8823F9
:10B5F00091F3F80160817181CE0101960E94F235CC
:10B60000CE0101960E94F911882359F08A859B8505
:10B61000009739F0DC01ED91FC910284F385E02D77
:10B620001995CE0101960E942F12F8010281138113
:10B63000D2CF80919F069091A006892B09F48ECFDE
:10B640000E94B0268BCF1092B7051092B60562E427
:10B6500073E185E799E00E94FD7685E799E00E9415
:10B66000067664E670E080E090E00E94B694109266
:10B670001D06109292066AE273E185E799E00E9446
:10B68000FD760E944811AB01BC0185E799E00E945C
:10B690002D8C8091B4059091B5050E94D2901092A6
:10B6A000B5051092B4051092B3051092B205109230
:10B6B0009E0610929D0610921F0610921E06109272
:10B6C0008F0610928E0610928D0610928C061092A4
:10B6D000A00610929F0665E273E185E799E00E945B
:10B6E000FD760E944811AB01BC0185E799E00E94FC
:10B6F0002D8C85E799E00E94067610929006809145
:10B70000B80581508093B8058F2D6D960FB6F894CB
:10B71000DEBF0FBECDBFDF91CF911F910F91FF9084
:10B72000EF90DF90CF90BF90AF907F906F905F9041
:10B730004F900895809102088F5F80930208A8952A
:10B7400083E090E00E947E590E944E78809102082A
:10B750008150809302080895CF92DF92EF92FF927A
:10B760000F931F93CF93DF93FC012485243059F06E
:10B7700090E080E0DF91CF911F910F91FF90EF90CB
:10B78000DF90CF9008956A018B01EC01F12C8F2D91
:10B790000E941784811127C0FC868C85843041F378
:10B7A00020910202309103022F5F3F4F21F130932D
:10B7B000030220930202409102025091030220E012
:10B7C00061E00E946883F80182818F3FB9F4838130
:10B7D0008F3FF9F484818F3FE1F485818F3FC9F475
:10B7E00084E08C87C5CF8B7F8831B1F2F394F4E08D
:10B7F000FF12CDCFD2CF20E030ECD9CF811109C0DC
:10B800008381811106C08481811103C085818823D1
:10B8100039F3C114D10421F3FC8480E590E00E9447
:10B820002291B8016E5F7F4F8F2D0E94E41CB601FC
:10B830008F2D0E94D31C64E070E08F2D0E948191B7
:10B840000E94FB966B017C01F4E9CF0EF1E1DF1E53
:10B85000E11CF11CCE010E94ED1C873149F161E031
:10B8600070E080E090E00E94B6940E949A5BCE0166
:10B870000E94ED1C882309F4B3CF0E94FB96C616E4
:10B88000D706E806F90630F78C850E945483EC85CC
:10B89000F0E0EE0FFF1FED56F94F1182108284E0A9
:10B8A0008C8761EC75E188ED98E00E94217760CF8C
:10B8B00066EB75E188ED98E00E94217781E090E0E9
:10B8C00059CFA89583E090E00C947E595F926F92D7
:10B8D0007F928F929F92AF92BF92CF92DF92EF9220
:10B8E000FF920F931F93CF93DF93CDB7DEB7A3974C
:10B8F0000FB6F894DEBF0FBECDBF8091B405909116
:10B90000B505892B09F421C48091910681111DC4CC
:10B91000809191068F5F8093910662E27EE084ECD5
:10B9200098E00E94FD7684EC98E00E9406760091F3
:10B93000B4051091B50561E974E0C8010E94A087C3
:10B9400090939E0680939D0667E974E0C8010E946B
:10B95000A08790931F0680931E0662ED74E0C801D5
:10B960000E94A0879093B3058093B2056EE974E0BE
:10B97000C8010E94A08790938F0680938E060E9434
:10B98000272B63EA74E08091B4059091B5050E947D
:10B99000A0879093A00680939F06009709F4BBC1EF
:10B9A0002091A1062111B7C1DC011696ED90FC9003
:10B9B00080918A0690918B06892B51F081E08093CB
:10B9C000A10662E17EE084EC98E00E94FD7655C01D
:10B9D00069ED7DE085E799E00E94FD7685E799E0D5
:10B9E0000E94067663ED7DE085E799E00E94FD7692
:10B9F0000E944811AB01BC0185E799E00E942D8CA3
:10BA000085E799E00E9406768FE090E00E943AB7C1
:10BA10008C0188E1F80181831282108216861586D6
:10BA200010926906109268061092DF0710920108C2
:10BA30000E946E148CE6A82E80E1B82EB0924206C9
:10BA4000A09241069DE6C92E90E1D92ED0924606DD
:10BA5000C092450610938B0600938A06012B09F0CD
:10BA6000B1C061EC7DE08EEC98E00E94FD768EEC3A
:10BA700098E00E9406761092A1061092C4051092DA
:10BA8000C305CC24C394D12CE114F10409F443C1BF
:10BA90008091A106882309F43EC1D70118968C91A4
:10BAA00018978F70863009F089C00D911C91FE01A6
:10BAB00031965F014801F0E18F0E911C3501D801EC
:10BAC0008C910E946411582EF80181810E946411AA
:10BAD0005294A0EF5A22582AD5015D925D010E5F63
:10BAE0001F4F8016910659F76EE37DE084EC98E0D5
:10BAF0000E94FD766091C3057091C40584EC98E0C6
:10BB00000E94378C67E37DE084EC98E00E94FD762C
:10BB10008091C3059091C405F3E0880F991FFA95B1
:10BB2000E1F72091C1053091C205820F931F0E9459
:10BB30009C8F84EC98E00E9406762091C30530919A
:10BB4000C40521313105D4F56091C1057091C2055C
:10BB500048E0C901E3E0880F991FEA95E1F7860FF5
:10BB6000971F415058F1FC01E40FF11D50815523FE
:10BB7000C1F3220F331F4091BB055091BC05240F28
:10BB8000351FF901D182C08228E0F301DC01019068
:10BB90000D922A95E1F7DC018C91883231F4809185
:10BBA0008A0690918B060E94DD208091C3059091BA
:10BBB000C40501969093C4058093C305F701E28004
:10BBC000F38062CF88E890E00E943AB79093C20574
:10BBD0008093C10565EB7DE085E799E00E94FD76E5
:10BBE0000E944811AB01BC0185E799E00E942D8CB1
:10BBF00085E799E00E94067682E290E00E943AB7DB
:10BC00009093BC058093BB0568EA7DE085E799E0E9
:10BC10000E94FD760E944811AB01BC0185E799E0C6
:10BC20000E942D8C85E799E00E9406768091C105DF
:10BC30009091C205892B31F08091BB059091BC0594
:10BC4000892B79F460E97DE08EEC98E00E94FD7626
:10BC50000E944811AB01BC018EEC98E00E942D8C33
:10BC600006CF88ED97E49093BE058093BD051092B2
:10BC70006906109268061092DF07109201080E9470
:10BC80006E14B0924206A0924106D0924606C0922F
:10BC9000450680918A0690918B060E94391081E0BA
:10BCA0000E94C393811130C06DE77DE085E799E084
:10BCB0000E94217700918A0610918B06C8010E948C
:10BCC000391040E060EFC8010E94E9200E94B3945F
:10BCD000E0918A06F0918B0681E080836DE57DE03E
:10BCE00085E799E00E94217780918A0690918B06E2
:10BCF0000E949C20882309F461CE61E57DE085E700
:10BD000099E00E9421775ACE63E47DE085E799E0CF
:10BD10000E942177B0CE1092B7051092B605E0913F
:10BD20009D06F0919E06309709F4F0C0E680F780FA
:10BD300000919D0610919E060115110509F4DFC0C2
:10BD4000E114F10409F4DBC0D70118968C918F70CF
:10BD5000853091F7C7010E943F8C823068F3B701AC
:10BD6000CE0101960E94D71ACE0101960E94F911C8
:10BD7000882309F462C08A859B85009759F5CE0116
:10BD800001960E944C8C8C01912C812C97FF06C04F
:10BD900011950195110988248394912CCE01019667
:10BDA0000E949617C82ED12C8985853009F44EC083
:10BDB000863009F042C0B02E61E0802F0E9445938A
:10BDC00061E0892809F479C0CA94CD2809F079C0C6
:10BDD00060E077C0DC01ED91FC910484F585E02DF5
:10BDE0001995892B49F08A859B85DC01ED91FC91A1
:10BDF0000284F385E02D19958A859B85DC01ED9100
:10BE0000FC910680F781E02D1995892BB1F0CE01C8
:10BE100001960E949617882331F060E071E0CE0110
:10BE200001960E94F4378D819E81892B31F060E06C
:10BE300072E0CE0101960E94F437D7011296ED9080
:10BE4000FC90CE0101960E942F1272CFCD2829F4CA
:10BE500062E0CE0101960E94661760E071E0CE01BB
:10BE600001960E94F4378D819E81892B31F060E02C
:10BE700072E0CE0101960E94F43761E0802F0E94AB
:10BE8000459360E0802F0E9417936AE07EE085E78B
:10BE900099E00E94FD76B80185E799E00E94378C11
:10BEA00065E07EE085E799E00E94FD7663E07EE054
:10BEB00085E799E00E94FD76C0CFCA94CD2809F0AD
:10BEC00087CFC62ED12C8B2D0E9417936EEF7DE06D
:10BED00085E799E00E94FD76B80185E799E00E9428
:10BEE000378C6CEF7DE085E799E00E94FD76B60126
:10BEF00085E799E00E94378C6AEF7DE0D9CFF801A1
:10BF0000868197819093B7058093B60585E799E080
:10BF10000E940676E091B205F091B305309709F4DE
:10BF20008AC0809191068F5F809391060681178168
:10BF30000115110509F47AC0D80118968C918F70FB
:10BF4000863009F069C01F8F0E8F70E060E0CE016F
:10BF50004E960E944D1B8AA19BA1892B09F45CC0BF
:10BF60008091B4059091B505892B09F455C0EE8CEC
:10BF7000FF8CF70180858F70863099F562E074E060
:10BF8000C7010E94A0870097F1F0DC0118962C9160
:10BF900018972F702530B9F41696CD90DC90C11407
:10BFA000D104F9F0DA82C982B701CE0101960E946C
:10BFB0004D1BED81FE811082118212821382F601E7
:10BFC000C280D380ECCFFA82E98270E060E0CE01DB
:10BFD00001960E944D1B62E070E0CE0101960E9426
:10BFE0008E52EAA1FBA1108211821282138288A1D3
:10BFF000843068F462E0823008F060E089A10E9439
:10C000004593EAA1FBA18181807F818305C08034B3
:10C0100041F060E0823431F0D80112960D911C910C
:10C0200087CF62E089A10E944593F6CF8091910667
:10C030008150809391066AE27DE084EC98E00E9452
:10C04000FD7662E27DE084EC98E00E94FD7681E07E
:10C0500020919D0630919E06232B09F480E00E94DA
:10C060008C1469E17DE084EC98E00E94FD7681E02B
:10C070002091B2053091B305232B09F480E00E9492
:10C080008C1462E17DE084EC98E00E94FD7681E012
:10C0900020918E0630918F06232B09F480E00E94B8
:10C0A0008C1469E07DE084EC98E00E94FD7681E0EC
:10C0B00020919F063091A006232B09F480E00E9476
:10C0C0008C1460E07DE084EC98E00E94FD76809125
:10C0D0001D060E948C1484EC98E00E9406766BEF9B
:10C0E0007CE084EC98E00E94FD760E944811AB0150
:10C0F000BC0184EC98E00E942D8C84EC98E00E94B6
:10C10000067681E08093920683E998E00E94F51C10
:10C11000882351F083E998E00E949A1D84E090E022
:10C1200090939C0680939B0680919B0690919C0621
:10C13000079731F484E090E090939C0680939B06EF
:10C1400080919106815080939106A3960FB6F89442
:10C15000DEBF0FBECDBFDF91CF911F910F91FF903A
:10C16000EF90DF90CF90BF90AF909F908F907F9097
:10C170006F905F900895CF93DF93EC01FB012481D2
:10C18000358140815181628173810E941176CE0197
:10C19000DF91CF910895AF92BF92CF92DF92EF924D
:10C1A000FF921F93CF93DF9300D000D0CDB7DEB7BF
:10C1B0006C017C0110E08AE0A82EB12C133061F1F3
:10C1C000F701828190E0B0E0A0E089839A83AB839D
:10C1D000BC83BE82AD82BE016F5F7F4F84EC98E06E
:10C1E0000E94BB606DE774E10E94FD761F5FFFEF68
:10C1F000EF1AFF0A143011F726960FB6F894DEBF37
:10C200000FBECDBFDF91CF911F91FF90EF90DF90D8
:10C21000CF90BF90AF900895F601858190E0B0E097
:10C22000A0E089839A83AB83BC83BE82AD82BE01CA
:10C230006F5F7F4F84EC98E00E94BB606BE774E116
:10C24000D3CF0F931F93CF93DF9300D000D0CDB700
:10C25000DEB70E944F2A62E77AE084EC98E00E9401
:10C26000FD76CE0101960E942591CE0101960E9495
:10C27000CB6005EA13E01A8309838091310890911D
:10C280003208A0913308B09134088B839C83AD832E
:10C29000BE83CE0101960E94CB601A8309831B8264
:10C2A0001C821D821E8280E590E00E94229144E063
:10C2B00050E0BE016D5F7F4F81E090E00E949F7B68
:10C2C000CE0101960E94CB601A8309831B821C82D7
:10C2D0001D821E8280E590E00E94229144E050E0A1
:10C2E000BE016D5F7F4F85E090E00E949F7BCE0195
:10C2F00001960E94CB6068E97AE084EC98E00E94A5
:10C30000FD7688EC90E026960FB6F894DEBF0FBE5F
:10C31000CDBFDF91CF911F910F910895CF92DF9202
:10C32000EF92FF921F93CF93DF9300D000D0CDB751
:10C33000DEB76EE37AE084EC98E00E94FD7688EA4E
:10C34000E82E88E0F82E10E090E1C92ED12CF701FC
:10C3500081917F01803130F466EA74E084EC98E0EA
:10C360000E949776153041F1F7013197808190E076
:10C37000B0E0A0E089839A83AB83BC83DE82CD8268
:10C38000BE016F5F7F4F84EC98E00E94BB606CE35E
:10C390007AE00E94FD761F5F1630C9F626960FB62A
:10C3A000F894DEBF0FBECDBFDF91CF911F91FF90FC
:10C3B000EF90DF90CF9008958091AD0890E0B0E0CD
:10C3C000A0E089839A83AB83BC83DE82CD82BE01E9
:10C3D0006F5F7F4F84EC98E00E94BB600E940676FE
:10C3E000DACFEF92FF920F931F93CF93DF9300D09A
:10C3F00000D01F92CDB7DEB77B01CE0107969F9389
:10C400008F9301979F938F9301979F938F9301979A
:10C410009F938F9301979F938F9301979F938F93F0
:10C420008E010F5F1F4F1F930F9388EA94E09F9335
:10C430008F93DB0113968C9113978F9312968C91A7
:10C440008F930E9459CA0FB6F894DEBF0FBECDBFBE
:10C450000697ECF468E17FE08EEC98E00E94FD76B0
:10C46000D70112966D917C918EEC98E00E949776A0
:10C4700080E991E027960FB6F894DEBF0FBECDBFDE
:10C48000DF91CF911F910F91FF90EF9008958091D0
:10C49000A0089091A108892BA9F10E94FD8888230A
:10C4A00089F181E60E94E8888091A0089091A10816
:10C4B000DC01ED91FC910088F189E02D64E070E0F1
:10C4C00019958091A0089091A108DC01ED91FC9153
:10C4D0000280F381E02D46E050E0B801199586E036
:10C4E000F801A8EAB8E001900D928A95E1F78091F1
:10C4F000A0089091A108DC01ED91FC910488F589D8
:10C50000E02D19950E948E616AE27FE084EC98E04C
:10C510000E94FD7688EC90E0ADCFCF93DF93CDB74E
:10C52000DEB72E970FB6F894DEBF0FBECDBF809159
:10C53000910681116EC06FE67EE084EC98E00E9467
:10C54000FD7684EC98E00E9406761092C008109266
:10C55000BF0880E090E19093BB088093BA0884E81C
:10C5600090E09093C2088093C10881E08093BC085A
:10C5700080E090E29093BE088093BD0882E78093AC
:10C58000C3088EEA98E00E94FD1B8B37910509F0E5
:10C59000AFC01C821B828DE792E09A8389838EEA6A
:10C5A00098E09E838D838FEF9FEF98878F83809194
:10C5B000B4059091B505892B11F00E946D5ACE01FA
:10C5C00001960E9404919093B5058093B4058EEA7C
:10C5D00098E00E943D128091B4059091B505892B99
:10C5E000D9F463E67EE08EEC98E00E94FD768EEC56
:10C5F00098E00E9406766FE175E0CE0109960E94F0
:10C600004475CE0109960E94039DCE0109960E94B1
:10C61000057590E080E014C060E57EE084EC98E071
:10C620000E94FD7684EC98E00E9406760E94665C8B
:10C630008091A0089091A108892B59F481E090E0A5
:10C640002E960FB6F894DEBF0FBECDBFDF91CF910F
:10C6500008950E94FD88882389F382E70E94E88874
:10C660008091A0089091A108DC01ED91FC910088D7
:10C67000F189E02D60E670E019956091A008709155
:10C68000A10840E0CE0109960E948375BE01675F54
:10C690007F4F82EA98E00E940B74CE0109960E94B7
:10C6A00005758091A0089091A108DC01ED91FC91A5
:10C6B0000488F589E02D199562E37EE085E799E02D
:10C6C0000E94FD7662EA78E0CE0109960E943B75F1
:10C6D000BE01675F7F4F85E799E00E94EF7685E7AF
:10C6E00099E00E940676CE0109960E940575A6CFB4
:10C6F0008EEA98E00E945C12892BA1F08EEA98E005
:10C700000E9486126FE175E0CE0101960E94447589
:10C71000CE0101960E94039DCE0101960E940575EF
:10C720000E948C9C8EEA98E00E943D126FE37EE0AE
:10C7300084EC98E00E94FD7684EC98E00E940676F6
:10C7400068CF0E948D62892B49F486EF9FEF90930A
:10C750009C0680939B0684EF91E0089588EC90E01E
:10C760000895AF92BF92CF92DF92EF92FF920F9314
:10C770001F93CF93DF9300D000D0CDB7DEB78C01ED
:10C780006B01B42EFB0184819581892BD9F1E08066
:10C79000F1806FE370E0C7010E9499C9009791F1A1
:10C7A0009C012E193F09790137FD2CC06FE175E01E
:10C7B000CE0101960E944475F6018481958100970F
:10C7C000B9F08E159F0508F47C01F6016081718136
:10C7D000FB01EE0DFF1DA0801082CE0101960E948C
:10C7E000DF74F60180819181E80EF91EF701A082C5
:10C7F000BE016F5F7F4FC6010E940B74CE01019690
:10C800000E9405756CEB74E0C6010E948673882354
:10C8100029F1F801128A118A80E090E195878487D6
:10C8200084E890E0948B838B81E0868780E090E2BF
:10C83000908B8787B58A81E090E026960FB6F894B2
:10C84000DEBF0FBECDBFDF91CF911F910F91FF9043
:10C85000EF90DF90CF90BF90AF90089569EC74E0B7
:10C86000C6010E948673882369F0F801128A118A32
:10C87000148A138A84E890E095878487168680E07E
:10C8800090E3D6CF90E080E0D8CFFF920F931F9334
:10C89000CF93DF9300D000D0CDB7DEB78C01BC01C1
:10C8A000CE0101960E943B75BE016F5F7F4F85E709
:10C8B00099E00E94EF7685E799E00E940676CE0126
:10C8C00001960E9405756DE87FE0CE0101960E94F9
:10C8D0000D75BE016F5F7F4FC8010E946B73F82E0C
:10C8E000CE0101960E940575FF2069F0B801CE01C6
:10C8F00001960E943B75CE0101960E94039DCE01D8
:10C9000001960E94057526960FB6F894DEBF0FBEFD
:10C91000CDBFDF91CF911F910F91FF9008955F924E
:10C920006F927F928F929F92AF92BF92CF92DF923F
:10C93000EF92FF920F931F93CF93DF93CDB7DEB7A4
:10C94000CF56D1090FB6F894DEBF0FBECDBF4C0154
:10C950008B01F42E642F85E799E00E94308C60ED06
:10C9600079E085E799E00E94FD76B801CE01019655
:10C970005C010E943B75B50185E799E00E94EF7666
:10C9800085E799E00E940676C5010E94057592E050
:10C99000F9126BC26EEC79E0C5010E940D75B5010C
:10C9A000C8010E949B73F82EC5010E940575FF20E7
:10C9B00009F4D0C220E04DE251E0B40181E798E0F3
:10C9C0000E949F77E0908C06F0908D0667EC79E0EE
:10C9D000CE0186599F4F0E940D7560EC79E0CE0123
:10C9E0008C599F4F0E940D75CE01885A9F4F0E940F
:10C9F00025916E961FAD6E976D960FAD6D976C96E7
:10CA0000DFAC6C976B96CFAC6B976FE175E0CE01A6
:10CA100081960E944475BE016F5D7F4FC5010E94E3
:10CA20003B756C2DC5010E94567465ED74E00E9443
:10CA300087746D2D0E94567465ED74E00E948774B2
:10CA4000602F0E94567465ED74E00E948774612F18
:10CA50000E945674BC01CE01825A9F4F0E943B75C2
:10CA6000C5010E940575CE0181960E9405756BEB8C
:10CA700079E0CE018E5A9F4F0E940D756FE175E0EF
:10CA8000CE01845B9F4F0E94447500EA18E0D801F4
:10CA900018966C9170E084E0759567958A95E1F73A
:10CAA000C5010E94BC884D815E8169817A81CE0179
:10CAB000845B9F4F0E94CB73C5010E940575F801EE
:10CAC00060856F7070E0C5010E94BC884D815E81F9
:10CAD00069817A81CE01845B9F4F0E94CB73C5012F
:10CAE0000E9405750F5F1F4FF8E0063A1F0779F6A1
:10CAF00065EB79E0CE018A5B9F4F0E940D7564E97A
:10CB000079E0CE0181960E940D75BE016F5D7F4F69
:10CB1000CE01CE960E943B75BE016A5B7F4FCE016F
:10CB2000CE960E94A174BE01645B7F4F0E94A174E7
:10CB3000BE016E5A7F4F0E94A174BE01625A7F4FA0
:10CB40000E94A174BE016C597F4F0E94A1748C0198
:10CB50004AE0B50180E590E00E94F2BAF50101904B
:10CB60000020E9F73197AF014A195B09B501C80107
:10CB70000E94CB73811103C0C8010E944474BE019E
:10CB800066597F4FC8010E94A174B7010E94877443
:10CB9000BC01C4010E94EF76C4010E940676CE015A
:10CBA000CE960E940575CE0181960E940575CE0134
:10CBB0008A5B9F4F0E940575CE01845B9F4F0E9448
:10CBC0000575CE018E5A9F4F0E940575CE01825A7F
:10CBD0009F4F0E940575CE018C599F4F0E9405758D
:10CBE000CE0186599F4F0E940575C4010E940676AA
:10CBF00064E670E080E090E00E94B694D401ED918C
:10CC0000FC910488F589E02DC401199501E010E03C
:10CC100088C028966EAD7FAD2897CE0181960E9480
:10CC2000018D892B09F450C122961CAE1DAE1EAE9B
:10CC30001FAE229726961CAE1DAE1EAE1FAE2697C7
:10CC40008FAD8F708FAF40E053E0BE016F5D7F4FBF
:10CC5000CE01CE960E94862F00E020E033E040E235
:10CC600050E0B501CE01CE960E94F02BBC01C6016A
:10CC70000E94DF7408EC10E129C1EE2009F4F3C032
:10CC800046E050E070E060E0C8010E940873D801FF
:10CC90006D917C91CE0181960E94F235CE018196F4
:10CCA0000E94F91100E911E08823B9F189A58730C4
:10CCB00061F4CE0181960E94F44D61E0892B09F464
:10CCC00062E0CE0181960E94661722961CAE1DAED0
:10CCD0001EAE1FAE229726961CAE1DAE1EAE1FAE18
:10CCE00026978FAD8F708FAF40E053E0BE016F5D30
:10CCF0007F4FCE01CE960E94862F00E020E033E0E9
:10CD000040E250E0B501CE01CE960E94F02BBC016E
:10CD1000C6010E94DF7408EC10E1CE0181960E94EA
:10CD20002F12C801C159DF4F0FB6F894DEBF0FBEF6
:10CD3000CDBFDF91CF911F910F91FF90EF90DF90CA
:10CD4000CF90BF90AF909F908F907F906F905F90AB
:10CD50000895F801608171810E94A0877C01892B70
:10CD600009F040C104E911E0DCCFEE2009F47BC0FA
:10CD700049E050E070E060E0C8010E9408734AE0BA
:10CD8000B401C5010E94837541E050E067EC73E097
:10CD9000C8010E94CB734D815E8169817A81C8018F
:10CDA0000E94CB7360E779E085E799E00E94FD7609
:10CDB000B801CE0181960E943B75BE016F5D7F4F29
:10CDC00085E799E00E94EF7685E799E00E94067674
:10CDD000CE0181960E94057568E679E0CE018196C4
:10CDE0000E940D75F801848195812DA13EA18217C5
:10CDF0009307E1F4892BA1F1E080F18069A07AA08A
:10CE0000D7018D917D01882359F1082E000C990BD3
:10CE10000E9429C96C01F30181913F01082E000C89
:10CE2000990B0E9429C9C816D90651F3CE018196E3
:10CE30000E940575552041F021E048EC50E0B40116
:10CE400081E798E00E949F77D8018D919C910E9484
:10CE5000CD77009711F484E991E08C01C5013DC0C4
:10CE600055245394E3CF01E97ECFB1E0FB1270C0AB
:10CE70006DE879E0C5010E940D75B501C8010E94F9
:10CE80006B73582EC5010E940575552049F1EE209F
:10CE900051F346E050E070E060E0C8010E94087382
:10CEA0004AE0B401CE018A5B9F4F0E948375F8016E
:10CEB00060817181CE0181960E94F235CE0181960A
:10CEC0000E94F9118111A5CE00E911E0CE018196F1
:10CED0000E942F12CE018A5B9F4F0E94057521CFC1
:10CEE00066E779E0C5010E940D75B501C8010E9491
:10CEF0006B73F82EC5010E940575F11036CF6BE5F6
:10CF000079E0C5010E940D75B501C8010E946B73DF
:10CF1000182FC5010E94057500E0112309F401CF07
:10CF200080E00E94F18B63E379E084EC98E00E945A
:10CF3000FD7684EC98E00E9406766FE175E0C5010D
:10CF40000E944475C5010E94039DC5010E9405759C
:10CF500000E05DCE66E879E0C5010E940D75B5017F
:10CF6000C8010E946B73F82EC5010E940575F1106F
:10CF700084CE60E879E0C5010E940D75B501C80155
:10CF80000E946B73F82EC5010E940575FF2001F306
:10CF9000EE2009F468CF45E050E070E060E0C801A1
:10CFA0000E94087365ED74E0C8010E9486738823AF
:10CFB00039F0E0909D06F0909E06E114F10491F4A2
:10CFC0006FE175E0C8010E948673811107C08091EE
:10CFD0009D0690919E06009709F0BBCEE090B405A7
:10CFE000F090B50520E048EC50E2B40181E798E00C
:10CFF0000E949F77C4010E9406761C821B828DE7E7
:10D0000092E09A8389839E828D828FEF9FEF98872B
:10D010008F83B701C5010E949478EACDAF92BF9289
:10D02000CF92DF92EF92FF920F931F93CF93DF93F4
:10D03000CDB7DEB7C859D1090FB6F894DEBF0FBE21
:10D04000CDBF8E010F5B1F4FD8011D921C92FE01B8
:10D05000ED5BFF4F8EE1DF011D928A95E9F780912C
:10D06000A0089091A108892B09F485C10E94FD8830
:10D07000882309F480C182E70E94E8888091A00893
:10D080009091A108DC01ED91FC910088F189E02DDF
:10D0900060E270E019954FE150E0B8018091A0087E
:10D0A0009091A1080E9442897C018091A0089091F2
:10D0B000A108DC01ED91FC910488F589E02D19951A
:10D0C000E114F10409F457C1F801EE0DFF1D1082BF
:10D0D0008091AD081F928F938091AC081F928F931F
:10D0E0008091AB081F928F938091AA081F928F9313
:10D0F0008091A9081F928F938091A8081F928F9307
:10D1000087ED94E09F938F931F9280E48F93FE01AD
:10D1100031966F01FF93EF930E94ECC965E670E1D1
:10D1200084EC98E00E94FD76B80184EC98E00E94BF
:10D130009776B60184EC98E00E94977684EC98E0AC
:10D140000E9406767E01F1E6EF0EF11CD7011396E0
:10D150001C921E92129788EE93E0A0E0B0E0F701D7
:10D1600084839583A683B78384E084878DE293E0EC
:10D170009183808316861586108B0787128A118A01
:10D1800080E590E0948B838B178A64E97FE085E7E4
:10D1900099E00E94FD7662EA78E0CE0187589F4FC1
:10D1A0000E943B75BE0167587F4F85E799E00E945A
:10D1B000EF7685E799E00E940676CE0187589F4F6B
:10D1C0000E94057566E075E0CE0185579F4F0E946D
:10D1D000447566E075E0CE0187589F4F0E94447504
:10D1E000BE0167587F4FCE018D579F4F0E943B7500
:10D1F00062EA78E0CE018D579F4F0E94A174BE0174
:10D2000065577F4F0E94A174BC01CE018F569F4F7E
:10D210000E943B75CE018D579F4F0E940575CE0130
:10D2200087589F4F0E940575CE0185579F4F0E94DA
:10D23000057588E095E0CD57DF4F99838883C35803
:10D24000D040C957DF4F19821882C758D040C757FE
:10D25000DF4F19821882C958D040CF56DF4F8881DE
:10D260009981C159D040CB57DF4F99838883C558E6
:10D27000D0406FE570E185E799E00E94FD760E945D
:10D280004811AB01BC0185E799E00E942D8C85E730
:10D2900099E00E94067664E670E080E090E00E94EB
:10D2A000B69485E494E6D7011E969C938E931D97C1
:10D2B00063E070E78BEC9AE70E9480BB8C010FB6AD
:10D2C000F894DEBF0FBECDBF892BA1F183E090E0C3
:10D2D0000E943AB7D8011D969C938E931C97FC012F
:10D2E000F182E0821282C7010E94F51C882319F0A6
:10D2F000C7010E949A1DD70151966D917C9152975A
:10D300005396AD90BC906115710509F44BC0CE01E8
:10D3100087589F4F0E943377A501BE0167587F4F02
:10D32000C7010E94AC5B181619060CF487C1C8012E
:10D330000E94A47A66EF7FE085E799E00E94FD767F
:10D34000EE24EA94FE2CCE018F569F4F0E94057565
:10D35000C701C856DF4F0FB6F894DEBF0FBECDBF72
:10D36000DF91CF911F910F91FF90EF90DF90CF90C1
:10D37000BF90AF90089540E250E067E970E1C801C6
:10D380000E94ADBA69E770E184EC98E00E94FD76F6
:10D39000B80184EC98E00E94977684EC98E00E94B3
:10D3A000067696CEF70167857089A501C7010E94B0
:10D3B0004013B9CF8FEE9FE09F938F931F930F93EE
:10D3C0000E9407BCD70156961C921E925597D80111
:10D3D0001C96ED91FC91A080B1800F900F900F9062
:10D3E0000F9093E3C92ED12CD501ED91FC910084CF
:10D3F000F185E02DC501199541975CF4B1E0CB1A98
:10D40000D10839F064E170E080E090E00E94B694C9
:10D41000EBCF6E01E7E9CE0ED11CDF92CF928FE900
:10D420009FE09F938F931F930F930E9424BC0F90B4
:10D430000F900F900F900F900F900197D1F4D6019D
:10D440008D919C91F701968B858B6FE175E0CE01F4
:10D4500085579F4F0E94447580E0C12CFAE0CF129F
:10D4600070C08A3009F071C0CE0185579F4F0E946D
:10D470000575D7015596ED90FC90B8ECEB16F104CC
:10D4800009F0BAC063E570E184EC98E00E94FD7693
:10D4900064EF71E080E090E00E94B694ED961FAEDC
:10D4A0001EAEED97EF961FAE1EAEEF978FEF9FEF7C
:10D4B000C158DF4F99838883CF57D04087E692E0E9
:10D4C000EB969FAF8EAFEB97CF57DF4F1983088353
:10D4D000C158D040F8948091B4059091B505892B3E
:10D4E00011F00E946D5ACE0187589F4F0E940491FF
:10D4F0009093B5058093B4057894C8010E94A47AEE
:10D500008091B4059091B505892B09F063C06FE156
:10D5100075E0CE0185579F4F0E944475CE01855717
:10D520009F4F0E94039DCE0185579F4F0E94057516
:10D530006CE370E18EEC98E00E94FD76F12CE12C1A
:10D5400002CF9DE0C91201C0C82EC8010E94CBBB0A
:10D55000D82ED7011D96AD90BC90A114B10499F1BD
:10D56000BAE08B1779F0EDE08E1761F0FFEF8F17BF
:10D5700049F0682FCE0185579F4F0E94F7738C2D7D
:10D58000CD2C6CCFC157DF4F88819981CF58D040C7
:10D59000892B91F0BE0165577F4FCE0187589F4F71
:10D5A0000E943B75CE0187589F4FF5011995CE011A
:10D5B00087589F4F0E9405756FE175E0CE01855732
:10D5C0009F4F0E94D574FFEFDF12D9CFC8010E9490
:10D5D000A47A4ACF0E94665C80919206882329F043
:10D5E0000E945C8B67FF0E94E11665E370E184ECAA
:10D5F00098E00E94FD76A7CEE0E3EE16E1E0FE069D
:10D6000051F461E270E184EC98E00E94FD76C8017B
:10D610000E94A47A98CE69E070E18EEC98E00E94B6
:10D62000FD76C8010E94A47AB7018EEC98E00E94B2
:10D63000378C8EEC98E00E94067685CED7011F9637
:10D64000BC901F975096AC90DF92CF9282EF9FE0F4
:10D650009F938F931F930F930E9407BCDF92CF92EB
:10D660008DEE9FE09F938F931F930F930E9407BCB3
:10D67000D8011C96ED91FC9181E08283DF92CF92DC
:10D680008AEE9FE09F938F931F930F930E9407BC96
:10D69000D8011C96ED91FC911282AF92BF9284EB5F
:10D6A0009FE09F938F931F930F930E9407BC0FB629
:10D6B000F894DEBF0FBECDBFB12C8BEAC82E8FE031
:10D6C000D82E8B2D94E08902F0011124A3E8B0E05C
:10D6D000AC0FBD1FEA0FFB1F80819181009709F4F9
:10D6E00069CE2281338121153105C1F33F932F93F8
:10D6F0009F938F93DF92CF921F930F930E9407BC4B
:10D70000B3940FB6F894DEBF0FBECDBFDACF0F9340
:10D710001F93CF93DF93EB0102970CF485C00A812E
:10D720001B8166E87FE0C8010E9458BA892B51F43A
:10D7300081E00E94F18B88EC90E0DF91CF911F9106
:10D740000F91089562E87FE0C8010E9458BA892BC2
:10D7500011F480E0EECF62E67FE084EC98E00E9476
:10D76000FD760E945C8B63FB662760F981E0682789
:10D7700070E084EC98E00E94378C84EC98E00E9482
:10D7800006768091A0089091A108892BE9F10A8181
:10D790001B810E94FD888823B9F1F80101900020C7
:10D7A000E9F73197E01BF10BB09770F582E70E9423
:10D7B000E8888091A0089091A108DC01ED91FC918E
:10D7C0000088F189E02D60E270E01995B801809140
:10D7D000A0089091A1080E9497768091A00890914E
:10D7E000A108DC01ED91FC910190F081E02D60E059
:10D7F00019958091A0089091A108DC01ED91FC9110
:10D800000488F589E02D19956A817B8184EC98E084
:10D810000E9497766BE57FE084EC98E00E94FD76AD
:10D8200084EC98E00E94067680919B0690919C067D
:10D8300002977CF10E940E68883C910539F424E03F
:10D8400030E030939C0620939B0677CF8F3F98075C
:10D85000C9F460E47FE085E799E00E94FD7685E702
:10D8600099E00E9406761092900683E090E09093F3
:10D870009C0680939B0683E998E00E949A1D89ECA0
:10D8800090E05BCF209192062111D9CF2FE030E0BC
:10D89000D8CF63E37FE08EEC98E00E94FD768EECBB
:10D8A00098E00E94067684EF91E047CF0895FC014E
:10D8B000248135816217730748F480819181009734
:10D8C00029F0860F971FFC018081089580E008955C
:10D8D0000895AF92BF92CF92DF92EF92FF920F9393
:10D8E0001F93CF93DF936C017B018B01040F151FF6
:10D8F000EB015E01AE18BF08C017D10759F069915E
:10D90000D601ED91FC910190F081E02DC6011995B1
:10D91000892B79F7C501DF91CF911F910F91FF906E
:10D92000EF90DF90CF90BF90AF900895FC01538DA2
:10D93000448D252F30E0842F90E0821B930B5417E9
:10D9400010F0CF96089501970895FC01918D828D76
:10D95000981761F0A28DAE0FBF2FB11D5D968C910F
:10D96000928D9F5F9F73928F90E008958FEF9FEF4E
:10D970000895FC01918D828D981731F0828DE80F0A
:10D98000F11D858D90E008958FEF9FEF0895FC01C4
:10D99000918D228D892F90E0805C9F4F821B910991
:10D9A0008F739927089588ED98E00E94C76C21E055
:10D9B000892B09F420E0822F0895FC01A48DA80F83
:10D9C000B92FB11DA35ABF4F2C91848D90E00196C1
:10D9D0008F739927848FA689B7892C93A089B189E1
:10D9E0008C91837080648C93938D848D981306C082
:10D9F0000288F389E02D80818F7D80830895EF92E6
:10DA0000FF920F931F93CF93DF93EC0181E0888FF8
:10DA10009B8D8C8D98131AC0E889F989808185FFC8
:10DA200015C09FB7F894EE89FF896083E889F9896A
:10DA300080818370806480839FBF81E090E0DF916C
:10DA4000CF911F910F91FF90EF900895F62E0B8DBF
:10DA500010E00F5F1F4F0F731127E02E8C8D8E117A
:10DA60000CC00FB607FCFACFE889F989808185FFE1
:10DA7000F5CFCE010E94DD6CF1CFEB8DEC0FFD2FC9
:10DA8000F11DE35AFF4FF0829FB7F8940B8FEA899C
:10DA9000FB8980818062CFCFCF93DF93EC01888DAB
:10DAA0008823B9F0AA89BB89E889F9898C9185FD19
:10DAB00003C0808186FD0DC00FB607FCF7CF8C91A7
:10DAC00085FFF2CF808185FFEDCFCE010E94DD6C16
:10DAD000E9CFDF91CF91089580E090E0892B29F084
:10DAE0000E94D36C81110E94000080E090E0892B9D
:10DAF00049F080E090E0892B29F00E94000081111C
:10DB00000E94000080E090E0892B49F080E090E0E6
:10DB1000892B29F00E94000081110E94000080E002
:10DB200090E0892B49F080E090E0892B29F00E9459
:10DB3000000081110C94000008950F931F93FC01C5
:10DB40006285738584859585028113812481358161
:10DB5000601B710B820B930B068517852089318919
:10DB6000601B710B820B930B1F910F910895DC01C9
:10DB7000ED91FC910190F081E02D19948FEF9FEFD2
:10DB80000895FC0162897389848995890895EF92CB
:10DB90000F931F93CF93DF93FC01248D222341F039
:10DBA000213051F1DF91CF911F910F91EF900895A6
:10DBB000228933894489558986899789A08DB18DB9
:10DBC000821B930BA40BB50B892F9A2FAB2FBB276E
:10DBD0008C010F5F1F4F6281738184819581CFB764
:10DBE000F894DCB7E1E0ECBFEE24E394E2E0FEEF72
:10DBF0001995DCBFCFBFD6CFF0E0E0E0DF91CF9149
:10DC00001F910F91EF901994FC01138E128E411108
:10DC10000CC082899389A489B589868B978BA08F44
:10DC2000B18F148E81E090E0089590E080E0089537
:10DC3000CF92DF92EF92FF92CF93DF93DC01CB0183
:10DC4000642FCFB7F8946D01EE24FF24CBBEDCB770
:10DC500041E04CBFA901E1E0FEEF1995DCBFCFBF69
:10DC6000DF91CF91FF90EF90DF90CF900895CF9309
:10DC7000DF93FC01248D211110C0EC01828D938D66
:10DC8000892B49F066897789808D918D30E020E07D
:10DC900045E00E94186E1B8E1A8EDF91CF91089579
:10DCA0001F93CF93DF93FC01248D211145C0162FC4
:10DCB000EC01828D938D892B49F466897789808D5B
:10DCC000918D30E020E043E00E94186E4A8D5B8D1C
:10DCD000CA0181709927FE01E80FF91F158F892B62
:10DCE00069F02D8D3E8D6E897F89888D998D640FA9
:10DCF000751F811D911D41E00E94186E8A8D9B8DBC
:10DD000001969B8F8A8F81159140B1F46E897F892E
:10DD1000888D998D30E020E045E00E94186E1B8EC2
:10DD20001A8E8E899F89A88DB98D9F5FAF4FBF4F87
:10DD30008E8B9F8BA88FB98F81E090E0DF91CF9180
:10DD40001F910895DC01ED91FC910280F381E02D9B
:10DD500040E01994FB0124813581428153812417CD
:10DD6000350750F4A081B181A20FB31F8C93848139
:10DD7000958101969583848380E00895CF93DF9306
:10DD8000EC01E881F9810284F385E02DCE0119953B
:10DD90000196B9F7DF91CF910895CF92DF92EF927C
:10DDA000FF920F931F93CF93DF937C016A018B0146
:10DDB000D0E0C0E0CC15DD0581F0D701ED91FC91FC
:10DDC0000284F385E02DC70119958F3F980729F04C
:10DDD000F80181938F012196EDCFCE01DF91CF9194
:10DDE0001F910F91FF90EF90DF90CF900895CF9308
:10DDF000C62FDC01ED91FC910088F189E02D199589
:10DE0000DC01ED91FC910190F081E02D6C2FCF9120
:10DE10001994062E000C770BFC0177836683089516
:10DE2000CF93DF93EC018E819F81019611F5E881FC
:10DE3000F9810088F189E02DCE011995DC01ED9181
:10DE4000FC910084F185E02D1995892BB1F0E881D2
:10DE5000F9810284F385E02DCE0119958132910577
:10DE600034F3E881F9810684F785E02D682FCE012F
:10DE7000199581E0DF91CF91089580E0FBCFCF939A
:10DE8000DF931F92CDB7DEB76983DC01ED91FC9182
:10DE90000280F381E02D41E050E0BE016F5F7F4FD3
:10DEA00019950F90DF91CF910895EF92FF920F9304
:10DEB0001F93CF93DF93EC018B017A010E94FB96B5
:10DEC000688B798B8A8B9B8B8C819D81DC01ED919A
:10DED000FC910280F381E02DA701B801DF91CF9181
:10DEE0001F910F91FF90EF9019941F93CF93DF93A1
:10DEF000EC01162F0E94FB96688B798B8A8B9B8B8B
:10DF00008C819D81DC01ED91FC910190F081E02DEF
:10DF1000612FDF91CF911F911994CF92DF92EF92F1
:10DF2000FF92CF93DF93EC018E819F818F3F980703
:10DF300059F02FEF3FEF3F832E83DF91CF91FF907A
:10DF4000EF90DF90CF9008950E94FB966B017C01CB
:10DF5000A4EFCA0EA1E0DA1EE11CF11CE881F981F0
:10DF60000088F189E02DCE011995DC01ED91FC913D
:10DF70000084F185E02D1995892B39F40E94FB96D8
:10DF80006C157D058E059F0548F3E881F9810088B1
:10DF9000F189E02DCE011995DC01ED91FC9102840F
:10DFA000F385E02DDF91CF91FF90EF90DF90CF9040
:10DFB00019940E9424C90F931F93CF93DF93EC0110
:10DFC00088819981009759F02A813B81261737076C
:10DFD00030F081E0DF91CF911F910F9108958B0177
:10DFE0006F5F7F4F0E9443C8009759F099838883E1
:10DFF0001B830A832C813D81232B59F7FC0110825E
:10E00000E8CF80E0E7CFEF92FF920F931F93CF937B
:10E01000DF93009751F4CFEFDFEFCE01DF91CF9187
:10E020001F910F91FF90EF900895DC011C96ED90E9
:10E03000FC90F70100811181D801ED91FC910688D7
:10E04000F789E02DC8011995882329F3D801ED91AE
:10E05000FC910084F185E02DC8011995D801ED915E
:10E06000FC91892B61F30284F385E02DC801199599
:10E07000EC01019681F2F8018789882329F06C2F41
:10E0800088ED98E00E94308CD70112968C918823FD
:10E0900021F2C532D10509F6D801ED91FC91008439
:10E0A000F185E02DC801199502975CF0D801ED913A
:10E0B000FC910688F789E02DC80119958111ECCFF4
:10E0C000AACFD1E0C0E0D801ED91FC910284F385A4
:10E0D000E02DC80119958F3F980709F49CCF9C014A
:10E0E000215431092A31310570F48D2F8295807FBA
:10E0F000829FC00D1124D11104C00C2E000CDD0B29
:10E100008CCFD0E0E0CF9C01215631092A31310576
:10E1100060F3C0978A30910570F79D2F9295907F9C
:10E12000989FC00D1124E7CFCF92DF92EF92FF921C
:10E130000F931F93CF93DF936C018B0186E090E0E8
:10E140000E943AB7EC019093210780932007F601D3
:10E1500001900020E9F7CF018C199D090E943AB780
:10E160007C01B6010E94ADC9F60101900020E9F7DB
:10E170003197EC19FD09EE0DFF1D1082F982E8823E
:10E180001B830A8380912207909123079D838C83B0
:10E19000D0932307C0932207DF91CF911F910F9156
:10E1A000FF90EF90DF90CF900895FC0186819781DA
:10E1B0008F3F980729F02FEF3FEF3783268308958D
:10E1C000808591850C94CBBB1F93CF93DF93182F41
:10E1D00066E270E00E94B51CC82F67E270E0812FF4
:10E1E0000E94B51C9C2FDF91CF911F910895CF9372
:10E1F000FC01C08D80E590E00E94229160E270E019
:10E200008C2F0E94819162E070E08C2F0E94B51CDF
:10E2100084FD1AC062E070E08C2F0E94B51C83FF61
:10E220000CC048E162E070E08C2F0E94AB1C0E94A1
:10E230002D1D90E080E0CF9108950E942D1D80E576
:10E2400090E00E942291DFCF40E162E070E08C2FED
:10E250000E94AB1C0E942D1D81E090E0ECCFFF924C
:10E260000F931F93CF93DF93EB01FC01178A168A5C
:10E270002A81211109C02B81211106C02C81211175
:10E2800003C02D812223F1F041155105D9F08A01F7
:10E29000FC01F08C80E590E00E942291BE016E5F4F
:10E2A0007F4F8F2D0E94E41CB8018F2D0E94D31C3C
:10E2B0000E942D1D81E090E0DF91CF911F910F9181
:10E2C000FF90089590E080E0F7CFAF92BF92CF9299
:10E2D000DF92FF920F931F93CF93DF938C015B012B
:10E2E000EA01FC01C688D788F08C80E590E00E94A6
:10E2F00022918F2D0E9439928C179D0720F48F2D2B
:10E300000E943992EC019E01A501B6018F2D0E9459
:10E31000D9910E942D1DF801868997898C0F9D1F28
:10E32000978B868BCE01DF91CF911F910F91FF903C
:10E33000DF90CF90BF90AF9008957F928F929F9281
:10E34000AF92BF92CF92DF92EF92FF920F931F9303
:10E35000CF93DF93CDB7DEB7A6970FB6F894DEBFA5
:10E360000FBECDBF8C01762E942E852E20E2A22EDC
:10E37000CE0101967C01DC01EA2D1D92EA95E9F7B8
:10E380006801F3E4CF0ED11C85EA93E09AA389A338
:10E390008FEF8BA38CA38DA38EA343E450E0BE012B
:10E3A0006F5D7F4FC6010E942F71019609F4BFC0B7
:10E3B00081E089838A8386E0B82EBB821C82D801E3
:10E3C00014966D917D918D919C9117970E944BC5EC
:10E3D0006D837E838F83988789869A8680E890E014
:10E3E0009C878B874CE150E0B701C6010E946571A4
:10E3F000FE0137968AE1DF011D928A95E9F748010F
:10E40000B8E08B0E911CF401D70101900D92BA94E3
:10E41000E1F740E150E0B701C6010E946571F701E4
:10E420001192AA94E9F796E0A92EB12C40E250E0AF
:10E43000B701C6010E946571F1E0AF1AB108B1F7EA
:10E4400083E6898392E89A8393E59B838C8385E3B3
:10E450008D8381E08E837F829DE3988797E0998703
:10E460008A8786E0F401DE011B9601900D928A9561
:10E47000E1F78CE0898B8A8B66E175E0CE014396EB
:10E480000E94ADC9D8011B966C91CE0149960E949D
:10E490005592F8016485CE014B960E945592D801A1
:10E4A0001D966C91CE014D960E9455924EE150E022
:10E4B000B701C6010E946571B3E07B121EC082E302
:10E4C000898384E08A83F80196859B8397859C8362
:10E4D00090899D8391899E8396E39F838887828D0F
:10E4E0008987838D8A87848D8B87858D8C874CE087
:10E4F00050E0B701C6010E94657187E3898386E019
:10E500008A8391E09B8393E09C838D838FE08E834D
:10E510008AE38F838BE388878FEF898749E050E018
:10E52000B701C6010E946571C6010E94F770A696E8
:10E530000FB6F894DEBF0FBECDBFDF91CF911F9114
:10E540000F91FF90EF90DF90CF90BF90AF909F9092
:10E550008F907F900895AF92BF92CF92DF92EF920B
:10E56000FF920F931F93CF93DF93DC01CD90DC904C
:10E570001197C114D10439F01496CD91DC918C011E
:10E580007601209761F4DF91CF911F910F91FF9059
:10E59000EF90DF90CF90BF90AF9008957501570135
:10E5A000BFEFAB1ABB0AF7018081082E000C990B54
:10E5B0000E944FBA892B91F72197CC0DDD1D8881E0
:10E5C000082E000C990B0E944FBA892B29F0CE150A
:10E5D000DF0510F02197F3CFAE014F5F5F4F4E196B
:10E5E0005F09D80115965C934E931497CE14DF04FF
:10E5F00020F4B701C6010E9460C9D801ED91FC91D9
:10E60000119714968D919C91E80FF91F1082BBCF42
:10E61000CF93DF93DC011496ED91FC916E177F0789
:10E6200028F54115510511F19F01261B370B4217A3
:10E63000530708F49A01DB01EC0188819981E21B00
:10E64000F30BFD83EC83AF01461B570B260F371FDF
:10E65000BC01620F731F8A0F9B1F0E94D2C9E88101
:10E66000F9818C819D81E80FF91F1082DF91CF9194
:10E670000895DF92EF92FF920F931F93CF93DF9352
:10E68000FC01E480F580E114F10451F48FEF9FEF79
:10E69000DF91CF911F910F91FF90EF90DF90089540
:10E6A000EC010190F081E02DEE0DFF1DD080108275
:10E6B00008811981062E000C770BC8010E94E1C960
:10E6C0000E0D1F1DF801D082009701F328813981BA
:10E6D000821B930BDDCFFB0144815581FC0124811A
:10E6E00035812417350778F080819181009759F0A2
:10E6F000FB01608171816115710529F00E94C4C917
:10E7000021E0892B09F020E0822F0895FC0124816B
:10E710003581232B39F421E0FB018081882349F0E6
:10E7200020E007C0808191810E94A4C921E0892B4B
:10E73000B9F7822F0895FC0124813581FB014481C2
:10E74000558124173507E1F4FC0180819181FB019B
:10E75000608171810097D1F061157105A1F4232BBF
:10E76000C1F0FC01808190E008C0232B91F0FB01F7
:10E77000808190E091958195910921E0892B09F0A4
:10E7800020E0822F08950E94A4C9F7CF611571057A
:10E7900061F721E0F6CFEF92FF920F931F93CF9393
:10E7A000DF936115710541F480E0DF91CF911F91F6
:10E7B0000F91FF90EF90089541155105B1F07B0145
:10E7C000EC010C811D81040F151FB8010E94DB6F45
:10E7D000882351F3288139818C819D81B701820F73
:10E7E000931F0E94ADC91D830C8381E0DECFCF93C0
:10E7F000DF931F921F92CDB7DEB769831A8241E083
:10E8000050E0BE016F5F7F4F0E94CB730F900F905F
:10E81000DF91CF9108950F931F93CF93DF938C01D6
:10E82000EB01FC01808191810097E1F068817981A1
:10E8300061157105A9F0428153812C813D814217F8
:10E84000530770F00E94ADC98C819D81F8019583BA
:10E8500084831D821C82DF91CF911F910F910895B7
:10E860000E94D6B788819981F801918380838A813B
:10E870009B81938382838C819D819583848319827C
:10E8800018821B821A82E5CFCF93DF93EC01888137
:10E890009981009711F00E94D6B7198218821D82C3
:10E8A0001C821B821A82DF91CF910895EF92FF9212
:10E8B0000F931F93CF93DF9300D01F92CDB7DEB796
:10E8C0007C01862F4AE08E010F5F1F4FB80190E058
:10E8D0000E94F2BAF80101900020E9F73197AF01E8
:10E8E000401B510BB801C7010E94CB73811103C0BB
:10E8F000C7010E944474C7010F900F900F900F90B2
:10E90000DF91CF911F910F91FF90EF900895CF93DA
:10E91000DF93EC016115710539F4CE010E94447456
:10E92000CE01DF91CF910895FB0101900020E9F71E
:10E930003197AF01461B570B0E94CB73882369F3B5
:10E94000EFCFCF93DF93EC01FB01448155816081D0
:10E9500071810E94CB73811103C0CE010E94447467
:10E96000CE01DF91CF910895EF92FF920F931F9305
:10E97000CF93DF93EC017B018A01BA010E94DB6F28
:10E9800081110BC0CE010E944474CE01DF91CF9162
:10E990001F910F91FF90EF9008951D830C83B70195
:10E9A000888199810E94ADC9F0CFFB0101900020C0
:10E9B000E9F73197AF01461B570B0C94B474CF9312
:10E9C000DF93EC016115710531F00E94D574CE0121
:10E9D000DF91CF9108950E944474F9CFCF93DF93D4
:10E9E000EC01FB018617970749F060817181611581
:10E9F000710541F0448155810E94B474CE01DF91CC
:10EA0000CF9108950E944474F9CFFC0180819181D7
:10EA1000009711F00C94D6B70895EF92FF920F93E0
:10EA20001F93CF93DF93EC018B01198218821B8215
:10EA30001A821D821C82CB010E9486BA7C01BC0115
:10EA4000CE010E94DB6F811109C0CE01DF91CF9111
:10EA50001F910F91FF90EF900C944474FD82EC8213
:10EA6000B80188819981DF91CF911F910F91FF901B
:10EA7000EF900C947FBAFC011182108213821282F3
:10EA8000158214820C94EE74FC01118210821382A0
:10EA9000128215821482FB0101900020E9F7319760
:10EAA000AF01461B570B0C94B4740F931F93CF9375
:10EAB000DF93EC010E94FB96688779878A879B87A2
:10EAC000E881F9810284F385E02DCE01199597FF45
:10EAD00015C00E94FB96088519852A853B85601B19
:10EAE000710B820B930B0C811D812E813F8160176E
:10EAF00071078207930720F38FEF9FEFDF91CF918C
:10EB00001F910F910895EF92FF920F931F93CF9350
:10EB1000DF93EC017B01042F6FE175E00E944475E7
:10EB2000C7010E945575002E000C110B97FD0BC0FC
:10EB30000817190741F0682FCE010E94F773C7012B
:10EB40000E945575F3CFCE01DF91CF911F910F91A8
:10EB5000FF90EF900895FB0101900020E9F73197B5
:10EB6000AF01461B570BDC01ED91FC910280F38154
:10EB7000E02D19948F929F92AF92BF92EF92FF92E5
:10EB80000F931F93CF93DF93CDB7DEB7A1970FB647
:10EB9000F894DEBF0FBECDBF7C01FA01CB0119A2F4
:10EBA000223008F42AE08E010F5D1F4F822E912C37
:10EBB000B12CA12CBF01A50194010E94B8C4F90198
:10EBC000CA016A300CF5605DD8016E938D01232B6C
:10EBD000242B252B79F790E080E0109721F0BD01E0
:10EBE000C7010E94AB75A1960FB6F894DEBF0FBEA9
:10EBF000CDBFDF91CF911F910F91FF90EF90BF900C
:10EC0000AF909F908F900895695CDECF6DE175E0C5
:10EC10000C94AB75DC01ED91FC910190F081E02D3D
:10EC20001994CF92DF92EF92FF920F931F93CF939D
:10EC3000DF932115310581F4DC01ED91FC91019008
:10EC4000F081E02D642FDF91CF911F910F91FF9004
:10EC5000EF90DF90CF9019942A30310501F52AE02A
:10EC600077FF1DC06A017B01EC016DE20E940A760C
:10EC70008C0144275527BA014C195D096E097F099B
:10EC80002AE0CE010E94BA75800F911FDF91CF91CB
:10EC90001F910F91FF90EF90DF90CF900895DF913B
:10ECA000CF911F910F91FF90EF90DF90CF900C9438
:10ECB000BA758F929F92AF92BF92CF92DF92EF92EE
:10ECC000FF920F931F93CF93DF937C018B014C0135
:10ECD00082E0880E911C5701E5E0AE0EB11CD0E039
:10ECE000C0E0F40161914F01C8010E94308C6C01B9
:10ECF0006EE2C8010E940A768C0D9D1DC80FD91FB7
:10ED00008A149B0471F7F7016581C8010E94308C59
:10ED10008C0F9D1FDF91CF911F910F91FF90EF906E
:10ED2000DF90CF90BF90AF909F908F900895611526
:10ED3000710511F00C94AB7590E080E008950F938D
:10ED40001F93CF93DF93EC018B0166E075E00E9487
:10ED5000977601151105C1F1F80161918F016623C4
:10ED600099F1603240F0623231F06C3521F0CE0121
:10ED70000E940A76F1CF6CE5CE010E940A76F80176
:10ED8000319780818C30D1F044F48930D9F08A30C9
:10ED9000B9F0883009F762E6EACF823259F024F4FC
:10EDA00062E78D3021F3D8CF8F3231F06CE58C35AE
:10EDB000F1F2D2CF62E2DBCF6FE2D9CF66E6D7CFF6
:10EDC0006EE6D5CF64E7D3CF62E2CE010E940A7629
:10EDD00090E080E0DF91CF911F910F910895DB01CA
:10EDE00014964D915C9115976D917C91DC01ED919C
:10EDF000FC910280F381E02D1994EF92FF920F9322
:10EE00001F93CF93DF938C017B01D0E0C0E0F7012B
:10EE1000EC0FFD1F6491662361F0D801ED91FC9128
:10EE20000190F081E02DC8011995892B11F02196F0
:10EE3000EECFCE01DF91CF911F910F91FF90EF9018
:10EE400008950F931F93CF93DF93EC010E94FD76FB
:10EE50008C01CE010E940676800F911FDF91CF9129
:10EE60001F910F910895DC0185EA93E08D939D93A6
:10EE700084E0FB0101900D928A95E1F708951F92BD
:10EE80000F920FB60F9211240BB60F922F933F9350
:10EE90004F935F936F937F938F939F93AF93BF93A2
:10EEA000EF93FF9388ED98E00E94DD6CFF91EF9166
:10EEB000BF91AF919F918F917F916F915F914F9192
:10EEC0003F912F910F900BBE0F900FBE0F901F9090
:10EED00018951F920F920FB60F9211240BB60F9236
:10EEE0002F938F939F93EF93FF93E091E808F09116
:10EEF000E9088081E091EE08F091EF0882FD1DC0E5
:10EF000090818091F1088F5F8F732091F2088217B2
:10EF100041F0E091F108F0E0E852F74F958F8093CF
:10EF2000F108FF91EF919F918F912F910F900BBE60
:10EF30000F900FBE0F901F9018958081F2CFDF9237
:10EF4000EF92FF920F931F93CF93DF9300D000D0E7
:10EF5000CDB7DEB78B017A01D22E6FE175E0CE011D
:10EF600001960E9444759E012F5F3F4F4D2DB701C2
:10EF7000C8010E94189ECE0101960E940575269632
:10EF80000FB6F894DEBF0FBECDBFDF91CF911F91BA
:10EF90000F91FF90EF90DF900895CF92DF92EF9264
:10EFA000FF920F931F93CF93DF93CDB7DEB7EC970C
:10EFB0000FB6F894DEBF0FBECDBFDC012C9122232B
:10EFC00009F469C067EC73E00E94BCBA9A83898334
:10EFD0007E01B3E0EB0EF11C01E010E0D02EC12E5B
:10EFE00067EC73E090E080E00E94BCBAF701819387
:10EFF00091937F010E31110521F00F5F1F4F892B77
:10F0000069F70091200710912107E980FA80011526
:10F01000110589F1D8016D917C91C7010E94A4C9A5
:10F02000892B29F5D8011296ED91FC91BE016F5FF5
:10F030007F4F8D2D9C2D19958C0188ED98E00E94B5
:10F0400006766FEC75E188ED98E00E94FD76C801C8
:10F05000EC960FB6F894DEBF0FBECDBFDF91CF9117
:10F060001F910F91FF90EF90DF90CF900895F801DE
:10F0700004811581CCCF63ED75E188ED98E00E94A5
:10F08000217788ED98E00E9406766FEC75E188EDB7
:10F0900098E00E94FD7610E000E0D9CFCF9388ED94
:10F0A00098E00E94C76C892BE9F188ED98E00E94F6
:10F0B000A56CC82F8A3089F08D3079F0883001F541
:10F0C00068E088ED98E00E940A7680912407882302
:10F0D00031F3815080932407E2CFE0912407F0E0E0
:10F0E000EC51F94F10826DE175E088ED98E00E94D7
:10F0F000977684EE96E00E94CD7710922407CFCFCA
:10F10000682F88ED98E00E940A76E0912407EB339F
:10F1100030F681E08E0F80932407F0E0EC51F94F38
:10F12000C083BDCFCF9108958F929F92AF92BF922F
:10F13000CF92DF92EF92FF920F931F93CF93DF93C3
:10F140006115710509F496C0DB011896EC911897CA
:10F15000E295E07FE595E595E595E595E73008F0E2
:10F1600089C0EC010E2E000CFF0B8827E554F748F0
:10F170008F4F0C9443C5C278D378DC78F3783D790F
:10F180004F79887960E275E0CE01DF91CF911F91D0
:10F190000F91FF90EF90DF90CF90BF90AF909F9036
:10F1A0008F900C94AB7519968C916AE275E0882368
:10F1B00059F365E275E0E8CF19964D915D916D9137
:10F1C0007C911C972AE030E0CE01DF91CF911F9116
:10F1D0000F91FF90EF90DF90CF90BF90AF909F90F6
:10F1E0008F900C9411761996CD90DD90ED90FC9057
:10F1F0001C9720E030E0A901C701B6010E946EC350
:10F2000087FF09C06CEB73E0CE010E949776F7FA96
:10F21000F094F7F8F094C701B6010E9447C64B017D
:10F220005C01BC01A401CE010E942D8C65ED74E04F
:10F23000CE010E949776C501B4010E9473C39B0161
:10F24000AC01C701B6010E9461C52DEC3CEC4CE459
:10F250005DE30E9462C520E030E040E251E40E949C
:10F26000D4C30E9447C6AB0170E060E02AE0CE0143
:10F270000E94BA7590E080E01DC019966D917C9156
:10F28000CE01DF91CF911F910F91FF90EF90DF9012
:10F29000CF90BF90AF909F908F900C949F761696D2
:10F2A0000D911C916BE5CE010E940A76019679F4CE
:10F2B0008FEF9FEFDF91CF911F910F91FF90EF9014
:10F2C000DF90CF90BF90AF909F908F9008950115E1
:10F2D000110579F0B801CE010E949478019641F3AE
:10F2E000D80112960D911C910115110511F06CE2D7
:10F2F000DACF6DE5CE010E940A7621E030E001967A
:10F3000011F030E020E088279927821B930BD2CFA1
:10F3100016960D911C916BE7CE010E940A7601961C
:10F3200039F20115110529F1D8016D917C91CE01B9
:10F330000E949F76019609F4BBCF6AE3CE010E943A
:10F340000A76019609F4B4CFB801CE010E949478F0
:10F35000019609F4ADCFD80112960D911C910115BB
:10F36000110539F06CE2CE010E940A760196C9F6C9
:10F370009FCF6DE7BFCFCF93DF93EC01E881F98199
:10F380000284F385E02DCE0119958F3F980769F02F
:10F39000E881F981813291059CF30684F785E02D9F
:10F3A000682FCE01199590E080E0DF91CF9108950C
:10F3B000CF92DF92EF92FF920F931F93CF93DF9341
:10F3C0007C016B01DC01ED91FC910284F385E02D61
:10F3D0001995829761F0CFEFDFEFCE01DF91CF91EA
:10F3E0001F910F91FF90EF90DF90CF900895F6015D
:10F3F0008085807F8460808786E090E00E943AB7B5
:10F400008C01009741F3E4EAF6E0DC01ED93FC9314
:10F4100080E4DF011D928A95E9F780E490E0F8012D
:10F420009383828315821482D701ED91FC9102842B
:10F43000F385E02DC7011995EC010196C9F0C232A0
:10F44000D10509F44DC0C032D1050CF449C0B80152
:10F450008C2FCC35D10549F5D701ED91FC91028473
:10F46000F385E02DC7011995EC018F3F980721F432
:10F47000C8010E94D6B7B1CF8236910541F15CF444
:10F480008F32910509F18C359105D9F0829761F69B
:10F49000B80182E20AC08E369105E1F04CF4B80161
:10F4A0008CE0C636D10509F0BFCF0E94AA6EBCCF52
:10F4B0008237910591F0B80189E0C437D105A9F3ED
:10F4C000B3CFB8018CE5F1CFB8018FE2EECFB80130
:10F4D00088E0EBCFB8018AE0E8CFB8018DE0E5CF56
:10F4E000F80184819581009749F00190F081E02D29
:10F4F000E80FF91F31978081882321F0B80180E05F
:10F500000E94AA6ED80114968D919C910E943AB7E0
:10F51000EC01009739F064EA76E00E94ADC9C801B9
:10F520000E94D6B7F601D287C187D0E0C0E055CFA0
:10F530008DE090E00E943AB7009729F02DE0FC01A1
:10F5400011922A95E9F708950F931F93CF93DF93B4
:10F550000097E1F0EC010C851D850115110579F08E
:10F56000D8018D919C91009739F0DC01ED91FC91CF
:10F570000488F589E02D1995C8010E94D6B7CE01FF
:10F58000DF91CF911F910F910C9456BBDF91CF91DA
:10F590001F910F910895AF92BF92CF92DF92EF9299
:10F5A000FF920F931F93CF93DF9300D01F92CDB79D
:10F5B000DEB761157105B1F06B01182FDB011C96E8
:10F5C000AD90BC90F501E080F180D701ED91FC9108
:10F5D0000688F789E02DC7011995811106C0C6017B
:10F5E0000E94A47A8FEF9FEF13C0F50192819111D1
:10F5F00024C0D701ED91FC910190F081E02D612FA5
:10F60000C7011995F7018789811111C090E080E049
:10F610000F900F900F900F90DF91CF911F910F914E
:10F62000FF90EF90DF90CF90BF90AF900895612F43
:10F6300088ED98E00E940A76E9CF812F8F7D815472
:10F640008A31B8F280ED810F8A3098F283ED810F14
:10F65000823078F21F3569F21E3759F21132B1F05B
:10F6600086EC810F823090F08AED810F873070F048
:10F670001D3361F0812F8F7E8F3241F08DED810F30
:10F68000823020F01B3511F01D3511F491FFB1CF00
:10F6900019821A821B821C82812F012E000C990B69
:10F6A0009F931F9380E395E09F938F938E010F5F4D
:10F6B0001F4F1F930F930E9429CA6E01F4E0CF0ED3
:10F6C000D11C0F900F900F900F900F900F90D801BA
:10F6D0006D918D01D701ED91FC910190F081E02DAC
:10F6E000C7011995F7018789882339F0F801319707
:10F6F000608188ED98E00E940A760C151D0539F7A7
:10F7000085CF2C9A08952C9808951F93CF93DF935B
:10F71000182F60E270E00E94B51CC82F61E270E013
:10F72000812F0E94B51C9C2FDF91CF911F910895CE
:10F730008EBD00000DB407FEFDCF8EB50895CF92AB
:10F74000DF92EF92FF920F931F93CF93DF93EC0121
:10F750007A018B016C01C40ED51ECC15DD05A9F014
:10F760000E94837B8FE00E94987B8D2F0E94987B64
:10F770008C2F0E94987B219680E00E94987BF80154
:10F7800081938F010E94817BE8CFC701DF91CF91E8
:10F790001F910F91FF90EF90DF90CF900895CF923F
:10F7A000DF92EF92FF920F931F93CF93DF93EC01C1
:10F7B0007A018B016C01C40ED51ECC15DD05A1F0BC
:10F7C0000E94837B80EF0E94987B8D2F0E94987B04
:10F7D0008C2F0E94987B2196F80181918F010E94C5
:10F7E000987B0E94817BE9CFC701DF91CF911F9168
:10F7F0000F91FF90EF90DF90CF9008951F93CF93DC
:10F80000DF93D82F192FC62F0E94837B80EF0E9491
:10F81000987B812F0E94987B8D2F0E94987B8C2F44
:10F820000E94987B0E94817B81E0DF91CF911F91A4
:10F830000895EF92FF920F931F93CF93C82F7B01F0
:10F8400080E590E00E94229168E270E08C2F0E9497
:10F85000B51C082F69E270E08C2F0E94B51C282F80
:10F86000302FB90121E030E0A7018C2F0E94919147
:10F870000E942D1D81E090E0CF911F910F91FF908C
:10F88000EF900895CF93DF931F92CDB7DEB7FC01C1
:10F89000218D328D8FEF9FEF232B41F0BE016F5FE3
:10F8A0007F4F808D0E94197C898190E00F90DF91BD
:10F8B000CF910895FF920F931F93CF93DF93F82E6C
:10F8C00080E590E00E94229110E000E08F2D0E94E0
:10F8D000E470EC01892B21F08F2D0E94E4708C01E3
:10F8E000C017D10799F70E942D1DCE01DF91CF914E
:10F8F0001F910F91FF900895AF92BF92CF92DF9228
:10F90000EF92FF921F93CF93DF93182F6B017A0131
:10F9100080E590E00E942291B12CA12C812F0E94C1
:10F92000E470EC01892B21F0812F0E94E4705C01CE
:10F93000CA15DB0599F72097F9F463E070E0812F91
:10F940000E94B51C843159F0882349F0C1E0D0E011
:10F950008C3111F4D0E0C0E0D195C195D1090E945D
:10F960002D1DCE01DF91CF911F91FF90EF90DF9081
:10F97000CF90BF90AF900895EC16FD060CF4E70110
:10F980001C161D0664F768E270E0812F0E94B51C0A
:10F99000E82E69E270E0812F0E94B51C282F3E2DD1
:10F9A00079019E01A601B701812F0E949191EC0E71
:10F9B000FD1E4F2D68E270E0812F0E94AB1C4E2D82
:10F9C00069E270E0812F0E94AB1C60E470E0812F3F
:10F9D0000E948191C4CFCF93DF93FC01218D328DA2
:10F9E0002115310529F48FEF9FEFDF91CF91089515
:10F9F000EC01808D4217530708F0A9010E947C7C1E
:10FA00001816190684F7298D3A8D281B390B3A8F61
:10FA1000298FEBCF0F931F93CF93DF931F92CDB717
:10FA2000DEB7FC01218D328D232B41F48FEF9FEF48
:10FA30000F90DF91CF911F910F9108958C0141E0BC
:10FA400050E0BE016F5F7F4FFC01808D0E947C7C87
:10FA5000181619065CF7F801818D928D0197928F27
:10FA6000818F898190E0E4CF0F931F93CF93DF9331
:10FA700000D000D01F921F92CDB7DEB78C01D80105
:10FA800059968D919C915A97892B41F0ED91FC915B
:10FA90000284F385E02DC8011995F1CFF801808D1E
:10FAA0000E945A7C18161906B4F548E050E0BE01D1
:10FAB0006F5F7F4FD80158968C910E947C7C1816FE
:10FAC0001906F4F4D801509684E0FE0131960190B5
:10FAD0000D928A95E1F78D8190E0982F88272E81ED
:10FAE000820F911DF801958B848B8F81282F30E038
:10FAF000322F22278885820F932F911D928F818F1D
:10FB000028960FB6F894DEBF0FBECDBFDF91CF9120
:10FB10001F910F91089590E080E0F2CF4F925F9295
:10FB20006F927F928F929F92AF92BF92CF92DF920D
:10FB3000EF92FF920F931F93CF93DF93CDB7DEB772
:10FB400063970FB6F894DEBF0FBECDBF7C016B018B
:10FB50003A01FB0120E090E080E06AE0319133233C
:10FB600009F461C040ED430F4A3008F04DC0689F72
:10FB7000A001699F500D1124CA01C097830F911DE8
:10FB800037FD9A958F3F910549F340F3F701428184
:10FB900053816481758180912B0890912C08A091EC
:10FBA0002D08B0912E08481759076A077B0709F4FA
:10FBB0002EC28701085F1F4F0E94FB966F70772748
:10FBC0007C5FC8010E94C813813009F025C285EA14
:10FBD00093E09A838983F70182819381A481B5811F
:10FBE0008B839C83AD83BE8345E350E0BE016F5F92
:10FBF0007F4FC8010E942F71892BA9F5D12CC12CF0
:10FC0000C8010E94B31317C03E3209F0BFCF2330A2
:10FC100009F4BCCFD301A20FB11D12968C932F5FB4
:10FC200090E080E09BCF233009F0B0CFF3018583D3
:10FC3000CC24C394D12CC60163960FB6F894DEBFD2
:10FC40000FBECDBFDF91CF911F910F91FF90EF902D
:10FC5000DF90CF90BF90AF909F908F907F906F90EC
:10FC60005F904F9008950E94FB96F701778366831B
:10FC70007627672776277A83698342E050E0BE01C2
:10FC80006F5F7F4FC8010E94657181E090E09E87A1
:10FC90008D8742E050E0BE01635F7F4FC8010E9444
:10FCA000657180E091E09E878D8742E050E0BE0163
:10FCB000635F7F4FC8010E9465711E861D8642E00A
:10FCC00050E0BE01635F7F4FC8010E94657142E052
:10FCD00050E0BE01635F7F4FC8010E94657142E042
:10FCE00050E0BE01635F7F4FC8010E9465715601FD
:10FCF000F6018081882301F16501F60181912F01D0
:10FD0000882311F08E32B1F446018A189B0818142A
:10FD1000190474F48F8641E050E0BE01615F7F4FAB
:10FD2000C8010E946571A401B501C8010E946571F6
:10FD30005201DECF6201E1CF1F8641E050E0BE01FB
:10FD4000615F7F4FC8010E946571C12CDD24D3948F
:10FD5000DE86CD8642E050E0BE01635F7F4FC80182
:10FD60000E946571DE86CD8642E050E0BE01635F91
:10FD70007F4FC8010E946571C8010E94F770892BEE
:10FD800009F43CCFF3E0AF2EB12C230122E0420E68
:10FD9000511CEEC0F7014281538164817581808DD1
:10FDA000918DA28DB38D481759076A077B0709F01B
:10FDB00024C1848D958DC59709F01FC181A192A1A1
:10FDC0005DEFC52EDD24DA940C970CF4C5C04CE031
:10FDD00050E0BE016F5F7F4FC8010E94EB7C8B81BA
:10FDE0009C819827892798279A8B898B29813A812A
:10FDF000322723273227F7014681578142175307BD
:10FE000009F000C197FFFEC08F7092703BEFC32EC8
:10FE1000DD24DA94892B09F09FC06F8078847624E2
:10FE2000672476242AEFC22EDD24DA94611471044B
:10FE300009F492C0D12CC12C8D819E8198278927ED
:10FE40009827C816D90640F541E050E0BE01635F2F
:10FE50007F4FC8010E94EB7C8D85882351F08D85F2
:10FE60009FEF980F9D87882321F0C8010E940A7D8B
:10FE7000F6CF8D858111E8CFC8010E940A7DC801A7
:10FE80000E940A7DC8010E940A7DC8010E940A7D65
:10FE9000FFEFCF1ADF0AD0CF912C812C41E050E048
:10FEA000BE016D5E7F4FC8010E94EB7C8B89982F4D
:10FEB000907C61F4882389F08B899FEF980F9B8B4E
:10FEC000882341F0C8010E940A7DF6CFC8010E9434
:10FED0000A7D1B8A8B898111E1CF42E050E0BE018F
:10FEE000615F7F4FC8010E94EB7C42E050E0BE01A1
:10FEF000635F7F4FC8010E94EB7CC8010E940A7DAE
:10FF0000C8010E940A7DC8010E940A7DC8010E94A2
:10FF10000A7D42E050E0BE016F5E7F4FC8010E9443
:10FF2000EB7C8F8598898115914009F040C0CD8484
:10FF3000DE84DC24CD24DC2481E0C816D104B9F5AC
:10FF400089899A898115944009F04EC044E050E0B7
:10FF5000B201C8010E94EB7C0E949A5B81E0A81A62
:10FF6000B10809F44DCEFFEFCF16DF0609F048CEF9
:10FF70000E94FB963B014C01C8010E94347D18167B
:10FF800019060CF407CF0E94FB96661977098809B9
:10FF90009909613A7F408105910558F50E949A5B65
:10FFA00061E070E080E090E00E94B694E5CFD12C53
:10FFB000C12C89899A89982789279827C816D90634
:10FFC00038F4C8010E940A7DFFEFCF1ADF0AF1CF93
:10FFD0002FEF821A920A6814790409F05FCF96EF26
:10FFE000C92EDD24DA94B8CFE7EFCE2EDD24DA94E3
:10FFF000B3CFCC24CA94DC2CAFCF6EEFC62EDD2459
:020000021000EC
:10000000DA94AACF4CEFC42EDD24DA94A5CF8EEF7C
:10001000C82EDD24DA940FCED12CC12C0CCE2F9219
:100020003F924F925F926F927F928F929F92AF9288
:10003000BF92DF92EF92FF920F931F93CF93DF93C4
:10004000CDB7DEB7E4970FB6F894DEBF0FBECDBFD5
:100050007C014A015B0119010E94FB962B013C01C6
:1000600087010D5B1F4FC8010E94347D18161906C9
:100070009CF00E94FB9664197509860997098616FB
:100080009706A806B90608F488C162E370E080E02C
:1000900090E00E94B694E7CF42E250E0BE016F5F6D
:1000A0007F4FC8010E94EB7C89818230D1F0D12C36
:1000B0008D2DE4960FB6F894DEBF0FBECDBFDF9155
:1000C000CF911F910F91FF90EF90DF90BF90AF9075
:1000D0009F908F907F906F905F904F903F902F9068
:1000E0000895F801848995898334910501F76D811C
:1000F0007E818F8198850E944BC52B013C01F101C7
:10010000408251826282738246E050E0B701685FAC
:100110007F4FCE014D960E9453C9892B41F6F701BE
:1001200080819181A281B381481659066A067B06B7
:1001300008F4BDCF84819581A681B781841595058A
:10014000A605B70508F4B3CF89899A89AB89BC891C
:1001500086879787A08BB18B8EECA82EB12CC80117
:100160000E940A7DF1E0AF1AB108C9F7D12CC7018E
:1001700082969AA789A7F701B696FCA7EBA70896DF
:100180009EA78DA73C974F01899698AB8FA738976C
:10019000FAABE9AB1701F6E12F0E311CC5979CAB0A
:1001A0008BABF801818D928D181619060CF080CF5B
:1001B000C8010E940A7D8333910509F4D4C0A4F5D7
:1001C0008130910509F474C074F4892B51F3C8018E
:1001D0000E940A7DB82EBA94FFEFBF1611F3C80132
:1001E0000E940A7DF8CF8330910509F46CC0069710
:1001F00071F7C8010E940A7DA82E44E050E06BA967
:100200007CA9C8010E94EB7C712C612CEA2DE45082
:10021000FF0B5F016A147B0424F6C8010E940A7D6B
:10022000FFEF6F1A7F0AF6CF8A33910509F46FC08A
:1002300074F585339105A1F1C69749F6C8010E946E
:100240000A7DB82EF701828D811109C0838D81113D
:1002500006C0848D811103C0858D8823A1F0EFA590
:10026000F8A94080518062807380B401CE018396EA
:100270000E9433778DA19EA1AFA1B8A584159505E5
:10028000A605B705D9F544E050E0B40118C08B339A
:10029000910509F452C08F3F910509F482CF97CFA1
:1002A000C8010E940A7DC8010E940A7DD82E79CF1C
:1002B000C8010E940A7D44E050E069A97AA9C801FA
:1002C0000E94EB7C6ECFC8010E940A7DA82E44E0FC
:1002D00050E0B101C8010E94EB7C712C612C8A2D89
:1002E0008450990B5C016A147B040CF05ACFC8014E
:1002F0000E940A7D9FEF691A790AF5CFBA94FFEF41
:10030000BF1609F44ECFC8010E940A7DF7CFC8017D
:100310000E940A7D44E050E06BA57CA5C8010E94C4
:10032000EB7CF70166A177A180A591A50E944BC542
:1003300066A377A380A791A734CFC8010E940A7D46
:1003400044E050E06DA57EA5C8010E94EB7CF7015A
:1003500062A573A584A595A50E944BC562A773A746
:1003600084A795A71ECFC8010E940A7D44E050E0F3
:1003700069A57AA5C8010E94EB7CF70162A173A16F
:1003800084A195A10E944BC562A373A384A395A3E6
:1003900066A777A780AB91AB04CFDD24DA9488CE33
:1003A0002F923F924F925F926F927F928F929F9285
:1003B000AF92BF92CF92DF92EF92FF920F931F9373
:1003C000CF93DF9300D000D0CDB7DEB78C010E9471
:1003D000ABB82FEC37E040E050E00E94DAC4DC011B
:1003E000CB010196A11DB11DF80184839583A683DD
:1003F000B78380839183A283B3835801F3E4AF0E64
:10040000B11CC5010E94B31364E470E0C5010E94F1
:10041000C813882309F445C10E94FB962B013C01B7
:10042000480182E4880E911C48EEC42E43E0D42E8D
:10043000E12CF12C52E0252E1E821D82D4018C91DC
:100440008330B1F1811166C0F80184819581A68164
:10045000B7810196A11DB11D84839583A683B783BF
:100460000E94FB966419750986099709A7019601F0
:100470000E94B8C4A90161E0C8010E949D7181E099
:10048000D4018C938D819E810197C1F20E94FB96CD
:100490006419750986099709D801D6962D913D9161
:1004A0004D915C91D997261737074807590720F6D1
:1004B000C5010E94B313F80184819581A681B7819B
:1004C0000196A11DB11D84839583A683B7830E94E5
:1004D000FB96F801FE9660837183828393838D81FE
:1004E0009E8126960FB6F894DEBF0FBECDBFDF917A
:1004F000CF911F910F91FF90EF90DF90CF90BF9021
:10050000AF909F908F907F906F905F904F903F90B3
:100510002F9008958430F1F4F80184819581A681AB
:10052000B7810196A11DB11D84839583A683B783EE
:100530000E94FB966419750986099709A70196011F
:100540000E94B8C4A90163E0C8010E949D71D40152
:100550002C9298CF813051F5F80142AD53AD64AD86
:1005600075AD9E012F5F3F4FC8010E940F80382E4E
:10057000F2E08F1390C089819A81AB81BC81F80130
:1005800084839583A683B7830E94FB9664197509BB
:1005900086099709A70196010E94B8C4A90163E0E2
:1005A000C8010E949D71D4013C926CCF823009F049
:1005B00069CFF80142AD53AD64AD75AD9E012F5FBB
:1005C0003F4FC8010E940F80382EF5E08F135DC0A9
:1005D000E3E0D401EC93F80182A193A1A4A1B5A119
:1005E000892B8A2B8B2B41F484E893E0A0E0B0E0C8
:1005F00082A393A3A4A3B5A3F80186A197A1A0A564
:10060000B1A5892B8A2B8B2B61F482A193A1A4A184
:10061000B5A1B695A7959795879586A397A3A0A70B
:10062000B1A7F80182A593A5A4A5B5A5892B8A2B0E
:100630008B2BA9F482A193A1A4A1B5A1AC01BD010A
:1006400023E076956795579547952A95D1F7841BB2
:10065000950BA60BB70B82A793A7A4A7B5A7F80184
:1006600086A197A1A0A5B1A586A797A7A0ABB1AB7E
:1006700082A593A5A4A5B5A582AB93ABA4ABB5AB5E
:1006800081E090E09E838D83FDCE96E0891303C0C8
:10069000D4011C92F7CEBFEF3B12F4CEF4011082CE
:1006A000F1CE1E821D821BCFCF93C82F80E590E034
:1006B0000E94229160E170E08C2F0E9481914FEFA7
:1006C00062E070E08C2F0E94AB1CCF910C942D1D2A
:1006D000FF920F931F93CF93DF93C82FD62F8A01DA
:1006E000F22E0E94548380E590E00E9422914D2FCB
:1006F0004F2970E060E08C2F0E94AB1C01151105A2
:10070000D1F0412F64E070E08C2F0E94AB1C402F91
:1007100065E070E08C2F0E94AB1C61E070E08C2FD4
:100720000E9481910E942D1D81E0DF91CF911F9148
:100730000F91FF9008950091A2061091A3060F5FFC
:100740001F4F1093A3060093A206DBCFBF92CF9258
:10075000DF92EF92FF920F931F93CF93DF9300D01E
:1007600000D0CDB7DEB7FC01208D243009F05DC08C
:100770006A017B018C01B12C63E070E08B2D0E943B
:10078000B51C81114AC0F801B08EF801808D84300B
:1007900009F44BC096E0ECE9F2E0DE01119601901D
:1007A0000D929A95E1F7F70193819F779C8394814D
:1007B0009D8395819E83B7016E5F7F4F0E94E41CED
:1007C000B601F801808D0E94D31CF801808D90E065
:1007D000982F882746E050E0BE016F5F7F4F8A5F09
:1007E0009B4F0E94CF7BF801128E118E20E8A6014C
:1007F00062E0808D0E94688381E026960FB6F894AF
:10080000DEBF0FBECDBFDF91CF911F910F91FF9043
:10081000EF90DF90CF90BF900895883109F4B3CF67
:10082000B394F4E0BF12A8CFB0CF80E0E6CFCF936F
:10083000C82F80E590E00E94229163E070E08C2F49
:100840000E94B51CC82F0E942D1D8C2FCF9108959A
:100850008F7099278230910518F0029761F0089502
:1008600080917D0890917E08DC01ED91FC910680DD
:10087000F781E02D199480917F089091800800976E
:1008800091F0DC01ED91FC91008CF18DE02D19953A
:1008900080917F0890918008DC01ED91FC910488A3
:1008A000F589E02DE7CF08958F929F92AF92BF9286
:1008B000CF92DF92EF92FF92CF93DF93EC014A0148
:1008C0005B01C12CD12C7601CE010E94F51C88233E
:1008D00099F0C814D904EA04FB0474F4CE010E9410
:1008E0005414892B89F38FEFC81AD80AE80AF80A3A
:1008F000CE010E943A14E8CFDF91CF91FF90EF90A4
:10090000DF90CF90BF90AF909F908F9008952F92DF
:100910003F924F925F926F927F928F929F92AF928F
:10092000BF92CF92DF92EF92FF920F931F93CF93DC
:10093000DF9300D000D01F921F92CDB7DEB78C019D
:100940006B010E94BB79019619F48FEF9FEF1DC0D8
:10095000D801ED91FC910284F385E02DC801199531
:100960007C018F3F980789F3D801ED91FC910684B3
:10097000F785E02D682FC8011995B2E2EB16F10456
:10098000E9F4B601C8010E94D87928960FB6F89408
:10099000DEBF0FBECDBFDF91CF911F910F91FF90B2
:1009A000EF90DF90CF90BF90AF909F908F907F900F
:1009B0006F905F904F903F902F900895EDE2EE166C
:1009C000F10429F0C701C0970A9708F043C1D80184
:1009D000ED91FC910284F385E02DC80119957C010D
:1009E0008F3F980709F4B1CF8D9799F5D801ED9114
:1009F000FC910284F385E02DC80119957C010196D4
:100A000009F4A3CFEFEFFFEFF887EF83C701C0979B
:100A1000812C912C54010A9708F5AAE0B0E0A501B9
:100A200094010E94F9C430E3E31AF1084701FF0C76
:100A3000AA08BB08860E971EA81EB91ED801ED9104
:100A4000FC910284F385E02DC80119957C01C097C3
:100A5000E2CF21E030E038872F83D8CFBEE2EB161B
:100A6000F10401F1C7018F7D85349105D9F0AF8183
:100A7000B885A50194010E9404C5F60161877287BB
:100A8000838794878085807F82608087D801ED91FD
:100A9000FC910684F785E02D6E2DC801199590E034
:100AA00080E073CFC501B4010E9475C32B013C01E6
:100AB000312C212CFEE2EF16F10499F5D801ED91CD
:100AC000FC910284F385E02DC80119957C01312C3D
:100AD000212C20E030E040E251E4C301B2010E9449
:100AE000D4C34B015C01B70160537109072E000CA0
:100AF000880B990B0E9475C3A50194010E9462C5E1
:100B00002B013C01B1E02B1A3108D801ED91FC9189
:100B10000284F385E02DC80119957C01C0970A97DE
:100B2000C0F2C7018F7D8534910509F040C0D8011E
:100B3000ED91FC910284F385E02DC80119957C01AB
:100B4000D801ED91FC918B32910519F50284F38562
:100B5000E02DC80119957C01E1E0EE83B12CA12CB8
:100B60008AE0982ED801ED91FC91C701C0978A3098
:100B7000910508F59A9C90019B9C300D11245C0115
:100B8000A20EB31E0284F385E02DC80119957C01E5
:100B9000E9CF8D9749F40284F385E02DC8011995BA
:100BA0007C013FEF3E83DACF81E08E83D7CFB1E087
:100BB000BE83B12CA12CEF81F885BF01FF0F880BFC
:100BC000990B0E9475C3A30192010E94D4C32B010B
:100BD0003C01B501BB0C880B990B0E9475C34B01FE
:100BE0005C01FE816F2FFF0F770B880B990B0E9422
:100BF00075C39B01AC01C501B4010E94D4C34B0174
:100C00005C01B101330C880B990B0E9475C39B01E9
:100C1000AC01C501B4010E9462C59B01AC0160E05A
:100C200070E080E291E40E947BC69B01AC01C301AD
:100C3000B2010E94D4C3D60119966D937D938D9312
:100C40009C931C9718968C911897807F83601896B8
:100C50008C931CCFBBE5EB16F10409F062C0D80100
:100C6000ED91FC910284F385E02DC80119958B3537
:100C7000910509F06ACEF6018085807F85608087C6
:100C8000C8010E94BB79D801ED91FC910284F385E3
:100C9000E02DC80119958D35910509F400CFD801D3
:100CA000ED91FC910684F785E02D682FC801199518
:100CB000BB24BA940E94987A7C01009709F445CE2F
:100CC000BB2031F1F60197838683C8010E94BB796E
:100CD000B701C8010E948784892B09F036CEC8016C
:100CE0000E94BB79D801ED91FC910284F385E02D3F
:100CF000C8011995B12C47018C329105D9F221E038
:100D000030E08D35910509F08DC030E020E08AC0DB
:100D1000D40113969C938E931297FC019582848242
:100D2000D4CFBBE7EB16F10409F08AC0D801ED91EE
:100D3000FC910284F385E02DC80119958B3791054C
:100D400009F003CEF6018085807F86608087C80128
:100D50000E94BB79D801ED91FC910284F385E02DCE
:100D6000C80119958D37910509F499CED801ED91F7
:100D7000FC910684F785E02D682FC8011995992408
:100D80009A940E94987A7C01009709F4DECD99200C
:100D900009F44DC0F60197838683C8010E94BB7990
:100DA000B701C8010E94D879019609F4CECDC801D7
:100DB0000E94BB79D70119968D919C911A97119633
:100DC0009C938E931A961C921E921997D801ED91BE
:100DD000FC910284F385E02DC8011995CA9709F0AA
:100DE000B4CDC8010E94BB79B701C8010E948784B5
:100DF000019609F4AACDC8010E94BB79D801ED91F2
:100E0000FC910284F385E02DC8011995912C5701BE
:100E10008C32910509F4B5CF21E030E08D37910592
:100E200009F473CF88279927821B930BAECDD50188
:100E300013969C938E931297FC01B582A482ADCF3A
:100E4000BEE6EB16F10421F519821A821B821C8280
:100E5000D801ED91FC910484F585E02D44E050E04B
:100E6000BE016F5F7F4FC8011995049709F06DCDE2
:100E700044E050E060E275E0CE0101960E94C4C9F2
:100E8000009709F062CDF6012085207F20877DCD77
:100E9000F6E6EF16F10441F59E012F5F3F4F790111
:100EA00085E0D9011D928A95E9F7D801ED91FC9171
:100EB0000484F585E02D45E050E0B901C80119959D
:100EC000059709F042CD45E050E06AE275E0C701C0
:100ED0000E94C4C9009709F038CDF6012085207F13
:100EE00021602087118651CDF4E7EF16F10409F057
:100EF0002CCD19821A821B821C82D801ED91FC91A3
:100F00000484F585E02D44E050E0BE016F5F7F4F23
:100F1000C8011995049709F018CD44E050E065E246
:100F200075E0CE0101960E94C4C9009709F00DCD6D
:100F3000F6012085207F2160208721E0218725CDB3
:100F40000F931F93CF93DF938B01FC01C681D78151
:100F5000209759F0B801888199810E947BC9892B1B
:100F600021F00A80DB81C02DF3CFCE01DF91CF913C
:100F70001F910F910895809147089091480800971C
:100F800011F480E02FC0DC01ED91FC910688F78917
:100F9000E02D199520916A0830916B0881111FC0CE
:100FA000232B79F78DEF9FEF90936B0880936A085E
:100FB0008091470890914808DC01ED91FC910680F2
:100FC000F781E02D19958091470890914808DC0140
:100FD000ED91FC910488F589E02D1995D2CF81E03F
:100FE000232B79F60895CF93DF93EC01FA01329623
:100FF000E60FF71FDC019D012C1B3D0BCF01861B6B
:10100000970B4D91442311F04193F5CFAC01421B56
:10101000530B640F751FFB013297308361507109C8
:10102000FB012083DF91CF910895FC018681978198
:10103000009739F0662329F06150FC018281938189
:10104000F7CF0895CF92DF92EF92FF92DC011196D5
:10105000EC911197E295EF70EC3098F4F0E088276E
:10106000EB5CF7478F4F0C9443C598885B885B888F
:101070004188418841887E885F88418841884888C6
:1010800048888FEF9FEFFF90EF90DF90CF9008950B
:1010900014968D919D910D90BC91A02DB7FD48C0E7
:1010A0008F3F9105A105B10571F36CF38FEF90E0CF
:1010B000A0E0B0E0E8CF14968C9190E0E4CF1496D5
:1010C000CD90DD90ED90FC90179720E030E0A901E5
:1010D000C701B6010E946EC387FD2AC020E030E040
:1010E0004FE753E4C701B6010E9476C618161CF1FB
:1010F000C701B6010E9440C6CB01C5CF14966D91C1
:101100007D918D919C9117976D392FEF7207820712
:10111000920774F0611524E67207810591055CF46D
:1011200024E630E040E050E00E94DAC4C901ABCFD1
:1011300090E080E0A8CF8FEF90E0A5CFEF92FF92F4
:101140000F931F93CF93DF937C018B01D0E0C0E01E
:10115000C7010E94557597FD07C0F80181938F0163
:101160002196C430D105A1F7CE01DF91CF911F9117
:101170000F91FF90EF9008950F931F93CF93DF93FC
:10118000CDB7DEB762970FB6F894DEBF0FBECDBF06
:101190008C01CB01F8011182108213821282158218
:1011A000148240E1BE016F5F7F4F0E94F2BABE0120
:1011B0006F5F7F4FC8010E94D57462960FB6F89496
:1011C000DEBF0FBECDBFDF91CF911F910F9108956C
:1011D000E091A008F091A108128A118A148A138A5A
:1011E00024E830E035872487168620E030E3308B12
:1011F0002787858B81E090E00895CF93DF938091DE
:10120000A0089091A108892B99F182E70E94E888B3
:101210008091A0089091A108DC01ED91FC910088DB
:10122000F189E02D70E060E01995CEEBD2E080917D
:10123000A0089091A108DC01ED91FC91B2E0C23CC4
:10124000DB07C1F00284F385E02D19952991022E68
:10125000000C330B8217930751F38091A0089091F3
:10126000A108DC01ED91FC910488F589E02D199528
:1012700080E005C00488F589E02D199581E0DF91B3
:10128000CF910895AF92BF92CF92DF92EF92FF92EB
:101290000F931F93CF93DF935C017B018B01040FAE
:1012A000151FEB016E01CE18DF08C017D10741F002
:1012B000C5010E9455751816190614F48993F2CFCA
:1012C000C601DF91CF911F910F91FF90EF90DF90BA
:1012D000CF90BF90AF900895CF93DF932091A00857
:1012E0003091A108232B11F480E041C0EC010E9451
:1012F000FD888823C9F3FE0101900020E9F73197AA
:10130000EC1BFD0B709780F782E70E94E8888091C4
:10131000A0089091A108DC01ED91FC910088F18971
:10132000E02D60E470E01995BE018091A0089091D5
:10133000A1080E9497768091A0089091A108DC01F5
:10134000ED91FC910190F081E02D60E01995EC01A8
:101350008091A0089091A108DC01ED91FC91048896
:10136000F589E02D199581E0CD2B09F4BDCFDF91F2
:10137000CF910895CF93DF932091A0083091A108D9
:10138000232B11F480E041C0EC010E94FD888823EA
:10139000C9F3FE0101900020E9F73197EC1BFD0B2A
:1013A000709780F782E70E94E8888091A00890916A
:1013B000A108DC01ED91FC910088F189E02D60E548
:1013C00070E01995BE018091A0089091A1080E943B
:1013D00097768091A0089091A108DC01ED91FC9195
:1013E0000190F081E02D60E01995EC018091A0085A
:1013F0009091A108DC01ED91FC910488F589E02D24
:10140000199581E0CD2B09F4BDCFDF91CF910895DF
:101410000F931F93CF93DF9300D01F92CDB7DEB70A
:10142000FC0182819381A481B58189839A83AB83F6
:10143000BC838091A0089091A108892B11F480E0D1
:1014400033C00E94FD888823D1F382E70E94E88898
:101450008091A0089091A108DC01ED91FC91008899
:10146000F189E02D60E170E019958091A0089091DC
:10147000A108DC01ED91FC910280F381E02D44E0B4
:1014800050E0BE016F5F7F4F19958C018091A008DD
:101490009091A108DC01ED91FC910488F589E02D83
:1014A000199581E0012B59F20F900F900F900F903A
:1014B000DF91CF911F910F9108950F931F93CF93B9
:1014C000DF9300D01F92CDB7DEB7FC0182819381FC
:1014D000A481B58189839A83AB83BC838091A00862
:1014E0009091A108892B11F480E033C00E94FD88FF
:1014F0008823D1F382E70E94E8888091A008909128
:10150000A108DC01ED91FC910088F189E02D6CE1EE
:1015100070E019958091A0089091A108DC01ED91EF
:10152000FC910280F381E02D44E050E0BE016F5F4A
:101530007F4F19958C018091A0089091A108DC0142
:10154000ED91FC910488F589E02D199581E0012B3E
:1015500059F20F900F900F900F90DF91CF911F9144
:101560000F9108950F931F93CF93DF9300D01F9295
:10157000CDB7DEB7FC0182819381A481B5818983D7
:101580009A83AB83BC838091A0089091A108892B9A
:1015900011F480E033C00E94FD888823D1F382E7F4
:1015A0000E94E8888091A0089091A108DC01ED914B
:1015B000FC910088F189E02D64E170E0199580913B
:1015C000A0089091A108DC01ED91FC910280F381CB
:1015D000E02D44E050E0BE016F5F7F4F19958C0114
:1015E0008091A0089091A108DC01ED91FC91048804
:1015F000F589E02D199581E0012B59F20F900F909C
:101600000F900F90DF91CF911F910F9108950F933D
:101610001F93CF93DF9300D01F92CDB7DEB7FC01AD
:1016200082819381A481B58189839A83AB83BC83B2
:101630008091A0089091A108892B11F480E033C01B
:101640000E94FD888823D1F382E70E94E888809178
:10165000A0089091A108DC01ED91FC910088F1892E
:10166000E02D68E170E019958091A0089091A108A3
:10167000DC01ED91FC910280F381E02D44E050E02B
:10168000BE016F5F7F4F19958C018091A0089091EA
:10169000A108DC01ED91FC910488F589E02D1995F4
:1016A00081E0012B59F20F900F900F900F90DF9176
:1016B000CF911F910F910895CF93DF9300D01F9288
:1016C000CDB7DEB719821A821B821C8287E7898315
:1016D0008091A0089091A108892B41F10E94FD887A
:1016E000882321F182E70E94E8888091A0089091E8
:1016F000A108DC01ED91FC910088F189E02D6CE0FE
:1017000070E01995BE016F5F7F4F8091A0089091A6
:10171000A1080E949E888091A0089091A108DC01F8
:10172000ED91FC910488F589E02D199569817A8104
:101730008B819C810F900F900F900F90DF91CF9134
:1017400008950F931F93CF93DF9300D01F92CDB7CF
:10175000DEB769837A838B839C838091A008909104
:10176000A108892B11F480E033C00E94FD888823F2
:10177000D1F382E70E94E8888091A0089091A108A7
:10178000DC01ED91FC910088F189E02D6CE070E0C6
:1017900019958091A0089091A108DC01ED91FC9130
:1017A0000280F381E02D44E050E0BE016F5F7F4F87
:1017B00019958C018091A0089091A108DC01ED9110
:1017C000FC910488F589E02D199581E0012B59F2EF
:1017D0000F900F900F900F90DF91CF911F910F916D
:1017E0000895CF93C82F0E945C8B677FC0FF68600D
:1017F000CF910C94A18BCF93C82F0E945C8BC770A4
:10180000687F6C2BCF910C94A18BCF93C82F0E9433
:101810005C8BC770C295C07F6F786C2BCF910C9496
:10182000A18B61157105C1F0DC011696ED91FC915B
:101830001797309731F417967C936E931697089507
:10184000FC01828193810097D9F773836283DB0166
:101850001596FC93EE93149708952AE00C94BA75AC
:10186000462F50E070E060E02AE00C94BA75AB01BE
:10187000770F660B770B2AE030E00C941176DC01D1
:101880001696ED91FC9180E0309729F08F5F0280F1
:10189000F381E02DF9CF0895CF93DF93FC01C2814E
:1018A000D3812097C1F088858F70823029F4898593
:1018B0009A85DF91CF910895853069F4CE010E9419
:1018C0003F8C882341F060E0CE010E941588FC0126
:1018D00081859285EECF90E080E0EBCFDF92EF92B2
:1018E000FF920F931F93CF93DF93EC017B0140E0B6
:1018F00052E00E94862FD82E811171C06EE77EE1E2
:1019000085E799E00E94FD76D70119968D919C910B
:10191000009709F441C0DC01ED91FC91028CF38D3C
:10192000E02D19958C0180E00231110520F4F801B9
:10193000E455FD4F8081982F9295907F89818F701B
:10194000892B898363E77EE185E799E00E94FD7634
:10195000B80185E799E00E94378C6BE67EE185E768
:1019600099E00E94FD76698162956F7085E799E044
:101970000E94308C85E799E00E94067689818295E5
:101980008F70843068F4823098F58130B9F11C8210
:101990001D821E821F8215C0F701008510E0C3CF93
:1019A000883039F0893099F780E090E0A6E9B2E418
:1019B00004C080E090E0A0EAB1E48C839D83AE8314
:1019C000BF8340E052E0B701CE010E940F2FCE014D
:1019D0000E94112E60E07AE0C7010E941A388D2D16
:1019E000DF91CF911F910F91FF90EF90DF900895BD
:1019F00084E68E838F818E7F8F831D828FEF8C8311
:101A0000E0CF8F929F92AF92BF92CF92DF92EF92F0
:101A1000FF920F931F93CF93DF93CDB7DEB7C454DC
:101A2000D1090FB6F894DEBF0FBECDBF25967FAFAC
:101A30006EAF259723961FAE1EAE2397672B09F432
:101A400078C2FC012385222339F09C01255F3F4F9A
:101A500023963FAF2EAF23975C012396EEADFFADEB
:101A600023973097F1F4F501E38CF48CE114F10441
:101A700019F510E000E02596CEACDFAC25974601C5
:101A8000800E911EF4018081882309F45DC0082E28
:101A9000000C990B0E9431C9F40180830F5F1F4F26
:101AA000EACF80818823F9F2CE018F5B9F4F0E949D
:101AB000BE357C01892BB9F2FCE0EF16F104C9F6C2
:101AC00025962EAD3FAD259719861A861B861C8656
:101AD0001D861E861F86188A8A858F70806C8A876D
:101AE0003E872D876CE0CE0109960E9450302983F5
:101AF0003A834B835C836D837E838F8398872396A1
:101B0000EEACFFAC2397CC24C39409851A852B85B2
:101B10003C854D855E856F857889C5010E9480383A
:101B2000CC5BDF4F0FB6F894DEBF0FBECDBFDF91A9
:101B3000CF911F910F91FF90EF90DF90CF90BF90CA
:101B4000AF909F908F900895C114D10481F1F60158
:101B50008081882361F18D3209F47EC090ED980F69
:101B60009A3008F479C008E010E0853211F10EEFE8
:101B70001FEF8B37F1F007E110E08332D1F096E8E8
:101B8000892E9DE1992E01E010E0C4010E9486BAE1
:101B9000AC01B401C6010E949FBA892B51F00F5FBE
:101BA0001F4FF9E08F0E911C0931110571F70FEFEE
:101BB0001FEF19AE1AAE1BAE1CAE21961CAE1DAEA9
:101BC0001EAE1FAE21978AAD8F708AAF09AF85E038
:101BD000E816F10409F443C096E0E916F10411F4A3
:101BE00007E110E0DE2C6E2DCE01C9960E94503028
:101BF00029873A874B875C876D877E878F87988B8D
:101C00000A3011057CF5083011050CF06CC10E3F4F
